:100000005446495300010000E88B0200E640C63D1B
:10001000105402251910041242593059105402028A
:1000200019100412425930591054020219100412C6
:100030004259305903000000000000000000000099
:100040005446435300200000105F020000000000EF
:1000500000800110012100002521000029E6010097
:10006000292100002B2100002D2100003D2100004E
:100070003D2100003D2100003D2100002F21000016
:10008000312100003D21000033210000615F0000AC
:100090005B600000372100003D2100007952001014
:1000A00037210000694300006D4300003D2100003E
:1000B0003D210000775B0000B55200007143000055
:1000C000F5580000372100003D2100003D210000CF
:1000D0000000000000000000000000000000000020
:1000E0000000000000000000000000000000000010
:1000F0000000000000000000000000000000000000
:1001000000000000000000000000000000000000EF
:1001100000000000000000000000000000000000DF
:1001200000000000000000000000000000000000CF
:1001300000000000000000000000000000000000BF
:1001400000000000000000000000000000000000AF
:1001500000F003F800F020F8FEE70D480168890878
:100160008900002001C101C101C101C17047000027
:100170004C5B0010FEE7FEE7FEE7FEE7FEE7FEE76A
:10018000FEE7FEE7FEE703480047FEE7FEE7000064
:10019000202100003D21000000F002F800F068F886
:1001A0000AA090E8000C82448344AAF10107DA45D2
:1001B00001D100F05DF8AFF2090EBAE80F0013F0BC
:1001C000010F18BFFB1A43F0010318475800020043
:1001D000B80002000A444FF0000C10F8013B13F085
:1001E000070408BF10F8014B1D1108BF10F8015B90
:1001F000641E05D010F8016B641E01F8016BF9D183
:1002000013F0080F1EBF10F8014BAD1C0C1B09D1D9
:100210006D1E58BF01F801CBFAD505E014F8016B4B
:1002200001F8016B6D1EF9D59142D6D370470000DD
:10023000103A24BF78C878C1FAD8520724BF30C812
:1002400030C144BF04680C607047000000230024E4
:1002500000250026103A28BF78C1FBD8520728BFD6
:1002600030C148BF0B6070471FB51FBD10B510BD32
:10027000DFF80CD0FFF7F8FF05F0E2FD1CF0EEF917
:100280000080011003B4FFF7F1FF03BC1CF0EEF98E
:1002900008B500200346024600900121022000F02C
:1002A000F8FA08BD38B5FF4D0024FF48EC802C81DA
:1002B0006C81406980476861FF202871FB480023FA
:1002C0001A46046044608460C4600461012068715F
:1002D0002C706C7001460220009400F0DAFA0120C4
:1002E00038BD38B5EF4D02282C7922460DD00528AF
:1002F00010D0A24208BF38BD002003460246214666
:10030000009000F0C6FA2C7138BD022914BF0124F8
:100310000224EEE7022914BF04240824E9E708B503
:10032000009313460A460146012000F0B2FA08BDC8
:1003300008B50346009103220221012000F0A9FA2A
:1003400008BD38B500240CF017F9002818BF0124A7
:1003500010F026F9002818BF0224D2480178A142E3
:1003600008BF38BD047000200346022100902246D9
:10037000084600F08EFA38BD08B500210B4602464B
:1003800000910821022000F084FA08BD08B5002180
:100390000091002814BF0122002200230321022023
:1003A00000F077FA08BD08B500210B46024600911F
:1003B0000721022000F06DFA08BD08B500200346B1
:1003C000024600900421022000F063FA08BDB54BFC
:1003D00000285A7814BF0121002159708A4208BFB1
:1003E0007047021C18BF012208B500200346009088
:1003F0000921022000F04DFA08BDAA4840780028E3
:1004000018BF012070470120A64988707047A54891
:1004100080787047A3490020887070472DE9F0412B
:1004200004460127002503F007009E4E8846012858
:1004300004BF0020708148D0022846D170899A49B3
:1004400004280BD2002818BF306902D148688047C1
:10045000306110F8011B217030612FE0062809D2AD
:1004600088688047718980B2C1F10501C900C84020
:10047000207023E0082808D2086980477189C1F1FB
:100480000701C900C840207018E00C2808D248694C
:1004900080477189C1F10B01C900C84020700DE08F
:1004A0000E2808D2886980477189C1F10D01C90001
:1004B000C840207002E0FF20207000277089401C97
:1004C00080B270810E2828BF012588F80050384678
:1004D000BDE8F08130B403F007000024DFF8C4C1A8
:1004E000012804BFACF80640ACF80A401BD013F05A
:1004F000070F18D16B4BBCF80A00DB88022805D225
:10050000120242EA1322ACF8062009E003449D1EC1
:10051000B5F5806F04DADCF814502B4403F8022C94
:10052000401CACF80A000C7030BC00207047F0B4DE
:100530000746002003F007045A4D0646012C04BF6D
:100540006E81EE6025D0DFF85CC1022CBCF808C0DB
:1005500003D013F0070F0DD01BE06A890CEB0203E8
:10056000B3F5806F15D26869C05C3870501C688123
:1005700001200EE0120242EA1C222A81EB68012BC4
:1005800005D1B2F5806F24BF40F2FF322A815A1C98
:10059000EA600E70F0BC704738B503F00700002425
:1005A0000D46012809D13F4800231A464481C480E2
:1005B00019460220009400F06CF92C70002038BD20
:1005C0002DE9F04182B017460C0005464FF00008B7
:1005D00008BF002608D026783549012E18BF022E04
:1005E0004ED0032E5DD09EB985F8008085F801803D
:1005F000A5F80280A5F80480A5F80680A5F8088073
:10060000A5F80A80A5F80C80A87B20F00100A8734B
:10061000012E18BF032E06D00BF0FCFC002804BFEF
:1006200002B0BDE8F08105F01FFC05281CBF02B038
:10063000BDE8F081012E04BFC0208DF8000005D078
:10064000022E0CBFC220C1208DF8000060788DF80A
:10065000010060880123000A8DF80200A0788DF85F
:100660000300A0880622000A8DF8040020798DF886
:100670000500694607200FF050F802B0BDE8F08190
:100680006078421E05EB001000F8102C607805EB36
:10069000001000F80F6C08686288438BC08A5A43C8
:1006A00008E041E000840010E82002007C8800108F
:1006B0000888001092FBF0F0627805EB021222F835
:1006C0000E0C0868A288018B808A514391FBF0F0E0
:1006D000617805EB011121F80C0C6178A07905EB2C
:1006E000011121F80A0C6178207A05EB011121F83B
:1006F000080C6178607A05EB011121F8060C61782D
:10070000A07B05EB011121F8040CE0790528607845
:1007100005EB001010F8021C0CBF41F0010121F0A4
:10072000010100F8021C73E76078421E05EB00101F
:1007300000F8102C6278032005EB021202F80F0C6F
:1007400008686288438BC08A5A4392FBF0F0627853
:1007500005EB021222F80E0C0868A288018B808A31
:10076000514391FBF0F0617805EB011121F80C0C7D
:1007700005F07AFB052821D107B36178B87905EB3C
:10078000011121F80A0C6178387A05EB011121F882
:10079000080C6178787A05EB011121F8060CF879DC
:1007A0000528607805EB001010F8021C0CBF41F022
:1007B000010121F0010100F8021C17E0607805EB4F
:1007C000001020F80A8C607805EB001020F8088CE7
:1007D000607805EB001020F8068C607805EB0010BF
:1007E00010F8021C21F0010100F8021C607805EBF2
:1007F000001020F8048C0BE72B490020C8707047CC
:100800002948C078704728490120C8707047274B95
:1008100003EB80004254704700B583B001788DF837
:10082000001041788DF8011081788DF80210C178A0
:100830008DF8031001798DF8041041798DF80510B9
:1008400080798DF8060000208DF8070005F022FC65
:1008500001280CD11BF020FF012801BF9DF80000EA
:1008600046289DF80100012804BF03B000BD68467A
:100870001BF017FF03B000BD70470B49002818BFDD
:100880000120487170470848407970477047084810
:10089000704708B5DDF808C0CDF800C0DFF814C017
:1008A000DCF800C0E04708BD008400107C88001020
:1008B000B01B0200E82002007047FE48D0F8500349
:1008C00000F00100704770B5FA4D04000AD001F045
:1008D0008FFC38B9D5F8500310F0010F1CBF002071
:1008E000A86005D10120A860002C08BF002011D00D
:1008F000D5F8600310F0010F0BD1D5F8600340F07C
:100900000100C5F86003D5F8600320F00100C5F8C8
:1009100060030120286270BDE648006A002818BF05
:1009200001207047C00000F1804000F5A040416305
:100930007047C00000F1804000F5A040006B00F45B
:10094000807070471021C00000F1804000F5A04089
:1009500041637047D749D1F8402160F30D22C1F8B7
:1009600040217047D348D0F84001C0F305207047BC
:10097000D049D1F8402160F31742C1F840217047B7
:10098000CC48D0F84001C0F30740704700F00F0298
:1009900002EB42029201C0F3031002EB801000F15F
:1009A000804000F5A0400029D0F8401114BF41F06C
:1009B000010121F00101C0F84011704700F00F0162
:1009C00001EB41018901C0F3031001EB801000F13C
:1009D000804000F5A040D0F8400100F001007047D1
:1009E00000F00F0202EB42029201C0F3031002EB8F
:1009F000801000F1804000F5A0400029D0F840119F
:100A000014BF41F0020121F00201C0F8401170470B
:100A100000F00F0101EB41018901C0F3031001EB6C
:100A2000801000F1804000F5A040D0F84001C0F3F4
:100A30004000704770B4DFF880C286B00328DCE95C
:100A40000045DCF808600296CDE90045DCE9034585
:100A5000DCF814C0CDF814C0CDE9034522BF06B0C0
:100A600070BC7047032988BF0321FF2A88BFFF227B
:100A7000FF2B88BFFF235DF820C0DCF8004061F346
:100A80004614CCF8004003A951F82000016862F335
:100A900018410160016863F30801016006B070BC91
:100AA0007047844AD2F84403D2F87013C0F30B00A5
:100AB00011F0010F814940F2FF13096818D04FF07F
:100AC000320C01FB0CF100280EBF0121B1FBF0F14B
:100AD000491CFF2988BFFF21D2F870C361F3174C6E
:100AE000C2F870C3D2F824111943C2F8241105E0EA
:100AF000D2F824C161F3080CC2F824C1D2F8601303
:100B000011F0010F6D49496818D04FF0320C01FB0C
:100B10000CF100280EBF0121B1FBF0F1491CFF29A7
:100B200088BFFF21D2F860C361F3174CC2F860C3DD
:100B3000D2F8E4111943C2F8E41105E0D2F8E4C197
:100B400061F3080CC2F8E4C1D2F8681311F0010F88
:100B50005A49896804BFD2F8A40261F3080015D08D
:100B60004FF0320C01FB0CF100281ABFB1FBF0F082
:100B7000401C0120FF2888BFFF20D2F8681360F3D3
:100B80001741C2F86813D2F8A4021843C2F8A402AD
:100B90007047484900230B6202680A6042684A6055
:100BA00082688A60C268CA60426A0A64826A4A6469
:100BB00002698A614269CA61826B0A66826C0A674D
:100BC000C26C4A67026D8A67426DCA67826DC1F85E
:100BD0008020C26DC1F88420026EC1F88820426E68
:100BE000C1F88C20426FC1F8B020C26FC1F8B820A4
:100BF000C26EC1F8A820D0F89422C1F85023D0F8D2
:100C00009822C1F85423D0F89C22C1F85823D0F878
:100C1000A022C1F85C23D0F88420C1F8F020D0F8DD
:100C20008820C1F8F420D0F88C20C1F8F820D0F842
:100C30009020C1F8FC2021224A63CA63C2694A623B
:100C4000C26A8A64026BCA64026FC1F8AC20026A8D
:100C5000CA62426B0A65C26B4A66026C8A66426C63
:100C6000CA66826FC1F8B420D0F88020C1F8BC20D9
:100C7000D0F8A422C1F86023D0F8A822C1F86423D8
:100C8000D0F8AC22C1F86823D0F8B022C1F86C23A8
:100C9000D0F8B422C1F87023D0F8B822C1F8742378
:100CA000D0F8BC22C1F87823D0F8C022C1F87C2348
:100CB00006E0000000500040CC1B0200308900100C
:100CC000D0F88C2222F48032C1F84023D0F8902250
:100CD000C1F84C23D0F89420C1F80021D0F8982016
:100CE000C1F80421D0F89C20C1F80821D0F8A02038
:100CF000C1F80C21D0F8A420C1F81021D0F8A82008
:100D0000C1F81421D0F8C820C1F83421D0F8AC20A3
:100D1000C1F81821D0F8B020C1F81C21D0F8B420B7
:100D2000C1F82021D0F8B820C1F82421D0F8BC2087
:100D3000C1F82821D0F8C020C1F82C21D0F8C42057
:100D4000C1F83021D0F8CC20C1F84021D0F8D02013
:100D5000C1F84421D0F8D820C1F84C21D0F8E420C3
:100D6000C1F86021D0F8E820C1F86421D0F8EC2067
:100D7000C1F86821D0F8F020C1F86C21D0F8D42057
:100D8000C1F84821D0F8DC20C1F85021D0F8E0208B
:100D9000C1F85421D0F8F420C1F87021D0F8F8201F
:100DA000C1F87421D0F8FC20C1F87821D0F80021D6
:100DB000C1F87C21D0F83C21C1F8C021D0F84021F5
:100DC000C1F8C421D0F84421C1F8C821D0F8482185
:100DD000C1F8CC21D0F84C21C1F8D021D0F8502155
:100DE000C1F8D421D0F87021C1F8F421D0F85421F1
:100DF000C1F8D821D0F85821C1F8DC21D0F85C2105
:100E0000C1F8E021D0F86021C1F8E421D0F86421D4
:100E1000C1F8E821D0F86821C1F8EC21D0F86C21A4
:100E2000C1F8F021D0F87421C1F80022D0F878215F
:100E3000C1F80422D0F88021C1F80C22D0F88C210E
:100E4000C1F82022D0F89021C1F82422D0F89421B2
:100E5000C1F82822D0F89821C1F82C22D0F8AC2172
:100E6000C1F84022D0F8B021C1F84422D0F8B8210E
:100E7000C1F84C22D0F8C421C1F86022D0F8C821B2
:100E8000C1F86422D0F8CC21C1F86822D0F8D02172
:100E9000C1F86C22D0F87C21C1F80822D0F8842156
:100EA000C1F81022D0F88821C1F81422D0F89C2172
:100EB000C1F83022D0F8A021C1F83422D0F8A42102
:100EC000C1F83822D0F8A821C1F83C22D0F8B421CA
:100ED000C1F84822D0F8BC21C1F85022D0F8C02176
:100EE000C1F85422D0F8D421C1F87022D0F8D8210A
:100EF000C1F87422D0F8DC21C1F87822D0F8E021C2
:100F0000C1F87C22D0F8E421C1F88022D0F8E82191
:100F1000C1F88422D0F8EC21C1F88822D0F8F02161
:100F2000C1F88C22D0F8F421C1F89022D0F8F82131
:100F3000C1F89422D0F81822C1F8B422D0F8FC21CC
:100F4000C1F89822D0F80022C1F89C22D0F80422DF
:100F5000C1F8A022D0F80822C1F8A422D0F80C22AF
:100F6000C1F8A822D0F81022C1F8AC22D0F814227F
:100F7000C1F8B022D0F81C22C1F8C022D0F820223B
:100F8000C1F8C422D0F82822C1F8CC22D0F83422EB
:100F9000C1F8E022D0F83822C1F8E422D0F83C228F
:100FA000C1F8E822D0F84022C1F8EC22D0F854224F
:100FB000C1F80023D0F85822C1F80423D0F86022E9
:100FC000C1F80C23D0F86C22C1F82023D0F870228D
:100FD000C1F82423D0F87422C1F82823D0F878224D
:100FE000C1F82C23D0F82422C1F8C822D0F82C2232
:100FF000C1F8D022D0F83022C1F8D422D0F844224F
:10100000C1F8F022D0F84822C1F8F422D0F84C22DE
:10101000C1F8F822D0F85022C1F8FC22D0F85C22A6
:10102000C1F80823D0F86422C1F81023D0F8682250
:10103000C1F81423D0F87C22C1F83023D0F88022E4
:10104000C1F83423D0F88422C1F83823D0F888229C
:10105000C1F83C23FE4A126832F0FF0C05D1D1F8EA
:1010600090C062F3030CC1F890C0FA4A5370D0F8F4
:10107000943213F0010F1CBF01235370D1F8503389
:1010800023F00103C1F85033D0F8A43213F0010F5C
:1010900003D0537843F002035370D1F8603323F048
:1010A0000103C1F86033D0F8B43213F0010F03D05C
:1010B000537843F004035370D1F8703323F00103E5
:1010C000C1F87033D0F8AC0210F0010F03D05078A3
:1010D00040F008005070D1F8680320F00100C1F81A
:1010E0006803D1F82401C0F30802DB480260D1F89C
:1010F000E421C2F308024260D1F8A412C1F308014E
:1011000081607047D34800787047D2488078704734
:10111000D049C8707047CF48C0787047CF49D1F8E0
:10112000542360F30902C1F854237047CB48D0F828
:101130005403C0F309007047C64948607047C74868
:10114000C06870472DE9F047DFF80893054615F4AD
:10115000003F99F8010099F8031000EA010418BF54
:1011600024F0010415F4802F18BF24F0020415F4B4
:10117000002F18BF24F0040415F4801F18BF24F0BA
:101180000804DFF8D882D8F8400320F48030C8F88B
:10119000400314F00F0F65D0D9F80460D8F8480365
:1011A000002740F00100C8F84803D8F8480320F0B1
:1011B0000100C8F84803D8F8400340F48030C8F86C
:1011C00040034FF0630A0DE002F065FF5046D8F887
:1011D000481311F0010F01D0012703E0011EA0F117
:1011E0000100F4DC301EA6F1010601DD002FEBD07A
:1011F000BFB3D8F8500314F0010F0CBF20F001006A
:1012000040F00100C8F85003D8F8600314F0020F52
:1012100014BF40F0010020F00100C8F86003D8F8C6
:10122000700314F0040F14BF40F0010020F001001F
:10123000C8F87003D8F8680314F0080F14BF40F022
:10124000010020F00100C8F8680389F8024001207D
:1012500089F80000D8F8400340F48030C8F8400313
:101260003AE0FFE7D8F8500320F00100C8F8500337
:10127000D8F8600320F00100C8F86003D8F87003C4
:1012800020F00100C8F87003D8F8680320F00100CE
:10129000C8F86803002089F80200ACB1022089F880
:1012A0000000D8F8400340F48030C8F84003D8F874
:1012B000480340F00100C8F84803D8F8480320F07C
:1012C0000100C8F8480307E0D8F8401321F4803142
:1012D000C8F8401389F80000D8F8400115F0020F53
:1012E00020F00D0018BF40F0010015F0080F18BFE6
:1012F00040F0040015F0040F18BF40F00800C8F8D3
:10130000400115F0010F21D001F008FA044601F068
:1013100008FA0146D8F80C0000280EBF20460846FF
:1013200021460028D8F8000214BF40F0010020F048
:101330000100C8F80002D8F84002002914BF40F0AC
:10134000010020F00100C8F840020BE0D8F80002CC
:1013500020F00100C8F80002D8F8400220F0010097
:10136000C8F8400215F0200F18BF002416D0204600
:1013700001F0DEF900284FEA841000F1804000F50A
:10138000A040D0F8C01214BF41F0010121F00101CA
:10139000C0F8C012641C022CE9D30BE0D8F8C002DC
:1013A00020F00100C8F8C002D8F8000320F00100C6
:1013B000C8F80003BDE8F047FFF773BB2DE9F00361
:1013C00000F00F01002201EB41018C01C0F3031179
:1013D00004EB811101F1804101F5A041D1F84011E8
:1013E00011F0010F0ED140F01001C1F3031104EB15
:1013F000811101F1804101F5A041D1F8401111F0B6
:10140000010F4DD0144951F820801449C96901F0E9
:10141000080700EB40018E01114989591FFA81F933
:10142000002140EA0113C3F3031304EB831303F118
:10143000804303F5A043D3F8403113F0010F24D0CB
:1014400006EB811303F1804303F5A0430AE000009B
:10145000E0FE0300188400103089001000500040A6
:1014600000510040D3F844C1CCF3080517F1000C3B
:101470001CBFD3F844C1CCF3023CD3F8403105FA89
:101480000CFCC3F3054362441A44491C0229C8D327
:1014900008EBC80102FB09F001EB081100EB410267
:1014A000BDE8F0031046704710B50120FFF786FF36
:1014B00004460220FFF782FF044400F07BFC204436
:1014C0004FF47A7148434CF25031B0FBF1F010BD4B
:1014D0002DE9F041FA4E0546306810F01F0408BFB0
:1014E00001240120FFF76AFF07460220FFF766FF8D
:1014F000074400F05FFC3918F24F002D18BF002997
:1015000059D0D6F85003002210F0010FEE48A0FB8E
:1015100005C04FEA501033D07823B3EB151F08D91C
:10152000D6F85C0320F00F0040F00100C6F85C0321
:1015300034E0D6F85433DFF894C3C3F309036343AC
:101540006FF018056B430CEB43034FEA101CB3FB21
:10155000F1F0102828BF0F20844598BF604600286E
:1015600008BF012005D0012884BF00FB1132B2FB67
:10157000F0F2D6F85C3360F30303C6F85C330DE099
:10158000D6F85C33C0F3031023F00F031843C6F8FA
:101590005C03B7FBF5F0884288BF421A32206043F3
:1015A000B2FBF0F0B0F5005F28BF41F6FF70726843
:1015B00060F30C0272607068C0F30C00604300EBD3
:1015C000C00202EB001001EB4000B7FBF0F0BDE8F9
:1015D000F081BB48D0F8501311F0010F07D0D0F8BC
:1015E0005C0300F00F00C0EB00108001704770B585
:1015F0000168406801F01F05C0F30C060120FFF7E9
:10160000DDFE04460220FFF7D9FE044400F0D2FBC1
:1016100006FB05F1322201FB02410844A949B1FB56
:10162000F0F070BDA648D0F85C0300F00F007047E2
:10163000A3494A684B68C2F30C0260F30C034B6089
:10164000104670479E484068C0F30C00704700EB9E
:101650004000800100F1804000F5A040D0F800017A
:101660009B4980B2B1FBF0F0401C4008704730B499
:10167000974B31B1B3FBF1F1491C4A08B2F5804FE9
:1016800001D343F6FF72B3FBF2F1491C4D088C49BC
:101690004FEA520C51F8803F096803F00704C1F388
:1016A000031300EB4001890101F1804101F5A041E4
:1016B00018B3D1F80401DB1C634380B2A2EB4303EF
:1016C000D1F8004123F0010362F30F04C1F8004197
:1016D000D1F800216CF31F42C1F80021D1F8042198
:1016E00060F30F02C1F80421D1F8180163F30F0071
:1016F000C1F81801284630BC7047DB1CACF106006D
:101700006343A0EB4303DBE700EB4000800100F103
:10171000804000F5A040D0F80001000C704700EBBD
:101720004002920102F1804202F5A042D2F800315B
:1017300061F31F43C2F80031002818BF7047604AA8
:1017400052F8800F00F0070C52F81C0BC0F3031383
:10175000881FD91C01FB0CF1A0EB4101936E21F015
:10176000010160F30F039366D06F61F30F00D06740
:10177000704700F00F0101EB41018901C0F3031034
:1017800001EB801000F1804000F5A040D0F844014A
:10179000C0F30800704700F00F0202EB4202920112
:1017A000C0F303104B4B02EB801000F1804000F5BA
:1017B000A0409B58D0F84421CB1A61F30802C0F82E
:1017C0004421D0F844119B1E63F31841C0F8441122
:1017D00070473B49C969404A11F0100F00F00F01F2
:1017E00001EB41014FEA8111C0F3031001EB8010BE
:1017F00000F1804000F5A0405258D0F84401D2B228
:10180000C0F3080008BF0022801A0004000C08BFC3
:101810000120704700F00F0303EB43039B01C0F36B
:10182000031003EB801000EB810000F1804000F515
:10183000A040C0F85021704700F00F0202EB4202B6
:101840009201C0F3031002EB801000EB810000F165
:10185000804000F5A040D0F850017047184A0021A0
:10186000D26912F0080F10D000F00F0101EB410116
:101870008901C0F3031001EB801000F1804000F5F6
:10188000A040D0F84401C0F30231084670470C4A2A
:10189000D36943F00803D36100F00F0202EB420268
:1018A0009201C0F3031002EB801000F1804000F5BC
:1018B000A040D0F8442161F30E32C0F844217047B3
:1018C000005000400008AF2F89888888D8810C001C
:1018D000A08601001C51004028510040FD4A002113
:1018E000D26912F0080F10D000F00F0101EB410196
:1018F0008901C0F3031001EB801000F1804000F576
:10190000A040D0F84801C0F302410846704700F0FB
:101910000F0202EB42029201C0F3031002EB8010AF
:1019200000F1804000F5A040D0F8482161F3124258
:10193000C0F848217047042988BF704710B40023BD
:10194000E44CE26912F0080F00F00F0202EB4202D1
:101950004FEA8212C0F3031002EB801000EB040286
:101960001CBFD2F84401C0F302330020D4F81CC0DD
:101970001CF0080F1CBFD2F84801C0F30240C91A7E
:101980000844042803DD081A011D042003E0002890
:10199000BCBF014400201944E36943F00803E3613C
:1019A000D2F8443161F30E33C2F84431D2F8481111
:1019B00060F31241C2F8481110BC7047C5490028B5
:1019C000886914BF40F0080020F008008861704763
:1019D000C0488069C0F3C0007047BE4900288869CC
:1019E00014BF40F0020020F0020088617047B9483F
:1019F0008069C0F34000704700F00F0202EB420222
:101A00009201C0F3031002EB801000F1804000F55A
:101A1000A040C0F84C11704700F00F0101EB4101EC
:101A20008901C0F3031001EB801000F1804000F544
:101A3000A040D0F84C017047A64AD2F85C130229A6
:101A400003D110F0010F18BF7047D2F8400110F019
:101A5000010F0BD0D2F84C01D2F844110028C1F389
:101A600002311EBF0029C043C2F84C01012101EB25
:101A7000410100204FEA811C0CEB801101F18041F3
:101A800001F5A041D1F8402112F0010F0BD0D1F89F
:101A90004C21D1F84431002AC3F302331EBF002B7E
:101AA000D243C1F84C21401C0228E5D37047894A33
:101AB0000021D26912F0080F10D000F00F0101EBE5
:101AC00041018901C0F3031001EB801000F1804057
:101AD00000F5A040D0F84801C0F300510846704717
:101AE00001207047F0B4022ADDE9044C069E26BFAF
:101AF000921E52080022022B26BF9B1E5B08002369
:101B0000754DA5FB04542709BCF1020F0CBF01243D
:101B1000002400F00F0505EB4505AD01C0F30310EF
:101B200005EB801000F1804505F5A045D5F864016E
:101B3000002E61F31B6062F3144063F30C2067F323
:101B400007006CF38F3014BF40F4005020F40050B5
:101B5000002C14BF40F4001020F40010C5F86401FC
:101B6000F0BC70472DE9F00700F00F0606EB4606C3
:101B7000B601C0F3031006EB801000F1804000F5C1
:101B8000A040DDE90754DDF824C0D0F86401002945
:101B9000C0F3036AC0F30449C0F38137C0F3403691
:101BA000C0F30428C0B218BFC1F800A01AB14FEAB0
:101BB0004901891C11601BB14FEA4801891C196059
:101BC0001DB100EB800080002860002C18BF27604A
:101BD000BCF1000F18BFCCF80060BDE8F0077047FB
:101BE0003C490028C86914BF40F0200020F02000C4
:101BF000C86170473748C069C0F34010704770B47F
:101C000091B000224FF480456C10EC4601E0082AA8
:101C100005D2531C03EB8303B5FBF3F304E0D31F9E
:101C200003EB8303B4FBF3F35B1A48BF5B424CF84E
:101C30002230521C102AEAD30026009B01215CF8B6
:101C400021209A42BCBF13460E46491C1029F6D3E8
:101C500000F00F0101EB41018901C0F3031001EB1A
:101C6000801000F1804101F5A041D1F86801D1F860
:101C7000682100F00F0066F30302C1F8682108280C
:101C800007D2401C00EB8000B5FBF0F011B070BC37
:101C90007047C01F00EB8000B4FBF0F011B070BCC7
:101CA000704700F00F0101EB41018901C0F30310FF
:101CB00001EB801000F1804000F5A040D0F86801F1
:101CC00000F00F00082834BF401CC01F00EB80004C
:101CD00004E0000000500040CDCCCCCC34BF4FF429
:101CE00080414FF40051B1FBF0F0704710F00F0F3E
:101CF00008BF704700F00F0000EB4000800100F1CA
:101D0000804000F5A0400029D0F82C110CBF21F430
:101D1000803141F48031C0F82C117047002110F05F
:101D20000F0F0ED000F00F0000EB4000800100F11B
:101D3000804000F5A040D0F82C0110F4803F18BF7F
:101D400001210846704700F00F0000EB40008001C1
:101D500000F1804202F5A042D2F83401C2F83411F9
:101D600070472F4B58679967DA6770472C490028EE
:101D7000D1F8AC0014BF40F0020020F00200C1F81E
:101D8000AC00704726490028D1F8AC0014BF40F0E1
:101D9000010020F00100C1F8AC0070472048D0F8E5
:101DA000E00070471E49C1F8E40070471C48D0F8B5
:101DB0009800704770B41A4E0020D6F8401111F008
:101DC000010F04BF70BC704711F0040FD6F800C1BA
:101DD00001F00805134A12681FFA8CF4D6F844C1C2
:101DE000CCF3080C18BFC1F30740F369C1F3052118
:101DF00013F008031CBFD6F84431C3F30233002D9F
:101E000018BF491C0CFA03F301FB0300604302EB0B
:101E1000C20170BC01EB021100EB410070470000F1
:101E20000050004030890010FEF776BD10B5FEF777
:101E300073FD012818BF10BD0020FEF744FD2121CD
:101E40000020FEF76FFD2121BDE810400120FEF7C4
:101E500069BD10B5FEF730FDFEF75EFD01280AD121
:101E60000020FEF730FD21210020FEF75BFD21213F
:101E70000120FEF757FD0121052001F032FC012170
:101E8000052001F02EFCFA490020C87110BD10B5E4
:101E90004FF4066001F07BFCBDE810404FF4066093
:101EA00001F066BCF24A01465079002818BF0120B3
:101EB000002918BF01215171002191717047EC4A2E
:101EC000516A506208467047E949002008718870DD
:101ED00048707047E6490020087188704870704764
:101EE00070B50007C00E0D46801E00EB400101EBEF
:101EF0000014E0484FF4987200EBC40029461AF031
:101F0000D5FBDD4805F5987100EBC400BDE87040D5
:101F10004FF498721AF0CABB2DE9F0410546FEF75E
:101F200021FDD64FDFF858830446EDB14C2004FB69
:101F300000F21646294638461AF0B8FB324605F537
:101F4000006140461AF0B2FB04EB440000EB0414BD
:101F500007EB84004C211AF0AEFB08EB8400BDE8CF
:101F6000F0414C211AF0A7BB4C21401C41430C46C8
:101F700038461AF0A0FB21464046BDE8F0411AF071
:101F80009ABB10B5BA4CE061FFF7DCF8FFF7BAF87E
:101F9000A1696FF30F01A161A269C1B242EA0121F7
:101FA000A161022818BF10BDA06940F00100A06126
:101FB00010BDB4488168B44A114381600168521C65
:101FC0001143016000F067BE2DE9F041AD4A0546BE
:101FD0000C469068AC4B184390601068591C08433D
:101FE000106000F058FE0026002C7DD00020FEF787
:101FF0006AFC206820B1FEF7CCFD0020FEF763FCF0
:102000002846FFF7BEFF0020FEF7D8FC002835D099
:102010006068FFF781FF9D48E36853B1A1694FF401
:10202000407C4A420CEB820203EB81011AF03EFB3A
:102030001DE0974D4FF440711AF03DFB0020012345
:102040002956002910DB0A09120202EB800202F174
:10205000405202F540420907C90ED2F800C003FA07
:1020600001F14CEA01011160401C2628E8D389489F
:10207000616959B14FF400721AF018FB0120FEF7A4
:102080009DFCDFF8F0817C4F48B904E04FF400710B
:102090001AF011FBF2E71120FEF790FC70B1A56871
:1020A00065B140464FF4987229461AF0FFFA384657
:1020B0004FF4987205F598711AF0F8FA0220FEF7BD
:1020C0007DFC18B91220FEF779FC68B124695CB177
:1020D00071484FF4987221461AF0E8FA6F484FF4AD
:1020E000987204F5987100E001E01AF0DFFA604898
:1020F0000671867046704662417900214171867191
:102100004FF4066001F043FBBDE8F0414FF4066078
:1021100001F02EBB10B50020FEF7D5FB00F0A8FDA6
:102120005348C078002808BF10BD5648016821F008
:10213000030141F00D7141F080510160816821F08F
:10214000020141F00D7141F08051816010BD4FF4EA
:10215000066001F012BB10B54FF4066001F00DFBF4
:10216000FEF7DAFB01280AD10020FEF7ACFB2121A3
:102170000020FEF7D7FB21210120FEF7D3FB4848C2
:10218000D0F8401321F48031C0F840130020FEF74E
:102190009AFB00F06DFD3648C078002808BF10BDDE
:1021A0003848016821F0030141F00D7141F0805180
:1021B0000160816821F0020141F00D7141F0805110
:1021C000816010BD10B501F0DDFA10F0600018BF9D
:1021D000012010BD2648C0697047254880697047B6
:1021E00072B623498A6922EA0000886162B67047A4
:1021F0001F480078002818BF0120704770B5FEF70F
:102200008BFB002818BF70BD0024194D2C71AC70D9
:102210006C7021212046FEF785FB21210120FEF76D
:1022200081FB2C70BDE870400120FEF74CBB70B5FF
:102230000446FEF771FB002818BF70BD00210C4D4D
:102240002971A970697021210020FEF76BFB212103
:102250000120FEF767FB022C3CBF0120FEF772FB5A
:10226000012028702C62BDE87040FEF72CBB0000F6
:1022700020840010189D003018BD00300080003010
:1022800000A00030008000400200341200C0003086
:102290003C89001000D00030489E003048BE00301D
:1022A0000050004010B5FEF737FB002818BF10BDE6
:1022B0000020F94C2071A07060702121FEF732FBE4
:1022C00021210120FEF72EFB0120FEF73BFB012020
:1022D00020702062BDE81040FEF7F5BA0020FEF73E
:1022E000F2BAED490020887048700120FEF7EBBA81
:1022F000E94988627047E848806A7047E649C862E1
:102300007047E548C06A7047E34A0028D16A14BFA5
:1023100041F0010021F00100D0627047DE4890F8E2
:102320002C0000F00100704770B5DB4C0546A06A38
:10233000401CA062E16A11F0800F14BF01F010018F
:1023400001F00101002918BFFFF776FB207850B19A
:10235000206A10B1206A401E2062206A002804BF53
:102360000020FEF7B0FA20212846FEF7DBFA616A6A
:1023700000291CBF28468847FEF7C4FE022815D155
:10238000C648D0F8481311F0010F0FD0D0F8481309
:1023900041F00101C0F84813D0F8481321F00101C1
:1023A000C0F84813A06940F00200A061BC48016871
:1023B00041F02001016070BD0020B5E70120B3E7C6
:1023C00010B5FFF7EBFC0446FFF7ECFCB548044200
:1023D00008BF10BDB048816941F0040181610E2140
:1023E00001EAD43104F001020A43816962F31F411A
:1023F0008161AB48016841F02001016010BD0028F7
:1024000018BF0120A449C8707047A7487047A74863
:102410007047A148006B70479F48017A827A9142C9
:1024200014BF406B806B70479B48806B70472DE9F1
:10243000F04F9D4F4FF0000C8DB007F14C04E64675
:102440004FF0FF3807F80C8004F80CE00CF1010C99
:10245000BCF1260FF6DB4FF0000C002807DD12F868
:102460000C5007F80C500CF1010C6045F7DC002211
:102470000126CDF804E06D46CDF800E0002816DD19
:1024800017F902C0BCF1000F0EDBBCF1260F0BD216
:102490004FEA5C190CF01F0C55F829A006FA0CFC49
:1024A0004AEA0C0C45F829C0521C8242E8DB0022A3
:1024B00094460DF108094FEA521A02F01F0B55F825
:1024C0002AA006FA0BFB1AEA0B0F1ABF09F802C082
:1024D0000CF1010C09F80280521C262AEBDB0022C9
:1024E000002810DD17F902C0BCF1000F08DBBCF1B9
:1024F000260F3ABF19F80CC004F802C004F8028095
:10250000521C8242EEDBDFF890A100220028CAF8BC
:1025100030E009DD14F902C0944502D0CAF8304019
:1025200002E0521C8242F5DBDFF884B10020ABF1FF
:10253000720404F14C0704F8008007F800E00BF87F
:1025400000E0401C2628F6DB0020002904DD1A5C90
:102550002254401C8142FADC0020CDF804E0CDF882
:1025600000E0002912DD2256002A0CDB262A0AD2BE
:10257000530902F01F0255F823C006FA02F24CEA92
:10258000020245F82320401C8842ECDB0020024672
:10259000430900F01F0C55F8233006FA0CFC13EA2F
:1025A0000C0F1ABF09F80020521C09F80080401CCB
:1025B0002628EDDB002000290BDD2256002A05DB52
:1025C000262A3CBF19F802200BF80020401C884244
:1025D000F3DB0020CAF838E0002909DD1BF90020F0
:1025E000824202D0CAF838B002E0401C8842F5DBD3
:1025F00011F0010F18BF252015D0420900F01F036C
:1026000055F8222006FA03F31A420AD1420900F0D3
:102610001F0055F8223006FA00F0184345F8220052
:1026200001E0401EE9D500200246430900F01F0CDE
:1026300055F8233006FA0CFC13EA0C0F1ABF09F800
:102640000020521C09F80080401C2628EDDB0020E9
:1026500000290ADD2256002A04DB262A3CBF19F88D
:1026600002203A54401C8842F4DB0020CAF834E0CF
:102670000029DCBF0DB0BDE8F08F3A56824204D08D
:10268000CAF834700DB0BDE8F08F401C8842F4DB0E
:102690000DB0BDE8F08F0000208400100050004015
:1026A00060840010010007003C890010628900105E
:1026B000D489001040F2DB114843FE4901EB800051
:1026C0007047FD49C0EB001001EBC0007047DFF818
:1026D000ECC3012B8CF808008CF8091003D9401CBE
:1026E00020F0010011468CF80A008CF80B1000FB5A
:1026F00001F24FF6FF7101EA4202ACF8122001EA42
:102700004000ACF814007047EC48C07A7047EB48C2
:10271000807A7047E94A107351737047E748407BED
:102720007047E648007B7047E54A1070517070476B
:10273000E349085C70472DE9F047DFF880930446D1
:1027400099F80500002804BF99F8010019F0B8FFB6
:1027500099F80400002808BFBDE8F0874FF0000892
:10276000D9F81C0047464646454610F0020F1CBFEC
:10277000DFF8408310F0040F05D0B9F81210CD4AED
:1027800021F001018F1810F0010F18BFCA4E10F090
:10279000200F18BFCB4DD9F828002060FEF7B5FCFC
:1027A00010F0010F06D0FEF73DFF022828BF99F870
:1027B000020000D20020E760C4E90108C4E9046512
:1027C0000120BDE8F087BD4800210171817170478B
:1027D00070B50546FEF7C6F84C2100FB01F2144621
:1027E000B949284619F062FF224605F50060BDE8A8
:1027F0007040B64919F05ABFF0B583B0FEF7B2F891
:10280000044600210846FFF717F800900121002038
:10281000FFF712F800220190002C2AD96E464FF0E3
:10282000010C4FF6F07502EB4200002100EB0210A4
:102830004B0901F01F0756F823300CFA07F73B420B
:1028400011D0CB079B0C03EB80034F0803EB8703EE
:1028500003F1405303F500431B889BB2AB4202D9FE
:1028600003B00020F0BD491C2629E1D3521CA2422E
:10287000D9D303B00120F0BD70B50D460107C80ED5
:10288000811E01EB410000EB011491484FF4987256
:1028900000EBC401284619F009FF8E484FF49872E6
:1028A00000EBC40105F59870BDE8704019F0FEBE5C
:1028B0002DE9F04F00F00F07780083B0A0F1020B74
:1028C0000025E9464FF001084FF6F07647EA051A71
:1028D0005046FEF773F8002843D05046FEF7BEFF7F
:1028E00008FA00F4022C88BF022400215046FEF7AB
:1028F000A3FF009001215046FEF79EFF00210190AA
:10290000002C2ED90BEB0500982200FB02FA01EBFC
:102910004102002002EB011C420900F01F0359F89C
:10292000222008FA03F31A4215D000F001020AEB44
:10293000423202EB8C02430802EB830202F1405266
:1029400002F51042B2F8182D92B2B24203D903B088
:102950000020BDE8F08F401C2628DDD3491CA14291
:10296000D5D36D1C022DB1D303B00120BDE8F08F8B
:102970002DE9F0410026514D00280C4640D000F0D2
:102980000F01C0F3031001290EBF00210229BDE889
:10299000F081022828BFBDE8F0810F18FDF7BCFFC9
:1029A0005FEA00081CBF0020FDF78DFF0023982080
:1029B00007FB00FC03EB4300002200EB031702F0CF
:1029C00001000CEB4030510800EB870000EB810068
:1029D00000F1405000F51040521CC0F8184D262A56
:1029E000EDD35B1C022BE5D3B8F1000F08BFBDE8A7
:1029F000F081AE706E70BDE8F0410120FDF763BF5D
:102A0000FDF78AFF5FEA00081CBF0020FDF75BFFAF
:102A1000002303EB4300002200EB031CD007800CD3
:102A2000510800EB8C0000EB810707F1405707F5D8
:102A30000047521C3C60262AF0D35B1C312BE8D3A4
:102A4000B8F1000FD5D1BDE8F08110B5FEF7C1FE99
:102A50001A49088210BD194AC1B200F47F43128A94
:102A6000914288BF11464FF0640C01FB0CF1B1FBA1
:102A7000F2F11A0A02FB0C1110F4803F12BF08B2E7
:102A8000484200B2704710B54FF44071124C1348E1
:102A900019F011FE002001232156002927DB0A0925
:102AA000120202EB800202F14052090702F5404295
:102AB000C90E15E0B01701101C1F01102084001072
:102AC0002E8400100C2001100080003000A0003087
:102AD000189D003018BD00303C89001000C0003047
:102AE000D2F800C003FA01F14CEA01011160401C68
:102AF0002628D1D310BD10B5224C4FF44071224886
:102B000019F0D9FD002001232156002910DB0A0904
:102B1000120202EB800202F1405202F54042090724
:102B2000C90ED2F800C003FA01F14CEA01011160AC
:102B3000401C2628E8D341F67871144819F0BBFDF3
:102B4000BDE8104041F67871114819F0B4BD114844
:102B500010B5808B00F48170FFF713FA4FF44071C9
:102B6000094819F0A8FD41F61851084819F0A3FDCD
:102B700041F61851064819F09EFDBDE810400020AE
:102B8000FEF756BD3C89001000C0003000800030C8
:102B900000A00030208400102DE9F04100276D4D89
:102BA0000126002808BF2E701FD001282F7018BFE3
:102BB0006F701AD0DFF8A081D8F800006749084389
:102BC000C8F800002978664C002914BF49F608307F
:102BD0006448E06014BF64484FF0BB70A060634875
:102BE000006830F0FF0206D101E06E70E2E7E268B3
:102BF00060F30302E26051B1A06840F01800A060E9
:102C0000012000F085F8A06840F48050A060012009
:102C100000F07EF8687818B1E06840F03000E060BD
:102C2000D4F8B00040F00100C4F8B000012000F07A
:102C30006FF8E6674FF4E0602061C4F88870287888
:102C4000002818BFC4F89460E06820F03000E0600D
:102C5000A06820F48050A060D8F8000020F00400A4
:102C600040F00D7040F08050C8F80000BDE8F081E1
:102C70003B48C16821F03001C160816821F4805176
:102C800081603548016821F0040141F00D7141F087
:102C9000805101607047304802683049114301603B
:102CA0002C492F480A783AB1826842F018028260B3
:102CB000826842F480528260497819B1C16841F05B
:102CC0003001C160D0F8B01041F00101C0F8B0107F
:102CD0007047B0F5007F28BF40F2FF10244941EA59
:102CE00000201F49086470471D494FF020400864C8
:102CF00070471B4A116C4FF020401064506C11F06B
:102D0000FF0FC0F308201CBF41F020411164704741
:102D100082B040F24C42009013E000BF00BF00BF01
:102D200000BF00BF00BF00BF00BF00BF00BF00BFAB
:102D300000BF00BF00BF00BF00BF0198411E01914E
:102D4000EBD20098411E009128BF0192F5D202B04B
:102D5000704700005C8400100080004004003412C2
:102D60000060004005F4010020009B00D0FE03003D
:102D7000130000A0424841498161891CC1614A1E7B
:102D80004263036823F0030343F00D7343F0805361
:102D90000360436923F0010343F00D7343F0805354
:102DA000436103691A430261364A8260364AC2604F
:102DB000C2681143C160354900200860704710B5F2
:102DC00001F061F931480468002C08BF30BFFAD027
:102DD0000021016001F05BF9204610BD10B501F043
:102DE00052F92648294B2649421C1C682CB1002068
:102DF000186001F04CF9204610BD72B648638A6134
:102E000020BF88614A6362B6BFF36F8FBFF34F8FF5
:102E1000EBE71B48016821F0030141F00D7141F01F
:102E2000805101601A49816001691A4A11430161A8
:102E300030BF704772B6114911484163C91CC16166
:102E4000891E816162B670470D480168124A1143BC
:102E5000016070470A48016821F0030141F00D71DB
:102E600041F080510160704772B6044904488161A5
:102E7000891CC161491E416362B67047000034126B
:102E8000008000403C00341228003412608400109E
:102E900008003412010034120300341270477047E6
:102EA0000022B2EBD10F26D20368B3F1FF3F04BF7B
:102EB0004368B3F1FF3F17D18368B3F1FF3F04BF0D
:102EC000C368B3F1FF3F0FD10369B3F1FF3F04BF04
:102ED0004369B3F1FF3F07D18369B3F1FF3F04BFFB
:102EE000C369B3F1FF3F01D0002070472030521C6E
:102EF000B2EBD10FD8D30120704710B40023B3EB4D
:102F0000D20F30D2D0F800C00C68A44522D1D0F83E
:102F100004C04C68A4451DD1D0F808C08C68A445F5
:102F200018D1D0F80CC0CC68A44513D1D0F810C08B
:102F30000C69A4450ED1D0F814C04C69A44509D140
:102F4000D0F818C08C69A44504D1D0F81CC0CC6955
:102F5000A44502D010BC00207047203020315B1CFB
:102F6000B3EBD20FCED310BC012070472DE9F04156
:102F7000054601F090F8002021264FF48257844640
:102F80004FF4E0221660C5F800C0116841F004015A
:102F90001160116811F0040FFBD1176080232C46DB
:102FA0000021D4F80080B8F1FF3F04BFD4F80480BA
:102FB000B8F1FF3F1DD1D4F80880B8F1FF3F04BF3E
:102FC000D4F80C80B8F1FF3F13D1D4F81080B8F1D9
:102FD000FF3F04BFD4F81480B8F1FF3F09D1D4F803
:102FE0001880B8F1FF3F04BFD4F81C80B8F1FF3F50
:102FF00008D0C2F800C0401CC0B20828C2D30220CA
:10300000BDE8F081491C2034B1EBD30FC9D3C2F81D
:1030100000C00120BDE8F0812DE9F041054601F036
:103020003AF80020092684464FF4E0231E60C5F8D4
:1030300000C0196841F004011960196811F0040F0B
:10304000FBD12C464FF4806200212768B7F1FF3F87
:1030500004BF6768B7F1FF3F17D1A768B7F1FF3F1B
:1030600004BFE768B7F1FF3F0FD12769B7F1FF3F12
:1030700004BF6769B7F1FF3F07D1A769B7F1FF3F09
:1030800004BFE769B7F1FF3F08D0C3F800C0401C98
:10309000C0B20328CAD30220BDE8F081491C203405
:1030A000B1EBD20FD1D3C3F800C00120BDE8F0814D
:1030B0002DE9F05F8846814604274FF07F0A4FF0E4
:1030C000020B4FF4E02600F0E6FF49464246534625
:1030D0004FF0060CC6F800B052F8040B41F8040B90
:1030E000C6F800C0306810F0040FFBD15B1EF1D2AF
:1030F000002030604C4645461F20D4E900C3D4E987
:103100000221D5F800E0E64504BFD5F804C09C458F
:1031100005D1AB68934204BFEA688A4208D07F1E9B
:1031200003D34846FFF722FFCDE70220BDE8F09F1A
:1031300010341035401EE0D20120BDE8F09F70B57C
:103140000D46044600F0A7FF4FF4007221462846C2
:1031500019F0ACFA012070BD2DE9F0410546C0051B
:10316000ADF5007D14460E46C00D25D0A8466FF380
:1031700008086F4600F08FFF4FF400724146384652
:1031800019F094FAC5F30800C0F50077A74288BF8C
:10319000274668443A46314619F097FA4046FFF709
:1031A000E5FE022844D069464046FFF781FF022829
:1031B00043D03D443E44E41BB4F5007F19D34FF4A3
:1031C00000723146684619F080FA2846FFF7CEFEB5
:1031D00002282DD069462846FFF76AFF02282CD026
:1031E000A4F5007405F5007506F50076B4F5007FCA
:1031F000E5D2C4B16F4600F04EFF4FF4007229468D
:10320000384619F053FA22463146684619F05DFAFD
:103210002846FFF7ABFE02280AD069462846FFF78A
:1032200047FF022809D00DF5007D0120BDE8F0819F
:103230000DF5007D0A20BDE8F0810DF5007D0B2025
:10324000BDE8F0812E490860086100F010B82C49F3
:103250000860486100F00BB8294948677047284961
:1032600088677047264801210166016570474FF065
:103270004022116B10F0010F18BF21F4404110F0F3
:10328000020F1CBF21F4405141F4805110F0040F93
:1032900018BF21F4406110F0080F18BF41F44071CD
:1032A00010F0100F18BF41F0C00110F0200F18BF30
:1032B00041F0300110F0400F18BF41F00C0110F048
:1032C000800F18BF41F0030141F4BE0141F02041DD
:1032D0001163D2F8901010F4807F1CBF21F003011D
:1032E00041F0020110F4007F1CBF21F00C0040F0FF
:1032F000080141F4BE0040F02040C2F89000704741
:1033000000100040704772B6D3488268D3490A4320
:103310008260C2681143C16062B64169D04A1143FC
:1033200041617047CC48416921F0010141F00D71C4
:1033300041F08051416172B6C16821F0400141F015
:103340000D7141F08051C160816821F0400141F070
:103350000D7141F08051816062B6704710B572B650
:10336000BD4CA168BD480143A160E1680843E0602D
:1033700062B66069BA4908436061BA4843F63F7172
:10338000C160002181638164C0F8B01003210A206C
:1033900000F0A7F90A2000F0C7F9606920F00100E9
:1033A00040F00D7040F08050606172B6E06820F02F
:1033B000400040F00D7040F08050E060A06820F0C8
:1033C000400040F00D7040F08050A06062B610BD2B
:1033D000A44A10605160484390607047A14A106051
:1033E0005160484310F0010F18BF401C90607047B7
:1033F0009C49C1F8B00070479A49002818BF0120C5
:103400008864704797498863C86840F00200C860C4
:103410007047DFF850C2CCF82000CCF82410CCF86C
:103420002820CCF82C300120CCF83000DCF8340017
:1034300010F0010F05D020BFDCF8340010F0010FB0
:10344000F9D110F0020018BF4FF0FF3070478548E7
:10345000C16821F00201C16070478248C16841F033
:103460000101C16070477F4B186259629A62012066
:103470001864586C10F0010F04D020BF586C10F085
:10348000010FFAD110F0060018BF4FF0FF3070475F
:103490007448C16821F00101C16070477148C1687A
:1034A00041F00401C1607047027C017B02F03F02E1
:1034B00041EA02416B4A916501685162416891623B
:1034C0008168D16201211165516D11F0010F04D0A5
:1034D00020BF516D11F0010FFAD1D36D8382D36DEE
:1034E0001B0CC382136E0383136E1B0C4383536E3A
:1034F0008383526EC2F30E42C28311F0020018BFE2
:103500004FF0FF3070475748C16821F00401C16097
:1035100070475448C16841F00801C1607047DFF846
:1035200044C1CCF87820CCF82000CCF82430CCF87A
:1035300028100120CCF87000DCF8740010F0010FA6
:1035400005D020BFDCF8740010F0010FF9D110F0A5
:10355000060018BF4FF0FF3070474248C16821F0A5
:103560000801C160704701684FEA31423D49C1F826
:103570009C204068C1F8A000C86840F02000C860E6
:10358000704701684FEA31423649C1F89C20808873
:10359000C1F8A000C86840F02000C8607047314BF7
:1035A00018625A6299620120C3F89400D3F8980017
:1035B00010F0010F05D020BFD3F8980010F0010FD4
:1035C000F9D110F0060018BF4FF0FF307047254AC0
:1035D000106251620120C2F89000D2F8980010F0F9
:1035E000010F05D020BFD2F8980010F0010FF9D1DB
:1035F00010F0060018BF4FF0FF3070471948C1683F
:1036000021F02001C16070471648C16841F01001E7
:10361000C1607047A3F1050C124BC3F888C0186253
:103620005A6299620120C3F88000D3F8840010F038
:10363000010F05D020BFD3F8840010F0010FF9D19D
:1036400010F0060018BF4FF0FF3070470548C16802
:1036500021F01001C160704700800040400034122A
:1036600001003412009000401B4810B5022140F8C0
:10367000501F012101611021416241F206014161A7
:10368000002181610421816390214163416B41F0FC
:10369000010141634FF4817101610161032000F078
:1036A00043F80021032000F01CF8002010BD10B5E5
:1036B000032000F045F808484FF4807101660021AE
:1036C00001661021816702214165002010BD034978
:1036D0000020087070470000003000406484001033
:1036E000704700F00303DA004FF0FF0C0CFA02F20F
:1036F0004FF0050C0CEBC30301FA03F300F00C01CF
:1037000001F1E021002807DAD1F8140D90431A40A6
:103710001043C1F8140D7047D1F8000490431A40CB
:103720001043C1F80004704700F01F01012202FAA3
:1037300001F14009800000F1E020C0F8001170475D
:1037400000F01F01012202FA01F14009800000F19E
:10375000E020C0F88011704700F01F01012202FA3A
:1037600001F14009800000F1E020C0F880127047AC
:103770004FF0E021C1F8000170474FF0E021C1F89F
:10378000800170474FF0E020D0F8000170474FF003
:10379000E021C1F880027047084800687047074A76
:1037A0001168106008467047044A126800F110035F
:1037B00052F8230042F823107047000008ED00E0A3
:1037C00002210C20FFF78DBF72B6BC488268BC494D
:1037D0000A438260C2681143C16062B6704772B624
:1037E000B648816821F4805141F00D7141F080515B
:1037F0008160C16821F4805141F00D7141F0805128
:10380000C16062B67047AF4881B0016F11F4007FAC
:10381000FBD1816E11F0010F1CBFD0F88410009114
:1038200004D0D0F88410009A9142FAD0016F11F4BC
:10383000007F04BF4CF27101016642F241318166A2
:1038400001B070479F4981B04FF40D528A660A6FEC
:10385000CA66012898BF012005D9401EB0F5803FF7
:1038600028BF4FF6FF7082B24FF05C5040EA022052
:1038700048664FF01140C1F88000086F10F4007FD7
:10388000FBD1886E10F0010F1CBFD1F884000090AE
:1038900004D0D1F88400009A9042FAD0086F10F456
:1038A000007F04BF4CF27100086642F24130886626
:1038B00001B07047834881B0016F11F4007FFBD1E4
:1038C000816E11F0010F1CBFD0F88410009104D05C
:1038D000D0F88410009A9142FAD04FF40D518166CD
:1038E00001B070477548806810F4805008BF704779
:1038F0007448806E00F0010070477248406EC0F35B
:103900000F2070476F48D0F88400704710B50C2026
:10391000FFF722FF0C20FFF707FF6A4902204867E4
:1039200010BD684910B5032088670C20FFF708FF19
:10393000BDE810400C20FFF70FBF634A116810600C
:10394000084670475F4810B5016FC1665E48006861
:10395000002818BF80475D48016841F4805101602C
:1039600010BD59484068704710B572B65348826818
:1039700053490A438260C2681143C16062B60320A2
:10398000504988670C20FFF7DBFE0C20FFF7E4FEB0
:1039900000F062F94E4B0420C3F888004FF6FF7028
:1039A000C3F88C0072B66033FFF74CFF4FF4007021
:1039B000186062B610BDF8B572B64248016F11F4D6
:1039C000007FFBD1816E11F0010F1CBFD0F8841075
:1039D000009104D0D0F88410009A9142FAD04FF4AC
:1039E0000D5181663A494FF400320A6662B6D1F849
:1039F0000412324D002946D0334C4FF6FF73591A4A
:103A0000A160AA69D5F81CC002F00F020CF00F0CDF
:103A10006244121D01FA02F2A2F54341DFF8B4C07C
:103A2000513961452FD2D0F88400191AE160B1F5FF
:103A3000803F28D2284B4FF0000CA1FB03070CFB62
:103A4000037301FB0C31634618F044FE401C400830
:103A50002061B0F57A7F38BF4FF47A701F4B9968B8
:103A6000002908BF98605A681A609968C3E9011074
:103A70008A421DD9824205D9814201D9616002E0A2
:103A8000606000E0626000F0F5F872B6A86820F4AB
:103A9000805040F00D7040F08050A860E86820F43D
:103AA000805040F00D7040F08050E86062B6F8BD84
:103AB0008242E7D88142E3D8E0E70000008000407E
:103AC0000010341200C000406884001060840010B0
:103AD00000A000404F62250000E1F505FC890010C0
:103AE0000F4881680F4A114381600F48016841F413
:103AF00004710160001F016821F004010160016888
:103B000041F0100101607047084908607047BFF339
:103B10004F8F084906480860BFF34F8FFEE700004B
:103B2000008000400400341214ED00E008ED00E0D5
:103B30000400FA050CED00E015488168154A1143B0
:103B400081601003416941F001014161016A21F086
:103B50000F0211490A430262104B8A1EC3F8C420A7
:103B6000016570474FF04020006900F07000704719
:103B70004FF040200A4940F8301F0A4941600A4985
:103B800001660A49416670474FF04020406870471F
:103B9000008000400400341203005FA00060004079
:103BA000C0845FA050895FA00A005FA000005FA0F2
:103BB000022824BF00207047E44B53F8202043F82C
:103BC00020101046704770B5E14C206FDF4D10F0AB
:103BD000010F05D00120E0662868002818BF804743
:103BE000206F10F0020F08BF70BD0220E066686809
:103BF000002808BF70BDBDE87040004710B572B620
:103C0000D4488268D4490A438260C2681143C160C3
:103C100062B60222CE490A6501230B660323CB66F6
:103C20004A6572B6816821F0800141F00D7141F062
:103C300080518160C16821F0800141F00D7141F037
:103C40008051C16062B60920FFF76EFD0221BDE818
:103C500010400920FFF745BD72B6BE488268BE49D4
:103C60000A438260C2681143C16062B60220B8494B
:103C700008657047B6490220486572B6B548816844
:103C800021F0800141F00D7141F080518160C168E7
:103C900021F0800141F00D7141F08051C16062B6A8
:103CA0007047AC488068C0F3C0107047A848016FE7
:103CB00011F4007F14BF4FF440714FF4807101661E
:103CC000704710B5A24CE06F10F0020F4FF00100EA
:103CD00018BF0320606700F077F99E498A69C969B7
:103CE00002F00F02D04001F00F01C8400521B0FBE7
:103CF000F1F04FF405710009C4F880109749A1FB59
:103D000000104009C4F88400206F10F4007F14BF35
:103D10004FF440704FF48070206610BD8C48016FE6
:103D200011F4807F14BF4FF440714FF400710166AD
:103D30007047874B30B4DA6F12F0010F14BF0322C3
:103D400002225A6700EB4005C5EBC010C1EBC00072
:103D50004FF4FA744C43C0EB001000EB4000804974
:103D600004EBC000A1FB00107A4900224FF0020CC6
:103D70008C69C008C96904F00F0401F00F012144E7
:103D8000C8400521B0FBF1F0B0F5803F05D3511CD0
:103D90004008CAB2B0F5803FF9D242EA0C2141F0A6
:103DA0001001C3F88810C3F88C00186F10F4807FDE
:103DB00014BF4FF440704FF40070186630BC704769
:103DC0006348016F11F4003F14BF4FF440314FF4CA
:103DD0008031016670475E48016F11F4803F14BF67
:103DE0004FF440314FF40031016670475848006F7E
:103DF000C0F3002070475648006FC0F34020704762
:103E000054498968C1F3C011002904BF00207047DC
:103E10004F4900280CBFD1F80002D1F804027047C6
:103E20004C4B9A68C2F3C012002A04BF00207047AE
:103E3000474A00280CBFD2F88000D2F88800C0F3AF
:103E40000A200CBFD2F88020D2F8882002F00F029E
:103E5000D3F818C0DB690CF00F0C03F00F036344B8
:103E60001A449140012202EB400048433B49A1FB28
:103E70000010000970473B4901200870704770B47A
:103E8000344B322251439A69D3F81CC002F00F021E
:103E90000CF00F0C6244121DD14008BF012104D068
:103EA000B1F5803F28BF4FF6FF719A68C2F3C01288
:103EB000002A1CBF70BC704772B6D3F808C0264AEF
:103EC0004CEA020CC3F808C0D3F80CC04CEA02025A
:103ED000DA6062B61E4A4FF0020CC2F850C04FF4CE
:103EE000003414660425C2F88850C2F88C101E4DA8
:103EF000D566C2F874C01D4902283CBF134E46F86F
:103F000020100021174801704FF4007111660178EC
:103F100019B920BF01780029FBD014669567D566D2
:103F2000C2F854C072B6986820F0800040F00D705E
:103F300040F080509860D86820F0800040F00D700C
:103F400040F08050D86062B670BC7047808400102A
:103F500000A0004000800040800034121F85EB511B
:103F6000CDCCCCCC7C84001002000202275E000085
:103F70004FF0E021002088610861274948607047C0
:103F800010B54FF0E02460610020A0610221401EC6
:103F9000FFF7A7FB07202061BDE8104007F0F0BE47
:103FA00010B507F0F1FE4FF0E0210020086110BDD0
:103FB00010B507F0E9FE4FF0E02100200861164837
:103FC0000188491C018010BD1348806870472DE9A5
:103FD000F041114C002705462780A0684FF47A7104
:103FE000B0FBF1F04FF0E026401E7061B761022196
:103FF000C81EFFF776FB0720306107F0C1FE21885D
:10400000A942FCD307F0C0FE3761BDE8F081034947
:1040100048430149886070478884001040420F007F
:10402000704770B505464FF40D500406A066032096
:10403000E066264860664CF2710020662448C4F8A9
:10404000800042F24630A06602210020FFF749FBC3
:104050000020FFF769FB002D08BF70BDA06E42F283
:1040600041310843A06670BD012110B58807816702
:104070004FF40D5181660020FFF762FBBDE8104050
:104080000020FFF769BB01208107486770470120C6
:104090008107886770474CF2710081070866704796
:1040A0000C4A11681060084670470A4808B5006855
:1040B00018B18047002818BF08BD4CF2710188076D
:1040C0000166016FC166006F009008BD075E5F3733
:1040D00000AF2F9194840010FD490020C8717047F3
:1040E000FB48C079704770B5F94C00254FF4E46186
:1040F000257065702571F74818F0DDFA4FF4E4611A
:10410000F54818F0D8FAE56065714C21F34818F0CD
:10411000D2FA4C21F24818F0CEFAA5717421F14878
:1041200018F0C9FA7421F04818F0C5FA256170BD7D
:10413000E749002048707047E54840787047E448F8
:104140004079002818BF01207047E1488079002895
:1041500018BF01207047DE480079002818BF0120F1
:104160007047DB48407800EB4001C1EB4010DD496F
:1041700001EB800070472DE9F041D54C0546D94947
:104180006278DA4F02EB4200C0EB4210D84E01EBEE
:1041900080033A783078294610444200184618F0D7
:1041A00094FA6278D04902EB4200C0EB421001EB76
:1041B00080033A783078294610444200184618F0B7
:1041C00084FA0120A071E07940F00400E071BDE8BC
:1041D000F081BF4800697047BD484078C0EBC0011E
:1041E000C1EB8010BB4901EB401070472DE9F04155
:1041F000B74E07463078002814BFBE48BE48047842
:1042000014BFBE48BE48057804FB05F8FFF77BF8ED
:1042100029462046FFF7DCF87078AF4CC0EBC001B0
:10422000C1EB8010AB4904EB401201EB40103B4660
:104230000146FFF7EEF8FFF775F870784FEA48028D
:10424000C0EBC001C1EB801004EB4010394618F000
:104250003CFA01203071F07940F00100F07101204A
:10426000BDE8F0812DE9F047994D044699496A78F7
:10427000DFF88082C2EBC200C0EB821001EB40137A
:104280002878DFF874929D4E9D4F2146002815BF77
:1042900098F8000099F8000032783A7800FB02F0B4
:1042A0004FEA4002184618F010FA6A788A49C2EBC1
:1042B000C200C0EB821001EB401C28782146002888
:1042C00015BF98F8002099F8002033783B7802FB5E
:1042D00003F04FEA4002604618F0F7F90120287118
:1042E000E87940F00100E871BDE8F0877848C068DF
:1042F000704770B5834C05460146227877485200D6
:1043000018F0E3F9227829465200754818F0DDF9D3
:104310006F4801214171C17941F00201C17170BD45
:104320002DE9F04FADF25C7DDFF8A4910120CDF8CE
:10433000440799F80400CDF8400799F80500CDF836
:104340003C0799F80600CDF8380701F08DFD0446CA
:1043500001F0A2FD0546FDF767FDCDF85807FDF712
:1043600047FFCDF85407FDF76DF9CDF85007FCF77E
:10437000CCFE0746FCF7C6FE8046FDF757FD99F8D0
:1043800002000026002804BF0420C9F818000CD041
:10439000022C1CBF0A20C9F8180010D0062D04BF3B
:1043A0000420C9F8180089F80260FDF712F90830F6
:1043B00005094FF0010AB8F1020F26D109E013F008
:1043C000DCF810F4817F14BF3C201E20C9F81800CF
:1043D000E4E701F05FFEC0B9022C02D0052C0AD040
:1043E00013E04FF47A7068434FF47A7190FBF1F068
:1043F000C9F8180007E007F038FE002814BF0520B0
:104400001220C9F8180089F802A0D9F81800042869
:10441000BCBF0420C9F8180099F80200B9F81810B8
:10442000000240EA014040F00102002391210720F0
:104430000BF0EAF817F0010F2AD1022C28D0002047
:10444000FDF7F6F8FDF72EFF37464FF0000B06F0AC
:10445000C2FB012822D00DF5E460FEF76CF90028BC
:1044600000F031820DF5E46007F09AFA002089F837
:104470000100D9F81800C01E8642CABF8742012534
:104480000025DDF82C0710B3DDF83C0750B163E0E0
:10449000FDF7B4FE0020CDF84407D5E74FF0010B3F
:1044A00000F0FBB96846DDF82C1718F018F98046C3
:1044B00055B3144C414620784200084818F005F9DD
:1044C000207841464200064818F0FFF81DE043E01E
:1044D0009884001084200110088A0010689F001042
:1044E000B49F0010A427011000A00010EE8400105B
:1044F000EF840010EC840010E9840010ED840010BB
:10450000EA840010F084001008E089F805A099F80A
:10451000070040F0020089F807001DE0FEF7F3FEF7
:10452000FD4C01212078FEF753FFFC4A4346A2F1DF
:104530004C010846FEF76DFFFEF7F4FE2078414679
:104540004200F64818F0C1F889F805A099F807006C
:1045500040F0020089F80700DDF82807002800F085
:10456000E380DDF84007002840F0DE8099F8000085
:10457000DDF82847F0BBD9F80C80B8F1000F24D043
:10458000E7480078CDF84C07E6480078CDF84807B2
:10459000FEF7B9FEDDF84817DDF84C07FEF71EFF01
:1045A000214642460846FEF75EFFFEF7BBFEDE48A8
:1045B0000078022804BF404606F02DFFDA48007854
:1045C000092804BF204606F026FFD84800780128B5
:1045D00016D9DFF8548398F80000042804BF204659
:1045E00006F019FF2146684618F07EF8044698F850
:1045F000000000E004E0052804BF204606F00BFFA1
:10460000EDB399F8010099F80020C0EBC001C1EBAF
:104610008011C748002A00EB411021460CBFC54A53
:10462000BF4A137814BFBF4AC34A127803FB02F291
:104630004FEA420218F049F899F80100C0EBC001B6
:10464000C1EB8011BD4800EB411399F800002146F1
:10465000002814BFB248B748007814BFB14AB64A20
:10466000127800FB02F04FEA4002184618F02DF8CD
:1046700089F804A099F8070040F0010000E002E08A
:1046800089F8070041E0CDF8484799F80000002874
:1046900014BFA348A74890F8008014BFA148A648BB
:1046A000047808FB04F0CDF84C07FEF72CFE2146F9
:1046B0004046FEF78DFE99F80100A04CC0EBC0010A
:1046C000C1EB80109A4904EB401201EB4010014607
:1046D000DDF84837FEF79DFEFEF724FEDDF84C07B7
:1046E000420099F80100C0EBC001C1EB801004EB5F
:1046F0004010DDF8481717F0E8FF89F804A099F892
:10470000070040F0010089F8070087480078032877
:104710000AD199F80100C0EBC001C1EB80118448B7
:1047200000EB411006F077FEDDF8300700287DD061
:10473000DDF83807002879D199F80000DDF8304716
:1047400048BBD9F81080B8F1000F24D07C4801781C
:104750007C4800780844401C4008019002200090EA
:10476000FEF7D1FDDDE90010FEF738FE2146424696
:104770000846FEF778FEFEF7D5FD7348007802285C
:1047800004BF404606F0DEFF6F480078092804BFEA
:10479000204606F0D7FF75B399F80100684D00EB8D
:1047A0004001C1EB40116948DFF8988100EB8103BB
:1047B0002A7898F80000214610444200184617F065
:1047C00084FF99F801002A7800EB4001C1EB401109
:1047D0005F4898F8003000EB81001A4421465200EF
:1047E00017F073FF89F806A099F8070040F004005D
:1047F00089F8070035E0FFE75148A04601785148A5
:1048000000780C18FEF77FFD601C40080221FEF7BF
:10481000DFFD99F801004E4D00EB4001C1EB401067
:104820004A4905EB800201EB800100E028E00846E0
:104830004346FEF7EEFDFEF775FD99F801006200B4
:1048400000EB4001C1EB401005EB8000414617F042
:104850003CFF89F806A099F8070040F0040089F8A9
:1048600007003948007803280AD199F8010000EBC5
:104870004001C1EB4011354800EB810006F062FFBA
:10488000FDF7A1FFD9F81800761C7F1C8642A8BF4F
:10489000874211DBD9F8140070B1FDF7C7FADDF8D3
:1048A0005007FCF7C5FEDDF8580788B1DDF854075E
:1048B00060B1FDF7F7FC0BE0DDF84407002818BFF6
:1048C000FDF7F0FCC3E501F026FBC0E5FDF796FC23
:1048D000BBF1000F04BF0420C9F818000BD0DDF8AD
:1048E000400789F80400DDF83C0789F80500DDF889
:1048F000380789F80600B9F818104FEA0B2040EA8B
:1049000001420023912107200AF07EFE0DF25C7D1A
:104910005846BDE8F08F0000F0840010B49F0010EE
:10492000EC840010ED8400106D850010EB84001005
:1049300084200110E9840010EA840010088A001025
:10494000EE840010EF84001073850010A42701107E
:1049500000A0001010B50024FDF73CFCFB4910F04E
:10496000020F0AD00A79002A08BF012410F0040FB0
:1049700003D04A79002A08BF012410F0010F03D0A8
:104980008879002808BF01240020002C08BF10BD32
:1049900000200870BDE81040C2E408B50F2101F006
:1049A000E7FB012804D1FFF7D5FF009001F02AFDB5
:1049B000E648017900291CBF8179002904D040799B
:1049C00000281CBF012008BD002008BD08B50F212C
:1049D00001F0CEFB012804D1FFF7BCFF009001F0ED
:1049E00011FDDA48017900291CBF8179002904D022
:1049F000407900281CBF012008BD002008BD704779
:104A0000D24910B500220A714A718A7100281CBF70
:104A1000012088700BF0D6FCBDE81040FBF7CDBC40
:104A2000002818BF0120C94908727047C748007A9A
:104A3000704710B54FF4E461C54817F03CFEBDE87F
:104A400010404FF4E461C34817F035BEC2487047C8
:104A5000C2480178C248007848434100BE4817F078
:104A60002ABE70B50646BD480478BD480578FEF7F5
:104A70004AFC29462046FEF7B1FCB4484078C0EB1A
:104A8000C001C1EB8010B24901EB40123146B2487F
:104A9000FEF7E9FCFEF746FCB2480078152818BF7F
:104AA00070BDAD48BDE8704006F0B5BC70B50446B9
:104AB000AA480578AA480678FEF725FC314628461C
:104AC000FEF78CFCA14822464078C0EBC001C1EB48
:104AD00080109F4901EB40111046FEF7C4FCFEF721
:104AE00021FCA0480078162804BF204606F093FC5D
:104AF000204670BD002818BF0120944908717047F6
:104B000010B5924C002804BFE06010BDDFF858C219
:104B100096490B7896490A7801465A4352006046F6
:104B200017F0D3FD9048E06010BD10B54C219148BE
:104B300017F0C1FDBDE810404C218F4817F0BBBDF8
:104B40008C487047002818BF012080494871704781
:104B500010B57421894817F0AEFDBDE810407421EE
:104B6000874817F0A8BD002818BF01207749887131
:104B7000704710B5754C002804BF206110BD742229
:104B80000146804817F0A1FD7E48206110BD70B538
:104B90006E4D0021044629716971A9710BF012FC58
:104BA000FBF70BFC002C14BF012000202870BDE88F
:104BB0007040FFF7B5BB2DE9F04F89B04FF4E461C9
:104BC000694817F078FD74216E4817F074FDFDF701
:104BD00001FB0446FDF728F90890FDF709FB079053
:104BE000FCF730FD0690FDF721F90020FCF720FDD1
:104BF000FDF758FB00252E4605F0EDFF012853D0A8
:104C00006846FDF798FD00285BD0684606F0C8FEB0
:104C100014F0020F1CD05548DFF84CB1DDF80890B5
:104C200090F800805248DA460778FEF76CFB0120C6
:104C3000FEF7E2FB39464046FEF7D0FB52464946B6
:104C40005846FEF710FC0020FEF7D6FBFEF76AFB85
:104C500014F0010F20D04C48DFF828B14FF00208C3
:104C600001784A48DA46DDF8109000780844401C84
:104C70004708FEF748FB0120FEF7BEFB41463846D9
:104C8000FEF7ACFB524649465846FEF7ECFB0020C7
:104C9000FEF7B2FBFEF746FBFDF795FD6D1C102DF0
:104CA00003D2FDF7FFFAA7E70126FDF7BFF8069844
:104CB000FCF7BEFC089848B1079828B1FDF7F2FA56
:104CC00004E001F028F997E7FDF798FACEBB1F4FF3
:104CD00014F0020F19D02548DFF88CC00178244861
:104CE0006346007801FB00F210200021002A0AD957
:104CF00033F9118008EB5008B8FBF0F52CF811508F
:104D0000491C8A42F4D81848F86014F0010F18D0F2
:104D10001D481C4B01781D489C4600780A184FF02E
:104D200010014FF000000AD03CF9105005EB51057E
:104D3000B5FBF1F423F81040401C8242F4D811482E
:104D4000386109B03046BDE8F08F0000988400104B
:104D500084200110088A001028910010E9840010B6
:104D6000EA8400106D85001048980010EC84001053
:104D7000ED840010689F0010B49F0010A42701105C
:104D800000A0001074A00010EE840010EF8400104A
:104D9000012070474FF43F3070474FF43F300068B8
:104DA0007047034600209A682C2A88BF2C220021D5
:104DB000B1EB920F28BF704753F821C0491C6044E3
:104DC000B1EB920FF8D37047FE4A0168914214D1BB
:104DD0004168B1F5807F10D9836800222C2B88BFF1
:104DE0002C230021B1EB930F09D250F821C0491CAC
:104DF0006244B1EB930FF8D30AB100207047012051
:104E000070474FF43F31EF4B0A689A423ED191F818
:104E100027300022012B08BF0122052804BF91F88A
:104E20002300704713DC012804BF087F7047022865
:104E300004BF91F820007047032804BF91F82100B7
:104E40007047042804BF91F82200704731E014280D
:104E500008D015280CD0162811D0172804BF1846E2
:104E6000704726E0002A1CBF91F82400704704E038
:104E7000002A1CBF91F8250070472D207047002A9A
:104E80001CBF91F82600704728207047052812D0D3
:104E900007DC01280DD002281CBF032804280AD0F3
:104EA00007E0142818BF1528E7D01628ECD01728DB
:104EB00001D0FF207047002070472DE9F047ADF585
:104EC000007D00244FF40071684617F0F4FBFF20CA
:104ED000A04660F307082D20254660F3070560F320
:104EE0000F25282060F317454FF43F37B54E64F384
:104EF0001F654FF481794FF02C0AFF224FF40071A7
:104F0000684617F0F6FBCDE902A4CDE90648059402
:104F10000A94CDE900690494CDE908453846FEF7C6
:104F200025F869463846FEF7C3F8012818BF002067
:104F30000DF5007DBDE8F0872DE9F047ADF50C7D5E
:104F4000894605461F4690464FF0000A4FF400710F
:104F50006846949E17F0AFFB4FF0000CCDF800C2EE
:104F60004FF43F34CDF804C2CDF808C2CDF80CC2DE
:104F7000CDF810C2CDF814C2CDF818C2CDF81CC2BD
:104F8000CDF820C2CDF824C2CDF828C28D492068C2
:104F9000884206D0FFF791FF0DF50C7D5046BDE825
:104FA000F087D4E901120DF5007AE3688AE80F0072
:104FB00004F110010DF5047A0FC98AE80F00D4E955
:104FC0000801A26A8A92CDE9880184988DF820921E
:104FD0008DF82182401C8DF822728DF81C528DF8BC
:104FE00023628490002D14BF8698859800F10100FB
:104FF00014BF8690859080AB82980021CDF80CC2BA
:105000002C2894BF02462C220020B0EB920F06D22F
:1050100053F820C0401C6144B0EB920FF8D34842D3
:105020008390FF224FF40071684617F062FB80AC5A
:1050300094E80F008DE80F0084AC94E80F0004ACF6
:1050400084E80F00DDE988018A9A4FF43F34CDE906
:1050500008010A922046FDF789FF69462046FEF7BF
:1050600027F8012818BF00200DF50C7DBDE8F0875A
:105070002DE9F041ADF50C7D0F46804616464FF404
:105080000071684617F017FB002580954FF43F34F8
:105090008195829583958495859586958795889544
:1050A00089958A9547492068884218D16068B0F58B
:1050B000807F14D9A06821464FF0000C2C2888BFAF
:1050C0002C200023B3EB900F11D251F823205B1C4E
:1050D0009444B3EB900FF8D3BCF1000F07D0FFF767
:1050E000ECFE002804BF0DF50C7DBDE8F0810FCC6F
:1050F0000DF5007C8CE80F000FCC0DF5047C8CE8DE
:105100000F00D4E90001A2688A92CDE988018DF8E8
:1051100024828DF825728DF8266201208DF82702F1
:105120008298002180AB83952C2894BF02462C22C4
:105130000020B0EB920F06D253F820C0401C61440F
:10514000B0EB920FF8D348428390FF224FF40071E6
:10515000684617F0CEFA80AC94E80F008DE80F0097
:1051600084AC94E80F0004AC84E80F00DDE988010A
:105170008A9A4FF43F34CDE908010A922046FDF7A0
:10518000F5FE69462046FDF793FF012818BF002071
:105190000DF50C7DBDE8F0812DE9F04F0A4D4FF083
:1051A000000885B06C4246461720FFF72AFE4FF4F0
:1051B0003F3284460349106888421CD15068B0F5DC
:1051C000807F03E04353494DF1D8FFFF13D9936823
:1051D00000212C2B88BF2C230020B0EB930F80F0F4
:1051E000F98052F82090401C4944B0EB930FF8D35B
:1051F000002900F0EF80FFF760FE002804BF05B033
:10520000BDE8F08F1420FFF7FCFD02901520FFF79A
:10521000F8FD00901620FFF7F4FD40B20190162033
:10522000FFF7EFFD404240B20390FCF7D3FFDFF8F9
:10523000B4918246002089F8040089F8050089F8B5
:1052400006000BF0BFF8FBF7B8F8002089F8000063
:10525000FFF766F81AF0010F05D017F04FFA012892
:1052600008BF48F001081AF0020F7BD05E48002604
:1052700090F800E05D48037899F80100C0EBC001A8
:10528000C1EB80105A4901EB401299F80300A3EBDF
:10529000000984468145C4BFAEEB0C01A1F1010BAE
:1052A0001CDD61468B4516DD01F1010A01FB030798
:1052B0000AFB030A32F8177032F81AA0A7EB0A07A4
:1052C0003FB2002FB8BF7F423FB2B742C8BFBEB2A5
:1052D000491C8B45E8DC401C8145E2DC0098002835
:1052E00018BF864288BF48F002080027E246AEEBAE
:1052F0000A0000905045C8BFA9F1010B1BDD6046B4
:10530000834513DD0AFB030132F811E002EB410192
:105310004988AEEB010109B20029B8BF494209B280
:10532000B942C8BF8FB2401C8345EBDC00980AF13C
:10533000010A5045E3DC0298002818BF874288BF65
:1053400048F00408E2460098504516DD614689455C
:105350000EDD0AFB031032F91000A842C8BF054653
:10536000A04200E013E0B8BF0446491C8945F0DCC8
:1053700000980AF1010A5045E8DC0198002806DD92
:10538000854202DC0398844201DA48F00808FF2FC6
:1053900088BFFF27FF2E88BFFF267F2DC8BF7F2530
:1053A00004DC15F1800FB8BF6FF07F057F2CC8BFFC
:1053B0007F2404DC14F1800FB8BF6FF07F04E0B2EB
:1053C0000090EBB2F2B2F9B24046FFF7B5FD05B07E
:1053D000BDE8F08FBCF1000F18BFBCF1010F3FF426
:1053E00011AF08E798840010EA840010E9840010E7
:1053F00084200110FE4800787047FD4840787047CF
:10540000FB48002181710171017241728172704704
:10541000F74920F07E40C8617047F548C069704781
:10542000F348008A7047F248408A7047F048B0F964
:1054300014007047EE48B0F916007047EC48B0F918
:1054400018007047EA48C07A7047E9488078002819
:1054500018BF0120704710B54FF4E461E54817F01C
:105460002AF9E3490020887010BD084318BF70472F
:10547000DF48C16911F0807F08BF7047DE490968C5
:10548000C96D11F4003F08BF704700211170182149
:10549000C18170472DE9FF5FD8480027DDF83CA0A7
:1054A00005780E98119E8B46B9463C4650452CD047
:1054B00006FB050E10983BF91EC006FB05093BF9DB
:1054C0001900BCEB000148BFA0EB0C0106FB05A8CE
:1054D0003BF91840B4EB000C48BFA0EB040C01EB07
:1054E0000C0004B232F91EC032F91900BCEB000105
:1054F00048BFA0EB0C0132F918C0BCEB000248BF5A
:10550000A0EB0C0288180FFA80F9012B37D04FF06E
:10551000010817F0F8F8BA49002C0A7807DD10994D
:1055200006FB05113BF911101431282909D80099FF
:10553000B1F914103C2904DC0099B1F916103C298A
:1055400026DD0E9902EB0A0C11448C4520D9129BE2
:10555000139D13442A448B421CBF8D1A15F1020F70
:1055600030F9115000EB4106B6F90260A5EB0605D3
:1055700008D01E353C2D08D94FF0000808E0A145A1
:105580000CDD0AE00A35142DF6D8491C8C45E2D80A
:10559000A14503DDB8F1000F00D0012704B0384663
:1055A000BDE8F09F70479248B0F90C0070479049F1
:1055B000002088817047934A0280428000218280C7
:1055C000C1800181534243818181C1810182418235
:1055D0008182C182028370478548406A70470028F3
:1055E00018BF012082494862704710B506F006FDD9
:1055F00041F28831884294BF0120002010BD7C48D0
:10560000006A70477A490862FAF7E1BE7849886211
:1056100070472DE9F04F7C4987B002240A7877491A
:10562000A2F1020C521E91F8008000210091A8F115
:105630000101CDE9011C00212546A8F102090B4614
:10564000BCF1020F84BFA9F1010CCDF80CC05FD9E9
:105650004FF0000CCDF814C0CDF810C0AC464D454D
:1056600051D2039F04FB08C6BC450FD230F9167017
:1056700000EB4606B6F90260B7EB060E48BFA6EB94
:10568000070EBEF1320F01D9E34608E00CF1010C20
:10569000E145E6D8DDF814C0BCF1000F1BD0A9F13C
:1056A000010CAC4517D304FB08C665450FD230F991
:1056B000167000EB460636F9026CB7EB060E48BFD3
:1056C000A6EB070EBEF1320F01D9E24608E0ACF1BD
:1056D000010CAC45E7D2DDF810C0BCF1000F12D0D0
:1056E0004FF0010CCDF800C0DDF804C0DC4588BFE8
:1056F000CDF804B0514538BF5146A24288BF22467A
:10570000A34238BF2346641CDDF808C064459FD31C
:105710003748DDF800C0846A644518BFC0F828C067
:10572000019807B0BDE8F04F12F05ABE2DE9FF4FC7
:105730008BB00446DDE918B72D480025057045708B
:105740000AF051FE002840F0428100F08DFB052850
:1057500068D0DFF89CA0DDF830902C499AF80B0057
:10576000029025480978006890F8726000912449F9
:1057700009780191B0F97080BAF916003228BAF8A8
:10578000100005DA002804BF7006060E05D100E0FF
:1057900018B99AF80300012842D10AF063FEB8BB99
:1057A000012F3DD0BBF1010F03D1BAF81200C82878
:1057B00036D8BAF81200002804BFBAF81000002842
:1057C0002ED00AF0FCFD01282DD0B9F80000AAF86F
:1057D0000C00DDE9001200208A181DD039F91010E4
:1057E000BAF90C309942C8BFAAF80C10401C10E05E
:1057F000B4840010E8A0001048860010E98400106E
:10580000EF840010F1D8FFFFEA840010EE8400104E
:1058100006E080B28242E1D8BAF90C0040450EDDC4
:105820008AF8095028E0F748006890F873600298F9
:10583000012814BF4FF03C084FF04108C5E7DAF8E3
:105840001C0010F4803F17D0EE480068C06D10F4C3
:10585000803F11D09AF80900401CC0B28AF80900B4
:10586000B04209D91020AAF80E0001208AF80700DA
:105870004FF0FF348AF809500AF0A1FD012871D1D8
:10588000E048BBF1000F00680A9090F874106BDCE0
:10589000012F69D0DC4AD06910F4003F11D00A987A
:1058A000C06D10F4003F0CD0107A401CC0B21072D2
:1058B000884206D91120D0810120D0714FF0FF34E9
:1058C00015720C980090D1484FF0000B012F007812
:1058D0000390CF48007801900A9890F873000690E2
:1058E00045D001984008079003984008099000208F
:1058F000049082460590DDE9001001EB4000029023
:1059000000231A461946BAF1000F0CBFDDE90076F4
:10591000DDE902760020002E88BFA6F1010E29D90C
:1059200037F91080B8F1640FD8BF002214DD70453C
:105930000DD207EB400CBCF902C0B8EB0C0948BF14
:10594000ACEB08090FFA89FCDC45A8BFE346491C0B
:10595000002A04BF01225B1C401C8642E0D8012BB8
:1059600005D807E033E0FFE7A7480572A9E7A64896
:1059700085722CE0BAF1000F0CBF049105910AF179
:10598000010ABAF1020FBBD3079904988842EED9F5
:10599000099905988842EAD9BBF1320FE7DC9A49A8
:1059A000887A401CC0B28872CA6912F4801F0ED077
:1059B0000A9AD26D12F4801F1CBF069A904206D933
:1059C0001420C8810120C8714FF0FF348D7211F08E
:1059D000D4FD10F4807F29D000F046FA022825D1AA
:1059E0004FF0010816F094FE074611F0AEFD064692
:1059F00011F0A7FD024600210020002E08D900FB6F
:105A0000021337F913300F2B10DB401CB042F6D3D2
:105A1000B8F1000F0AD0491C0129EDD9B8F1000FE7
:105A200004D0794901204FF0FF34C8710DF087FC94
:105A3000032823D1744800950195817B8DF80010CF
:105A4000BDF8001064F30F21ADF800108279BDF8A5
:105A5000021062F30301027962F30711C27962F363
:105A60000821427962F34921ADF802108089ADF82E
:105A700004000222062168460DF064FCB4F1FF3FE9
:105A80002AD0002C1CBF0FB0BDE8F08F5E4C6079AF
:105A900001281CBF0FB0BDE8F08FFEF7D9FF65717C
:105AA000012020704FF4E4615A4816F004FEA570FE
:105AB00000F0E0F904280D982CD0002818BFFEF75C
:105AC000D1FB0E98002804BF0FB0BDE8F08F0FB0D7
:105AD000BDE8F04FFEF74FBB4B4CE07901281CBFEF
:105AE0000FB0BDE8F08F0D98FEF7BBFFE571012008
:105AF00060704FF4E461474816F0DDFDA5700D9825
:105B0000002818BFFEF7AEFB0E980028DFD10FB0BB
:105B1000BDE8F08F002818BFFEF768FB0E9800283C
:105B200004BF0FB0BDE8F08F0FB0BDE8F04F16F026
:105B3000F4BD2DE9FF4F0446324887B0984600680F
:105B4000B0F866B011F067F9012804BF4FF6FF7096
:105B500000EA4B0BB8F9141001232046149A16F0F2
:105B6000E1FD294F00200546F870FEF735FB06469B
:105B70002948047800F078F9052898F80C001DD021
:105B8000B8F80EA0C2B2924551D31E48B8F808909A
:105B9000B8F80A30D0F8008009F0FF018B4228BF26
:105BA000B8F960C03ED302FB041036F9100000289B
:105BB000B8BF4042604531DD012538E0B8F80E90AD
:105BC000C0B2814533D30F49B8F808C0B8F80A20ED
:105BD000D1F800800CF0FF018A4224BFB8F9603090
:105BE0005B4209D300FB041A36F91AA09A45E3DB9D
:105BF000491CC9B28A42F5D2CDB9401CC0B2814518
:105C0000E8D214E048860010B4840010EE8400103E
:105C1000EF840010E8A00010E9840010481CC1B215
:105C20008B42C0D21DB9501CC2B29245B4D280483A
:105C3000C57011F0A2FC10F4817F0CD11498B0F95A
:105C40001200002807DC0AF0BAFB012803D07848CC
:105C5000C07801287DD147F6FF70039075484FF05A
:105C60000009099E90F800A073484D46159C0778DE
:105C700011F083FC10F4817F1DBF70480068B0F8FC
:105C8000620058460FFA80F811F077FC10F4817F1B
:105C90001FBF6A480068B0F86200404208BFCBF1FD
:105CA000000000B2029011F068FC10F4807F19BF70
:105CB0004FF0010B4FF0220C4FF0000BBC460020C0
:105CC000CDE9000A0398804569DA009ABAF1000F1D
:105CD0007CD9ACF101000590AAF101000490ACF16F
:105CE000020003905846E34538BF0FFA82FA51D2BA
:105CF00002FB070399B236F911100029B4BFC1F1B4
:105D0000000E8E46C6451CDD41450CDDB4F904E0AD
:105D1000714503DDA180E080A4F808A009F101012C
:105D20000FFA81F90DE0DDF808E08E4509DDB4F9E0
:105D30000AE08E4503DD6181A081A4F80EA0691CF4
:105D40000DB20599884222D236F913E006EB4301E1
:105D500000E041E0B1F90230BEEB030148BFA3EB24
:105D60000E0109B2009B9A421CBF049B9A4204D0C8
:105D700058451CBF039B984204D1B4F902308B42B2
:105D8000B8BF6180B4F900308B42B8BF2180401C9D
:105D90006045ADD30198521C8242A3D316E000980F
:105DA000BAF1000F12D95B46E3450CD200FB073174
:105DB00089B236F9112002998A42BCBF691C0DB222
:105DC0005B1C6345F2D3401C5045ECD3A4F8109003
:105DD00065821799012008701598B0F91000002805
:105DE00008DC1598B0F91200002803DC1048C078D0
:105DF000012809D1052347F6FF71169A089816F075
:105E000091FC1899012008701498418A0848018271
:105E10001499098A4182149949898182149989883F
:105E2000C1821699098A01830BB0BDE8F08F00008A
:105E3000B4840010EA840010E98400104886001041
:105E400010B506F0EDFD06F08EFE002010BD00003E
:105E5000FD49C8707047FC48C0787047FA4908711E
:105E60007047F94800797047F74800787047F6485E
:105E700080787047F4480078022805D005281CBFB8
:105E80000020704706F0B1B80AF07CBAEE490870FD
:105E90007047ED4948707047EB484078704770B5DF
:105EA000E94E04460D463078A04212D002281ED09A
:105EB000052814BF002006F098F844EA052132783E
:105EC000002341EA024141EA00626121072009F012
:105ED0009BFB3078844218BF7070B570072C28BFC8
:105EE00070BDDFE804F016070B13160F16000AF05A
:105EF00049FAE2E7284600F093FA0AE028460AF059
:105F0000E9FA06E0284606F065F802E0284609F0BE
:105F10008BFC347070BDCD4900200968B1F89C102D
:105F200011F4807F08BF7047FCF749BFC7490020C4
:105F30000968B1F89C1011F4807F08BF7047FCF726
:105F40004DBFC24900200968B1F89C1011F4007FD0
:105F500008BF704716F0EBBBBC4900200968B1F8D8
:105F60009C1011F4806F08BF704716F0E5BBB6496E
:105F7000487900281CBF401E4871704770B5B4496D
:105F8000D1F8CC00B04C10F0030F0AD040F4BE00A2
:105F900040F02040C1F8C8006079002804BF01200B
:105FA0006071AC488068A94D10F0020F296807D1D4
:105FB0004FF04020406910F0010F01D0607940B1EE
:105FC000B1F89C10002011F4807F18BFFCF706FF89
:105FD00007E0B1F89C10002011F4806F18BF16F094
:105FE000ABFB9D49084208BF70BD2968D1F89C10E1
:105FF000090C617170BD10B572B6FEF735F8BDE8D9
:106000001040FDF784BD10B5012802D0022805D04C
:1060100008E04FF44330FCF7A9FF03E04FF04021C4
:106020008E48086772B6FEF71FF8BDE81040FDF70E
:106030006EBD854900288A7918BF01208871C0B2D9
:10604000824208BF70470022002818BF01220023A7
:106050000121022009F0D8BA7B488079002818BFB6
:106060000120704770B5784C0028E57918BF0120F1
:10607000E071C0B2FAF797F9E079854214BF0028C1
:1060800070BD207802281CBF052870BD0221BDE824
:10609000704004E76C48C079002818BF01207047A1
:1060A0006948007A70472DE9F041674E00281CBF0F
:1060B0000020307204D1307A002818BFBDE8F0818A
:1060C0004FF040273D6B0120FDF7C1F80420FDF79C
:1060D000BEF8634C0520E066FDF7DDFF40F2CF70AF
:1060E000216F11F0010F04D0307A40F00E003072B1
:1060F00003E0011EA0F10100F2DC307A78B1FDF777
:10610000CAFF5848216F11F0040F04D0307A40F0D4
:106110000100307203E0011EA0F10100F2DC45F441
:10612000BE0040F020403863BDE8F08146488069F9
:10613000704745484069704743484069002818BF88
:10614000C07A70474049C86170473F48C06970478E
:106150003D49086270473C48006A70473B48026806
:1061600002F5BE73118A508A02F59E72FCF75FB980
:106170002DE9F04FDFF8D0A099B00F460646CAF8D7
:10618000180006F06EFBCAF8140000286CD090F8D6
:1061900000C08AF809C041788AF80A10837804465A
:1061A0000CF101008AF80B3000F0FE008AF80C00B8
:1061B000E2788AF80D2020798AF80E0060798AF852
:1061C0000F000AF1110500202870687020788AF805
:1061D00010006046FCF77BFA9AF80F109AF80E0050
:1061E000FCF798FA6946204606F064FBE089DAF885
:1061F0001C5000281CBF6843050BB4F81290DAF855
:1062000020B0B9F1000F08BF4FF48059B4F81680E0
:10621000B8F1000F08BF4FF480584FF4805017902A
:10622000002017F0040F18BF4FF4857017F0080F07
:1062300018BF40F0040017F0020F1CBF40F201210C
:10624000084317F0010F10E0E084001048860010AA
:10625000006000400080004008000300AD2007B04F
:10626000001000403F0D03002BE018BF40F4846095
:10627000E1696FF30F0708406FF30F01084307430D
:106280000098109004981190089812900020149093
:1062900001981390A07A16900798159010A9384687
:1062A000FBF792FE17F0020F6FD006F034F918B129
:1062B00001460020FBF7DBF9012E18BF022E22D188
:1062C0000CE055480068B0F89C0010F4807F18BFBF
:1062D000FCF784FD002019B0BDE8F08F0AF060F9EA
:1062E00088B111F0BCF908280DD04B480068B0F80F
:1062F000281141B10020FBF7BAF92A23B522032166
:106300000020FAF797FB06F01DF96843050B06F02D
:1063100039F90BFB00F0000B4030C1090A200122C3
:1063200002FA00F30B4201D1401EF9D5461F207B33
:10633000002818BFA0F1010B02D1FBF78FFA8346AA
:10634000607B002814BF401EFBF7C8FA0BEB060168
:10635000052903DD711A4E1D052103E00029BCBF8C
:10636000761A00210644052E03DD701FC540052660
:1063700004E0002E02DA7042854000260020FBF780
:1063800086FA31460020FBF7C2FA17F0010F17D04A
:10639000207C18B1411E0120FBF779FA207D18B14D
:1063A000411E1120FBF773FA607C18B1411E0120D9
:1063B000FBF7ADFA607D18B1411E1120FBF7A7FA7B
:1063C000E07A00281CBF0001FBF782F8029806F073
:1063D00082F8039830B12B469AF80A209AF80910EF
:1063E00016F0AFF9424649462846179B16F0AEF91B
:1063F0000598FEF785FB0998FEF7BBFB19B0012055
:10640000BDE8F08F10B5FBF7A6FE06F06CF8034967
:1064100000204861012010BD48860010E084001073
:10642000FB4908707047FA4800787047F94810B483
:10643000F94A016891421CD14168B1F5987F18D89A
:10644000D0F808C00146BCF5007F12D800220B46E8
:106450001146B2EB9C0F24BF10BC704753F821408B
:10646000491C2244B1EB9C0FF8D3002A04BF10BC96
:106470007047002010BC7047E648FCF777BDE44940
:1064800001200870704770B50E4605461024FFF7CE
:1064900050FE15F0020F18BF052403D115F0010FAF
:1064A00018BF09243246102C28BF70BD002A08BF2F
:1064B00070BD204490F920102046BDE8704006F0E1
:1064C0002CBAF0B581B0ADF5805D0446FFF731FE22
:1064D000054614F0020F0AD0684604270646FCF76A
:1064E00077F995F924103246384606F016FA14F07A
:1064F000010F02BF01B00DF5805DF0BD08266946B1
:106500000C460120FCF7B8F995F9281022463046D0
:1065100006F003FA01B00DF5805DF0BD2DE9F34FF3
:106520008BB0002005900868029048680390087AB4
:106530000190487A0090887AB1F90C90B1F90EA0D8
:10654000CA690792D1E908840A8A4969C0F5807648
:1065500002EA000706910B9810F0010F16D0009880
:106560004FF0000E002840F2F6800121069801FA53
:106570000EF2104018BF012004900EEB4E010020D7
:1065800001EB0E1183460A9100F0DCB80020FBF706
:10659000A7FA0546DDE900014843032101EB40006D
:1065A00020F003024146204616F08FF82846FBF7FC
:1065B00097FA00980025002840F2CD800122069825
:1065C00002FA05F1084018BF01200021049005EBF4
:1065D000450000EB05108C4609904BE04A0902A8E3
:1065E00001F01F0350F822200120984002423ED0C3
:1065F00038F9020B049AA0EB0A000CF1010C002AF6
:106600000CBFA9EB000409EB000401F0010207989C
:106610004FEA510B00EB4232099802EB80000890E0
:1066200050F82B20C2F30720D3B212F4803F02D0DF
:10663000002C02DB03E0002C01DD9C1B00E09C1918
:10664000BC4205DDFF283ABF0024401C3C4606E062
:10665000002C04DA0028C6BF3C46401E002402F489
:10666000803242EA0020089A204342F82B00491C5D
:10667000262902D201988445B0D300986D1C85422A
:106680009CD368E0420902A900F01F0351F82220C0
:10669000012199400A4252D034F9021B049AA1EB1D
:1066A0000A010BF1010B002A0CBFA9EB01014944BF
:1066B00038F9022BA2EB0A0214BF4A44A9EB0202EA
:1066C0000029B4BF4B420B46002AB8BF52429A423F
:1066D00035D9079A00F0010302EB43330A9A03EB22
:1066E00082024308CDE9083252F82330C3F307226F
:1066F00003F0FF0C13F4803F02D0002902DB04E01A
:10670000002902DD0CEB060501E0ACEB0605BD42FD
:1067100005DDFF2A3ABF0025521C3D4606E0002D4C
:1067200004DA002AC6BF3D46521E002503F480311C
:1067300041EA0221DDE90823294343F82210401CE5
:10674000262802D201998B459CD300980EF1010EA8
:106750008645FFF40AAF0B98032826BF0120059059
:1067600005980DB0BDE8F08F2DE9F04F8BB00022F9
:1067700004920A6800924A6801920B7A4D7A8E7AE6
:106780000396B1F90C40B1F90E200592D1E907C288
:106790004E690696098A039EC0F1080801EA0607B9
:1067A00000B3B8F1000F6EDB4FF0000A002D6BD97B
:1067B000012000FA08FBA8F10100012101FA00F014
:1067C0000A904FF00109069809FA0AF1084018BF2B
:1067D0000120002102900AEB4A0000EB0A100E464D
:1067E0000990ACE04FF0000A002D4DD94FF001099F
:1067F000069809FA0AF1084018BF0120002102900A
:106800000AEB4A0000EB0A100E4608904EE000002A
:106810000485001000FE0200544352464FEA51190D
:1068200001F01F0B5DF82990012000FA0BF019EA26
:10683000000F38D032F9029B0598761CA9EB0000B6
:10684000DDF80890B9F1000F0CBFA4EB000904EBD0
:10685000000901F001000CEB403B08980BEB8000B5
:106860004FEA510B079050F82B0010F4803F0CD0EA
:10687000B9F1000F11DA10F47F4018BFA0F5807055
:1068800040F4803009E068E060E0B9F1000F04DD19
:1068900010F47F4018BFA0F5807040F08000DDF854
:1068A0001C9049F82B00491C262901D29E42B5D3E1
:1068B0000AF1010AAA4599D348E04FEA511901F0BB
:1068C0001F0E5DF82990012000FA0EF019EA000F62
:1068D00032D032F9029B0598761CA9EB0000DDF856
:1068E0000890B9F1000F0CBFA4EB000904EB0009FC
:1068F00001F001000CEB403E09980EEB80004FEADE
:10690000510ECDE907E050F82E0010F4803F03D07F
:10691000B9F1000F05DA02E0B9F1000F01DD20EA5C
:106920000B00B8F1000FC4BFDDF8289049EA000061
:10693000DDE9079E4EF82900491C262901D29E4216
:10694000BBD30AF1010AAA45FFF43BAFB8F1000F2F
:10695000C2BF04980BB0BDE8F08F0026002D35D9DA
:106960000398C0F5807A40F4807E002006EB460153
:10697000024601EB061B24E0440900F01F085DF805
:106980002440012101FA08F10C4217D000F0010166
:106990000CEB413101EB8B094FEA5008521C59F8BE
:1069A0002840E1B201EB5A0101EA0E01B94288BF69
:1069B000394624F0FF04214349F82810401C2628BA
:1069C00001D29A42D8D3761CAE42CED30120049095
:1069D0000BB0BDE8F08F2DE9F04F89B00022049292
:1069E0000A6800924A6801920E7A4A7A0292D1E9C4
:1069F0000772B1F90C30B1F90E5049690591FE49A1
:106A0000C968A0EB010CCCF10808814245D845D1FA
:106A100002984FF0000900283FD90121059801FA9A
:106A200009FC1CEA000018BF01200390002009EBBC
:106A30004901844601EB091B28E0440900F01F0AC4
:106A40005DF82440012101FA0AF10C421BD032F911
:106A5000021B039C491B0CF1010C002C0CBF5C1A9F
:106A60005C1800F0010107EB413101EB8B0E4FEA9E
:106A7000500A002C5EF82A10C8BF41F4803141F45E
:106A800000414EF82A10401C262801D2B445D4D328
:106A9000029809F101098145BFD35CE0B8F1000F0C
:106AA0005EDB02984FF00009002854D908F1080075
:106AB000012101FA00FA401E01FA00F008900124B9
:106AC000059804FA09F1084018BF0120002103903D
:106AD00009EB490000EB09108C46079034E04C09A3
:106AE00001F01F0B5DF82440012000FA0BF0044276
:106AF00027D032F9020B039C401B0CF1010C002C37
:106B00000CBF1C1A1C1801F0010007EB403B079852
:106B10000BEB80004FEA510B069050F82B0010F45D
:106B2000803F02D0002C04DA01E0002C01DD20EAD5
:106B30000A00B8F1000FC4BF089C2043069C44F82B
:106B40002B00491C262901D2B445C8D3029809F16B
:106B500001098145B3D3B8F1000F04BF01200490AF
:106B6000049809B0BDE8F08F2DE9F34FADF5757DC0
:106B700000208846E790E69072B6FBF72BFB0746AD
:106B8000FDF78FF848B1FDF731F9E790FDF718F9F7
:106B9000FDF731F9E690FDF71EF9FBF70AFAFBF76E
:106BA00043F9ED90FBF724FBEC90FBF73FF9FBF783
:106BB000B5FBE8900020FBF7A7FB0120FAF72CFFBC
:106BC000F0901120FAF728FFF190FCF78BFEEB9084
:106BD000FCF770FE4FF49350FCF7D9FD62B6FAF75C
:106BE000F7FEEA900120FAF7E9FEFAF700FFE990D4
:106BF0000020FAF7F2FE0120FAF772FFF29000206F
:106C0000FBF75DF9EF900020FBF74CF9EE900020C8
:106C1000FAF70EFDF39000200546D4AE46F820505A
:106C2000401C0628FAD3DFF8D49117F0020F4FF07A
:106C300001040AD041F618514846D49415F03BFDA2
:106C400041F618516E4815F036FD17F0010F15D0BA
:106C50004FF498716B4815F02EFD4FF498716A4807
:106C600015F029FD0120F9F7A9FE002818BFD694D8
:106C70001120F9F7A3FE002818BFD794DFF88CA1E4
:106C8000D4985D4F4FF0405B002830D0002108467B
:106C9000FAF7D2FD989001210020FAF7CDFD9990E6
:106CA0009AF800008DF8680259480078012894BFCE
:106CB0005848594800788DF869020020FAF7F7FE25
:106CC000002814BF00204FF0FF309D908DF86A829D
:106CD0007888ADF86C02ADF86E520020FAF779FDB5
:106CE000ADF870024D48CDF87C92CDE9A0B0D598B2
:106CF0004FF0FF0878B300210846FAF79DFDA290F7
:106D000001210020FAF798FDA3909AF800008DF871
:106D100090028DF89142A7958DF892827988ADF80E
:106D20009412ADF896520020FAF753FDADF8980290
:106D30009DF8690200EB400101EB001109EB8101B4
:106D4000A9919DF8681248430BEB4001AA91334981
:106D500001EB4000AB90DFF8C890DFF8C8A0D698F0
:106D600080B300210120FAF767FD0121AC900846AD
:106D7000FAF762FDAD90FAF7E2F900280CBF9AF835
:106D8000000099F800008DF8B8020120FAF766FDBE
:106D900004FA00F08DF8B9020120FAF73DFEB19037
:106DA0008DF8BA82B888ADF8BC02ADF8BE520120A9
:106DB000FAF70FFDADF8C0021248B3901A48B4902C
:106DC0001A48B590D79898B300211120FAF734FDEE
:106DD000B69001211120FAF72FFDB790FAF7AFF91D
:106DE00000280CBF99F800009AF800008DF8E00226
:106DF0001120FAF733FD1CE00485001000800030FC
:106E000000A00030189D003018BD0030EC84001048
:106E1000EB840010EA840010ED8400100040003084
:106E2000EE840010EF840010CC090030CC49003013
:106E300019E004FA00F08DF8E1021120FAF7ECFDF8
:106E4000BB908DF8E282B888ADF8E402ADF8E65266
:106E50001120FAF7BEFCADF8E802FE48BD90FE48EE
:106E6000BE90FE48BF9026A8B590CDF8D0D24CA8D1
:106E7000BE9072A8BF909DF8B9120220022988BF67
:106E80008DF8B9029DF8E112022988BF8DF8E10260
:106E90000120FAF7C1FD4FF0AA3720B13946012091
:106EA000FAF7AAFDB1971120FAF7B6FD28B14FF015
:106EB000AA311120FAF7A0FDBB97BDF8BE0200F57C
:106EC0008060ADF8BE02BDF8E60200F58060ADF866
:106ED000E602FBF7E7F94FF00008C346C246474613
:106EE000C14603F078FE012800F05281BBF1800F0B
:106EF00000F24E81DAA8FBF71EFC002800F0428168
:106F0000DAA804F04DFDD69800285AD09DF8B85262
:106F10000120FAF7A3FC012101FA00F3DFF840C3D6
:106F20000020B49CB0EB450F38BF002105D224F8F7
:106F30001010401CB0EB450FF9D30021B1EB530FFB
:106F400017D20020B0EB450F38BF01FB05F20CD281
:106F500000EB420E34F810603CF81EE0764424F852
:106F60001060401CB0EB450FF2D3491CB1EB530F3E
:106F7000E7D3022B0FD90020B0EB450F38BF5A08DA
:106F800009D234F91010B1FBF2F124F81010401CB2
:106F9000B0EB450FF5D30120FAF73EFD00F00300FA
:106FA00001280ED10020002D0BD9411934F81020F2
:106FB00034F8113024F81030401C24F81120854298
:106FC000F3D8D798E8B39DF8E0521120FAF746FCC1
:106FD000012101FA00F3DFF880C20020BE9CB0EB73
:106FE000450F38BF002105D224F81010401CB0EB2B
:106FF000450FF9D30021B1EB530F17D20020B0EBAE
:10700000450F38BF01FB05F20CD200EB420E34F8FD
:1070100010603CF81EE0764424F81060401CB0EB91
:10702000450FF2D3491CB1EB530FE7D3022B11D913
:107030000020B0EB450F38BF59080BD234F91020AF
:1070400000E01DE0B2FBF1F224F81020401CB0EB90
:10705000450FF3D31120FAF7DFFC00F003000128FD
:107060000ED10020002D0BD9411934F8102034F82E
:10707000113024F81030401C24F811208542F3D838
:107080001AF1010A70D04FF0000A5046E0AD012617
:107090000BF1010B45F82060401C0628FAD3002FA5
:1070A00008BF00240DD0012F08BF00241BD0022FE1
:1070B00008BF002429D0032F08BF4FF0010835D0A6
:1070C00066E0D4A850F8240048B104EB840198A8E5
:1070D00000EBC1014846FFF77EFC45F82400641C24
:1070E000062CEED322E0D4A850F8240048B104EBDB
:1070F000840198A800EBC1014846FFF735FB45F82D
:107100002400641C062CEED310E0D4A850F8240010
:1071100048B104EB840198A800EBC1014846FFF791
:10712000FDF945F82400641C062CEED30121002053
:1071300055F82020B2B1401C0628F9D391B11F2F79
:107140000DD27F1CF59806FA07F1014207D17F1C8A
:10715000032F04D8F59806FA07F10142F7D04FF053
:10716000000901E009F10109FBF72DFBB8F1000F5F
:107170000ED1E89818B1FBF7BEF8FAF75DFCFBF703
:1071800091F8AEE6FEF7D2FEB8F1000F3FF4A9AEDB
:10719000FBF719FBFAF74AFE0120F099FAF72CFCED
:1071A0001120F199FAF728FCE898FBF7ADF8E99877
:1071B000FAF713FCEA98FAF701FCF298FAF790FC58
:1071C000EF98FAF77CFEEE98FAF76CFEF398FAF770
:1071D0002FFAED9830B1EC9810B1FBF763F801E0AD
:1071E000FBF70CF8FCF75DFD48B1E798002818BFE5
:1071F000FCF75CFDE698002818BFFCF78FFDEB98C4
:10720000002818BFFCF7FFFAB8F1000F0CBF0120EF
:1072100000200DF5777DBDE8F08F70B5114D164655
:10722000D5F844231205120D28D000281CBFC1F345
:107230000800FBF74EFDD5F8480340F00100C5F803
:107240004803D5F8480320F00100C5F848030022A0
:10725000341E09E0B09D0030CC0E0030CC4E003022
:10726000CC0900300050004023DDD5F8481340F22F
:10727000D32011F0010F08D1401E01D2002070BDB3
:10728000D5F8481311F0010FF6D0D5F84403C0F338
:107290000B000244D5F8480340F00100C5F848034C
:1072A000D5F8480320F00100C5F84803641E002CFF
:1072B000DBDC1001B0FBF6F080B270BD2DE9F84FB9
:1072C000040016D0FE48006CC0F30829FBF711FD3E
:1072D00049EA004200237621072008F095F9F94891
:1072E000D0F8401341F48031C0F84013962000904C
:1072F0000AE0FBF7F9FC0120BDE8F88F00BF00BFF2
:1073000000BF00BF00BF0846411E0091F6D24FF0FB
:10731000000840F2FF17C246464608EB070000EBA4
:10732000D0704510A9B264220120FFF776FFF0B1BA
:10733000A04288BF6F1E38BF05F101081ED1AA46C2
:107340001FFA8AF14FF064024FF00100FFF765FF6A
:107350000446002352467721072008F055F9A4F58A
:10736000B0504B38A0289CBF0120BDE8F88FB9F180
:10737000000F10D04846FBF7ACFC0EE0011B48BFE5
:10738000211A321B48BFA21B9142BCBFAA46064627
:10739000B845C2DDD4E7FBF7A7FC49F480320023EF
:1073A0007721072008F030F90020BDE8F88F2DE99B
:1073B000F05FC54CADF5965D01272678FEF754FDCC
:1073C000012840F07B8104F0EFFCC0480068B0F970
:1073D0001E10B0F91C0015F0BEF916F0020F00F0F7
:1073E000648101ADFFF722F84FF00008A8B1B0E8C2
:1073F0000E1001AC84E80E10B0E80E1005AC84E865
:107400000E10B0E80E1009AC84E80E1070E80C12F3
:10741000806B0D91CDE90E2022E0FF223C21284611
:1074200015F067F9AA4801904FF4987002903C203B
:10743000CDE903085020CDE905084FF0FF30CDE934
:1074400008800A90ADF83C800C908DF83E800B903F
:10745000CDF81C80CDF83480CDF838808DF83F8091
:107460009C48FBF783FD0698401C0690FAF7A1FDA7
:1074700041F29B60FFF722FF93498860FAF74AFECA
:1074800040F277790025CDF800807CE0284605F0B1
:10749000E8F9002876D0008900EA090424F0CC003D
:1074A00030F47C406ED00F212846FEF761FE0028A4
:1074B00068D0FAF78FFE0099002961D1FAF761FDD3
:1074C000FF210F20FFF750FB0090FAF7AFFC009868
:1074D000002855D147B314F0010F0ED0FEF729FE56
:1074E00082460420109011A88346FBF771F99AF99F
:1074F00024105A46109805F010FA14F0100F11D00D
:10750000FEF717FE8246082041F2440169441090BC
:107510008B460120FBF7B0F99AF928105A461098CB
:1075200005F0FBF9009858BB14F0660F06D0FDF784
:1075300042FB0090FAF77AFC009808BB07B314F0FE
:10754000020F0DD0FCF7D2FE8246FEF7F2FD0523B6
:107550005FEA0A0204D090F92510184605F0DDF91B
:1075600014F0200F0CD0FCF734FE0446FEF7E1FDCA
:107570000923220004D090F92910184605F0CDF90E
:10758000FEF740FF6D1C05F068F9A842009803D98A
:1075900000283FF47BAF03E0002808BF012000D0A3
:1075A000002018B1FDF7F4FB01281FD00898002334
:1075B000401C0890502005901A462121072008F011
:1075C00023F800231A461946FE20CDF80080FDF767
:1075D000B3FC01AC05F019F950B381690991C16997
:1075E0000A9141690B91C0680C9027E016F0080FD2
:1075F00014BFA220A12005903348816859B13049B9
:10760000096CC1F30821ADF83C109DF83E10491CEF
:107610008DF83E1006E0ADF83C809DF83F10491C07
:107620008DF83F10C0F808800798401C0790D0E7FD
:107630004FF0FF300C900B900A9009902448019075
:107640004FF4987002903C20CDE903080021A36814
:107650002246084652F820C0401C6144B0EB930F0C
:10766000F8D34D4210AFFF224FF400713846E56069
:1076700015F03FF8A368F4E8040287E82D000FCC6A
:1076800014AD85E80F000FCC18AD85E80F00D4E9E4
:107690000001A2680F4CCDE91C011E922046FBF7A9
:1076A00065FC39462046FBF703FD0020FDF7A8F9ED
:1076B000002332464021072007F0A6FF0CE000001F
:1076C0000060004000500040048500104886001013
:1076D0005443524600FE02000DF5965DBDE8F05F92
:1076E00003F01EBA7D4A002804BF5180704701286C
:1076F00008BF9180704701004FF00000774A04BF37
:10770000B2F902007047012908BFB2F904007047BE
:1077100070B50126FEF78AFE20B10069A12818BFC6
:10772000A22801D0002070BD002405F096F80028A2
:1077300033D9204605F095F800281EBF058925F0AD
:10774000CC0030F47C4023D00F212046FEF710FD02
:10775000F0B115F0010F0AD0FBF74EF838B944F438
:10776000807200232021072007F04EFF002615F02D
:10777000100F0BD00120FBF79BF838B944F480526E
:1077800000232021072007F03FFF0026FEF73AFEE6
:10779000641C05F062F8A042CBD8304670BD0020D2
:1077A0007047002070474D48407870474B49002093
:1077B0004870704770B5002105220846FFF72DFD7F
:1077C0000023464A00282BD05178002908BF1361B6
:1077D000A0F5A05CACF5257CBCF10E0F20D9491CAE
:1077E000C9B25170D2F810C00A296044106121D981
:1077F0003B495370096CC1F308249CB14FF6A901B1
:10780000884294BF651C651E2846FBF762FA44EA6D
:10781000054200237521072007F0F6FE012070BD08
:10782000537007E041F29B60FFF748FD00281CBF42
:10783000012070BD002070BD10B5FEF7F7FD38B314
:10784000284A0168914223D14168B1F5987F1FD839
:10785000D0F808C00146BCF5007F19D800220B46BD
:107860001146B2EB9C0F07D253F82140491C224429
:10787000B1EB9C0FF8D35AB9188F00281CBFA0F5A4
:107880007F41B1F1FF0103D0FBF723FA012010BDC6
:10789000002010BD10B5FEF7C9FDD8B1114A01682E
:1078A000914217D14168B1F5987F13D8D0F808C03C
:1078B0000146BCF5007F0DD800220B461146B2EB05
:1078C0009C0F09D253F82140491C2244B1EB9C0F74
:1078D000F8D30AB1002010BD188F10BD0485001028
:1078E000006000405443524670470020704710B576
:1078F00003F00700042808BFFEF77DFB002010BD41
:1079000070B503F007020025FB4CFC4B012A02D0A6
:10791000022A14D011E005201870DD60FCF734F95C
:107920002268532111702268452151702268010A92
:1079300091702168C87020680571002070BD1A78A8
:10794000052A13D1DA68052A28BF104607D2D4F8D1
:1079500000C01CF802C080F800C0501CD860052888
:1079600004D10120DD60087003201870012070BD73
:1079700070B503F0070200250126DF4CDF4B012A1A
:1079800002D0022A23D020E005201870DD60FCF729
:10799000FBF82268AC2111702268010A517021683D
:1079A00088702068C6702068057104F0CFFE48B169
:1079B000D34D286804F0F6FF20B128682168007EC6
:1079C000487102E02168FF204871002070BD1A78DC
:1079D000052A12D1DA68062A28BF104607D2D4F841
:1079E00000C01CF802C080F800C0501CD8600628F7
:1079F00003D1DD600E7003201870012070BD03F00C
:107A00000702022A1CBF00207047202202700120BA
:107A1000087070472DE9F041B84F0D46064613F047
:107A2000070F04D003F00700022808D004E012F08A
:107A3000040F1CBF0020B8700020BDE8F08103F0E7
:107A400069F8002814BF0124002403F066F8002818
:107A500014BF0222002242EA0403B878002814BFAF
:107A60000422002242EA0300307001202870BDE8A1
:107A7000F08170B503F0070C0026A04C9E4DBCF1C0
:107A8000010F0AD0204613F0070F00780DD0BCF18B
:107A9000040F08BF062818D029E0E66028680670A1
:107AA000286846700520207021E005281FD1E06875
:107AB000022803D22B681A54401CE060022816D119
:107AC0000120E6600870062010E02868007855283C
:107AD0000BD128684078AC2818BFBC2805D128688D
:107AE0000122411C062002F0FBFF03202070002031
:107AF00070BD70B503F0070200257F4C7F4B012A53
:107B000002D0022A24D021E005201870DD6002F0A6
:107B1000B5FF41F6E8710144B0F53C3F10D8CA7892
:107B2000086862F31F60774A904208BF002007D1BF
:107B30000A18236812791A54401C1428F8D305E057
:107B4000002021680D54401C1428FAD3002070BD79
:107B50001A78052A13D1DA68142A28BF104607D2EA
:107B6000D4F800C01CF802C080F800C0501CD860D7
:107B7000142804D10120DD60087003201870012052
:107B800070BD70B503F0070200255B4C5B4B012A0A
:107B900002D0022A3FD03CE005201870DD6002F0E0
:107BA0006DFF41F6E8710144B0F53C3F2BD8CA782F
:107BB000086862F31F60534A904224D12268087C0F
:107BC00010702268487C50702268887C9070206811
:107BD000CA7CC27020680A7A02712268487A5071A1
:107BE0002268887A90712268C87AD0712268087DEC
:107BF00010722268487D50722268887D9072C87D1C
:107C00002168C87205E0002021680D54401C0C2832
:107C1000FAD3002070BD1A78052A13D1DA680C2A2D
:107C200028BF104607D2D4F800C01CF802C080F864
:107C300000C0501CD8600C2804D10120DD60087001
:107C400003201870012070BD70B503F007020025F5
:107C5000294C2A4E012A02D0022A36D033E004F001
:107C6000D4FD40B3D0E906212368C0681A70D4F867
:107C700000C0130A8CF80130D4F800C0130C120EA7
:107C80008CF802302368DA702268117123680A0ABE
:107C90005A7123680A0C090E9A712268D171216801
:107CA00008722268010A51722268010C9172010E59
:107CB0002068C17204E021680D54401C0C28FAD3DE
:107CC00005203070F560002070BD3278052A10D193
:107CD000F2680C2A28BF104604D223689B5C03700C
:107CE000501CF0600C2804D10120F56008700320BE
:107CF0003070012070BD0000E41B020020850010E0
:107D00004886001034CD12AB70B503F00702002492
:107D1000F94DFA4B012A02D0022A3ED03BE0052061
:107D200018700026DC6002F0A9FE00F50051B0F5E5
:107D30003C3F98BF11F0030F27D1F14A08689042E9
:107D400004BF0022104620D151F82030401C1A44B4
:107D50000728F9D302B1C6B128680A7C02702A68E4
:107D6000487C50702A68887C90702A68C87CD070E3
:107D70002A68087D10712A68487D50712A68887DBC
:107D80009071C87D2968C87105E0002029680C54ED
:107D9000401C0828FAD3002070BD1A78052A13D198
:107DA000DA68082A28BF104607D2D5F800C01CF8A8
:107DB00002C080F800C0501CD860082804D10120FF
:107DC000DC60087003201870012070BD2DE9F041BF
:107DD00003F0070C0027C94E4FF00508BCF1010F56
:107DE0000DD013F0070F0FD03246BCF1020F1278FE
:107DF00010D0BCF1040F08BF062A26D058E086F840
:107E000000807770F76053E07270BE4830630620E0
:107E100030704DE0052A15D1F268042A28BF1046BB
:107E200009D2C2F10303D6F830C0DB002CFA03F309
:107E30000370501CF060042804D10120F760087022
:107E4000032030700120BDE8F08170780125002406
:107E500010F0010F11D002F011FEB0F53C3F23D815
:107E60006A030021B1EB900F07D252F8043B491C82
:107E70001C44B1EB900FF8D3B5B1707810F0020F3D
:107E80000ED004F0C2FC78B182680021B1EB920FF1
:107E900006D250F8043B491C1C44B1EB920FF8D3B6
:107EA000002D18BF346300D13763777086F80080E7
:107EB0000020BDE8F081F0B503F0070C00268E4DE0
:107EC0008E4C83B0BCF1010F0ED013F0070F1DD004
:107ED000224603271278BCF1020F26D0BCF1040F12
:107EE00008BF062A36D03CE002AA01A9684603F082
:107EF00054F90520207029680198087029680098B5
:107F00004870296802988870E6602AE0E0680328D3
:107F100003D229680A54401CE060022821D30621BC
:107F20002170032808BFE6601BE0052A0FD1E26834
:107F3000032A28BF104604D22B689B5C0370501C98
:107F4000E060032803D10120E6600870277003B0C9
:107F50000120F0BD286882780178407803F010F99C
:107F6000277003B00020F0BD08B503F0070001281A
:107F70000AD104F0EBFB38B101208DF80000024675
:107F800069460D2002F0ACFD002008BD08B503F0E5
:107F9000070001280AD104F0D9FB38B100208DF880
:107FA0000000012269460D2002F09AFD002008BD64
:107FB00008B503F00700012809D104F0C7FB30B170
:107FC00003208DF800000122694602F089FD00209F
:107FD00008BD0020704708B503F0070001280AD14A
:107FE00004F0B4FB38B10B208DF800000122694683
:107FF000032002F075FD002008BD1FB513F0070F28
:108000000ED104F0A3FB58B19DF80800F0280AD067
:1080100004F09CFB20B1012202A9092002F060FDBE
:1080200004B0002010BDFEF727FAF9E700207047E2
:1080300070B503F00700304C304D012808D013F024
:10804000070F12D0042804BF2878062816D01FE096
:108050000020E860216808702168487021688870F5
:108060002168C8700520287012E0E86804280FD243
:1080700021680A54401CE860062008E004F066FB12
:1080800030B104221046216802F02AFD0320287036
:10809000002070BD10B503F00700012804D103F0E3
:1080A00083FE164900200871002010BD10B503F0B2
:1080B000070C124CBCF1010F06D013F0070F09D0CA
:1080C000BCF1020F20D015E00020E06007F093FA29
:1080D000E0610FE0E068002804BF1002E06106D014
:1080E000012804D1E0691043E06107F083FAE068F9
:1080F000401CE060002010BDE41B02002085001041
:1081000054464953EFBEADDEE26812B1012A04D0F5
:1081100007E0A18B090A017003E0237F03700120AF
:108120000870501CE0600120E5E710B503F0070C73
:10813000FD4CBCF1010F06D013F0070F09D0BCF1C4
:10814000020F18D015E00020E06007F057FAE06158
:108150000FE0E068002804BF1002E06106D00128AB
:1081600004D1E0691043E06107F04BFAE068401C7D
:10817000E060002010BDE26812B1012A04D007E0DF
:10818000A18B090A017003E0237F037001200870AE
:10819000501CE060012010BD70B503F0070CE24DEB
:1081A0000E460446BCF1010F06D013F0070F07D0AE
:1081B000BCF1020F18D015E00020E860286111E042
:1081C000E868002804BF1002E86108D0012806D141
:1081D000E869104381B2E861E8880FF0E3F9E868E4
:1081E000401CE860002070BD286902280ED2E88893
:1081F0000FF0DCF92B6982B2002B04BF100A20704B
:1082000004D0012B02D12270012030702869401C5B
:108210002861012070BD10B403F0070CC24CBCF102
:10822000010F08BF00200BD013F0070F03D0BCF1E3
:10823000020F09D005E0E068002808BFE280401C7A
:10824000E06010BC00207047E2681AB9A37903709F
:1082500001200870501CE06010BC012070472DE91F
:10826000F047064603F00700AF4F8946012808BFD4
:10827000002037D0DFF8B482AD4D13F0070F02D0E5
:10828000022833D02FE0F868002808BF7A7027D082
:10829000012804BF1002F86122D0022820D1F86919
:1082A0001043F8617E7884B204F050FAC0B1062E13
:1082B00016D2DFE806F00306090C1013A8F80E40EA
:1082C0000EE0A8F80C400BE02868848308E02868DA
:1082D000A0F8004104E02868848501E02868C4858E
:1082E000F868401CF8600020BDE8F0873869022873
:1082F0002AD297F801A0002404F028FAC8B1BAF1F4
:10830000060F16D2DFE80AF00306090C1013B8F8BE
:108310000E400EE0B8F80C400BE02868848B08E0B3
:108320002868B0F8004104E02868848D01E02868DE
:10833000C48D3869002804BF200A307004D0012899
:1083400002D1347089F800003869401C386101207E
:10835000BDE8F0872DE9F0411C4617460E4605465C
:1083600004F0F4F968B114F0070F04D004F007002A
:10837000022809D005E0002F14BF012000200BF0D7
:10838000EDFA0020BDE8F081684890F86C00C00864
:10839000287001203070BDE8F0812DE9F0411C46C5
:1083A00015460F46064613F0070F08D104F0CEF924
:1083B00028B1022D3CBF284609F0CDF803E004F0B7
:1083C0000700022802D00020BDE8F08109F0BCF8C7
:1083D000307001203870BDE8F08170B503F00702FD
:1083E0000026544C504D012A02D0022A15D012E02A
:1083F00008F090F821680870FDF736FD2168487094
:1084000004F086F821688870FDF734FD2168C87093
:1084100005202870EE60002070BD2A78052A10D152
:10842000EA68042A28BF104604D223689B5C0370C4
:10843000501CE860042804D10120EE60087003207D
:108440002870012070BD70B503F00702394C00257B
:10845000354E012A02D0022A54D051E0FDF7E6FF42
:10846000002836D04169FF292CBFFF21C9B22268FC
:1084700011708169FF2934BFC9B2FF212268517090
:10848000C169FF2934BFC9B2FF21226891702268F7
:10849000017CD170226890F820101171018C226843
:1084A000090A5171016A2268090C9171016A2268F6
:1084B000090ED171016BFF2934BFC9B2FF212268B7
:1084C0001172406BFF2834BFC0B2FF202168487290
:1084D00015E0206805702068457020688570216867
:1084E0005020C8702168FF200871216848712168F8
:1084F00088712168C8712068057220684572F5602E
:10850000002070BDF2680A2A28BF104604D22368F2
:108510009B5C0370501CF0600A2802D10120F560BA
:108520000870012070BD000020850010F82F011098
:1085300048860010E41B020003F00702FC4B4FF0DA
:10854000000C012A08BFC3F80CC001D0022A01D0D8
:1085500000207047DA68022A3DBF80F800C0501C36
:10856000D8601046022803D10120C3F80CC008705F
:10857000012070472DE9F047064603F00700EC4F55
:108580008A464FF00008012808BFC7F80C8001D0C8
:10859000022802D00020BDE8F087F868A0BB0024C4
:1085A000254602F06BFA014600F5005018384FF4EA
:1085B00000524FF04009B1F53C3F20D890F803C07D
:1085C00003686CF31F63DFF86CC3634517D1091FA1
:1085D000B4EB910F06D252F8043B641C5D40B4EB3F
:1085E000910FF8D3C17D406961F31F60A84206D1A5
:1085F00004F0ACF8012804BF8020307001D086F868
:108600000090F868401CF860012803D1C7F80C807E
:108610008AF800000120BDE8F0872DE9F04103F061
:1086200007020026C44CC24D012A02D0022A56D0AD
:1086300052E0FBF7A9FA0520287004F087F800281B
:1086400049D0BE4F386804F0ADF9002843D00EF091
:108650008CFF80460EF08DFF39680A7E12F0040F01
:1086600011D0C98A2268090A117039682268897D87
:10867000517039682268898A090A917039682268BC
:10868000097DD17010E0898A2268090A1170396861
:108690002268097D517039682268C98A090A917077
:1086A00039682268897DD17022684FEA18211171DA
:1086B000216881F805802268010A91712168C871DA
:1086C00038682268817C11722268017C5172008BAB
:1086D0002168000A8872EE600020BDE8F0812A78E7
:1086E000052A10D1EA680B2A28BF104604D2236855
:1086F0009B5C0370501CE8600B2804D10120EE60E5
:108700000870032028700120BDE8F0812DE9F047B2
:1087100003F007020026884D854B012A02D0022A69
:108720005DD059E0052018700024DE6002F0A6F943
:1087300000F50053B0F53C3F98BF13F0030F45D14F
:108740007F4A1968914204BF0022114608D153F8AC
:1087500021C0491C62440729F9D3002A08BF01241B
:108760009F7C93F8138084B341F6E8710144B0F51F
:108770003C3F07D8CA78086862F31F606D4A904290
:1087800008BF012491F8129091F813A0002C08BFA3
:10879000002014D004F039F82968806981F800902D
:1087A000296881F801A02A68010C000E91702968DF
:1087B000C87028680771286880F805800CE029686F
:1087C0000E54401C0628FAD306E0FFE70020296873
:1087D0000E54401C0628FAD30020BDE8F0871A7812
:1087E000052A13D1DA68072A28BF104607D2D5F820
:1087F00000C01CF802C080F800C0501CD8600728D8
:1088000004D10120DE600870032018700120BDE84B
:10881000F08770B5054603F007000C46022829D101
:1088200003F094FF30B3454800220068037EC3F391
:1088300080008000C3F3400100EB410003F0010120
:108840000844082812D2DFE800F00406080A0C0EDB
:10885000111004220AE0052208E0062206E00722A1
:1088600004E0022202E0032200E001222A7001203B
:10887000207070BD002070BD10B503F0070C2C4CAB
:10888000BCF1010F06D013F0070F0AD0BCF1020FA4
:108890001AD017E00020E06020610EF0E6FEE061F3
:1088A00010E0E068002804BF1002E06107D0012852
:1088B00005D1E0691043E06180B20EF0D3FEE068BC
:1088C000401CE060002010BD2269022A0BD212B1C8
:1088D000012A04D007E0A18B090A017003E0237F7D
:1088E000037001200870501C2061012010BD70B57C
:1088F00003F0070100260E4D0446012908BF6E63F0
:1089000001D0022901D0002070BD686B002804BF8F
:108910000C4813F025FF696B082928BF267002D286
:108920000848405C2070481C6863012070BD00004E
:108930002085001034CD12ABE41B020048860010E5
:1089400054464953588500102DE9F04103F00701C2
:108950000026FA4D0746012908BF6E6301D002299F
:1089600002D00020BDE8F08195F8340000F0070443
:108970002879204304D1F24813F0F2FE0120287137
:10898000052C28BF2E71EE48005D3870686B401CC6
:1089900068630120BDE8F08170B5044603F007006C
:1089A0000D4602281CBF002070BD13F0DEFE2070B3
:1089B0000120287070BD2DE9F04103F00702002668
:1089C000E04DDE4C012A02D0022A1AD016E0052022
:1089D0002070002211461046E66002F0DEFB4FF6E2
:1089E000FF7101EA40006061FDF73EFA032803BF12
:1089F00028782028D44802F0E3FBA0620020BDE8DC
:108A0000F0812278052A1DD1D4F814C0E2686245AD
:108A100028BF104607D212F0010F1CBF6378037005
:108A200013D0501CE06060450CD10120E660087056
:108A300003202070FDF718FA032806BF28782028A5
:108A400002F0CBFB0120BDE8F081A76A22F0010310
:108A5000FB5A1F0A07706370E3E770B503F0070263
:108A60000025B64C012A02D0022A11D00EE0B748E8
:108A700005220068B0F91210B0F910002270084405
:108A80004000E560606102F028FEA062002070BD39
:108A90002278052A17D1D4F814C0E268624528BFAD
:108AA000104607D212F0010F1CBF637803700CD080
:108AB000501CE060604506D10120E560087003208D
:108AC000207002F018FE012070BDA66A22F001039A
:108AD000F35A1E0A06706370EAE7002070472DE91A
:108AE000F0419A4A03F00703944E12684FF00008D1
:108AF000012B02D0022B10D00CE005203070C6F8FC
:108B00000C80108A518A400848434000706102F08E
:108B100057FBB0620020BDE8F0813378052B17D1F8
:108B20007469F368A34228BF184607D213F0010FF7
:108B30001CBF727802700ED0581CF060A04207D1A2
:108B40000120C6F80C8008700320307002F045FB4D
:108B50000120BDE8F081B2F812C05F08B7FBFCF558
:108B60000CFB1577128AACEB070C0CFB02F2D6F863
:108B700028C0521B0CEB420232F8022C4FEA122C96
:108B800080F800C07270D7E72DE9F0416F4A03F01A
:108B900007036A4E12684FF00008012B02D0022B27
:108BA00010D00CE005203070C6F80C80108A518A75
:108BB000400848434000706102F002FBB0620020B0
:108BC000BDE8F0813378052B17D17469F368A342AF
:108BD00028BF184607D213F0010F1CBF727802702D
:108BE0000ED0581CF060A04207D10120C6F80C80BE
:108BF00008700320307002F0F0FA0120BDE8F08127
:108C0000504D9C462D78282D03D1558A178A05FB97
:108C100007CC4FEA5C07B2F812C0128AB7FBFCF52A
:108C20000CFB1577ACEB070C0CFB02F2D6F828C056
:108C3000521B0CEB420232F8022C4FEA122C80F845
:108C400000C07270CDE770B503F0070200253B4C01
:108C5000012A02D0022A14D011E03C480522006803
:108C6000B0F91210B0F91000227008444000E5601D
:108C7000606102F032FD3649A06202F042FF00203E
:108C800070BD2278052A17D1D4F814C0E268624575
:108C900028BF104607D212F0010F1CBF6378037083
:108CA0000CD0501CE060604506D10120E5600870E2
:108CB0000320207002F01FFD012070BD244E22F021
:108CC0000103F35A1E0A06706370EAE770B50D4699
:108CD000044613F0070F04D003F00700022805D064
:108CE00002E01046FDF7BAF8002070BDFDF7B9F8B4
:108CF00020700120287070BD70B503F007020325B5
:108D00000E4C012A02D0022A24D014E003F0D9FF2D
:108D10000646FDF7A6F80146304603F0E3FF206261
:108D200000281ABF052020702570002003F0CCFF1A
:108D300060620020E060002070BD0000208500100F
:108D4000588500106D850010182801104886001005
:108D500008AA00102278052A0BD1236AE2689B5CDE
:108D60000370501CE060626A904202D301200870D8
:108D700025700120E0E700207047002070477FB594
:108D80001C460E46054613F0070F08D103F0DEFC23
:108D900028B1012202A9252001F0A2FE03E004F07F
:108DA0000700022802D004B0002070BD02F0D1FA02
:108DB00028700120307004B070BD2DE9F04103F03F
:108DC00007020027FE4E88460546012A02D0022AE5
:108DD0000BD007E0052030700A20F760706102F0C8
:108DE000EFF9B0620020BDE8F0813078052819D194
:108DF000F2687069824228BF104608D212F0010F53
:108E00001CBF7078287010D0F068401CF060716949
:108E1000884207D10120F76088F8000003203070F5
:108E200002F0DBF90120BDE8F081002402F091FAA4
:108E3000012804D1F068B16A20F001000C5A200A20
:108E400028707470E0E770B50D46044613F0070F04
:108E500004D003F00700022805D002E0104603F01A
:108E60002DFF002070BD03F02CFF20700120287022
:108E700070BD7FB51C460E46054613F0070F08D19E
:108E800003F064FC28B1012202A91F2001F028FE92
:108E900003E004F00700022802D004B0002070BDF7
:108EA00007F07FFC28700120307004B070BD7FB5E2
:108EB0001C460E46054613F0070F08D103F046FC8A
:108EC00028B1012202A9202001F00AFE03E004F0EB
:108ED0000700022802D004B0002070BD07F067FC34
:108EE00028700120307004B070BD7FB51C460E465E
:108EF000054613F0070F08D103F028FC28B1012222
:108F000002A91B2001F0ECFD03E004F00700022899
:108F100002D004B0002070BDFDF7BCF8287001201D
:108F2000307004B070BD7FB51C460E46054613F088
:108F3000070F08D103F00AFC28B1012202A90C2076
:108F400001F0CEFD03E004F00700022802D004B0D7
:108F5000002070BD07F0DEFA28700120307004B0E8
:108F600070BD7FB51C460E46054613F0070F08D1AD
:108F700003F0ECFB28B1012202A90F2001F0B0FDA3
:108F800003E004F00700022802D004B0002070BD06
:108F90000DF041FF00F00F0040F01000287001209C
:108FA000307004B070BD2DE9F04103F0070C844D22
:108FB0000E460746BCF1010F07D0824C13F0070F95
:108FC00007D0BCF1020F1BD017E00020E860286139
:108FD00013E0E86804283CBF21680A54032809D13B
:108FE000206821680068C97800BA20F0FF000843B3
:108FF000FCF70EFAE868401CE8600020BDE8F0814C
:10900000286970B9FCF709FA216820F07E42100E39
:1090100008702168100C48702168100A8870206858
:10902000C2702A69042A06D22068032A805C38703C
:1090300004BF01203070501C28610120BDE8F08180
:109040007FB51C460D46064613F0070F08D103F006
:109050007DFB28B1012202A9102001F041FD03E0AF
:1090600004F00700022802D004B0002070BD0DF00B
:10907000D6FE00F00F040DF0CEFE64F31F1030702A
:109080000120287004B070BD70B54D4D144613F02A
:10909000070F04D003F00702022A06D003E01046AF
:1090A000F7F76AF9EC62002070BD95F82C20027089
:1090B0000120087070BD10B503F00702404C012A72
:1090C00002D0022A0DD00AE003F0C8FE002120627F
:1090D00000281ABF4FF4056060626162E160002001
:1090E00010BD636AE2689A4228BF104607D2D4F8DE
:1090F00020C01CF802C080F800C0501CE0609842FC
:1091000004BF01200870012010BD10B413F0070F38
:109110004FF0402C04D003F00702022A13D00FE0D6
:10912000012A04BFDCF8140040F0010006D0002A38
:1091300004BFDCF8140020F0010001D1CCF81400C9
:1091400010BC00207047DCF81430002213F0010F2F
:1091500018BF01221C4BD3F83CC01C4B1B68B3F852
:10916000DC30C3F30334012303FA04F41CEA040FD4
:1091700018BF42F0020202700B7010BC0120704751
:1091800070B514460E46054613F0070F04D003F0E1
:10919000070002281CD010E0002C14BF0120002082
:1091A00002F0E0FD4CB14FF04020016B21F4405142
:1091B00041F4BE0141F020410163002070BD000078
:1091C00020850010E41B02000010004048860010BB
:1091D00002F0CFFD002814BF012200222A700120D6
:1091E0003070EBE72DE9F04103F0070CFF4C0F4620
:1091F0008046BCF1010F12D0FD4E13F0070F4FF067
:10920000030510D02046BCF1020F027822D0BCF139
:10921000040F02BFE0680128062A2FD032E00520A3
:109220002070002014E0E06810B1012804D00DE0A7
:1092300062700620207009E0607800EA0201316364
:1092400020EA02017163F9F7FDFF2570E068401C18
:10925000E06017E0E068012808BF062A03D16078C3
:10926000F9F7F5FF2570F06B88F8000001203870E1
:10927000E068401CE0600120BDE8F0816078F9F70B
:10928000E6FF25700020BDE8F08170B5044603F0CC
:1092900007000D4602281CBF002070BDFCF7DCFE55
:1092A000002814BF0122002222700120287070BD06
:1092B00070B50D46044613F0070F04D003F0070005
:1092C000022805D002E0104607F04EF8002070BDDD
:1092D00007F04DF820700120287070BD70B50D4664
:1092E000044613F0070F04D003F00700022805D04E
:1092F00002E01046F7F70CFF002070BDF7F70BFFF8
:1093000020700120287070BD70B503F00702DFF8EF
:10931000DCC20C460546012A08BF05200DD013F01B
:10932000070F08BF062008D0022A09D0042A04BF6C
:109330009CF80000062809D00EE08CF800000BE035
:10934000FCF7AEFE28700120207070BD03208CF861
:1093500000000120FCF7A7FE002070BD70B503F0EF
:109360000702A24D0E460446012A04BF0020E86011
:1093700001D0022A01D0002070BD0FF085F8EA6804
:10938000002A04BF000A207004D0012A02D12070F4
:1093900001203070501CE860012070BD03F007020E
:1093A00010B4924B012A04BF0020D86001D0022AD9
:1093B00002D010BC00207047DA68022A0CD24FF0AD
:1093C000010C002A08BF80F800C005D0012A03D193
:1093D0004024047081F800C0501CD86010BC0120EB
:1093E000704770B5044603F007000D46022807D009
:1093F00013F0070F04BF1046FCF72AFD002070BDD4
:10940000FCF729FD20700120287070BD70B504465E
:1094100003F00700754D0E46012804BF0020E860E8
:1094200014D013F0070F02D0022811D00EE0E86824
:10943000704904283CBF0B681A54401CE86004289B
:1094400004D104220968132001F04AFB002070BDFA
:109450000CF0F6F9EA68002A04BF000E20700FD065
:10946000012A08BF000C06D0022A08BF000A02D059
:10947000032A02D004E0207002E020700120307046
:10948000501CE860012070BD70B503F0070C574D0B
:109490000E460446BCF1010F04BF0020E86015D061
:1094A00013F0070F03D0BCF1020F11D00EE0E868F3
:1094B000504902283CBF0B681A54401CE86002283F
:1094C00004D102220968142001F00AFB002070BDBB
:1094D0000CF082F9EA68002A04BF000A207004D068
:1094E000012A02D1207001203070501CE860012058
:1094F00070BD70B5044603F007003C4D0E460128D0
:1095000004BF0020E86014D013F0070F02D0022837
:1095100011D00EE0E868374904283CBF0B681A54A4
:10952000401CE860042804D104220968152001F0D9
:10953000D7FA002070BD0CF0BEF9EA68002A04BF1B
:10954000000E20700FD0012A08BF000C06D0022A9E
:1095500008BF000A02D0032A02D004E0207002E013
:10956000207001203070501CE860012070BD2DE992
:10957000F041044603F0070000251C4E0F46012869
:1095800008BFF56042D013F0070F02D0022840D088
:109590003CE0F068174C002804BF21680A7021687D
:1095A0000978012901D039B11FE0002818BF062829
:1095B0003CBF21680A5418E00CF098F921680009B2
:1095C00048700CF087F9C0F303270CF08FF921687D
:1095D00047EA001088700CF07DF92168C870206897
:1095E0000571206845710520F06005E020850010B8
:1095F00000100040E41B0200F068401CF0600628E8
:1096000004D106221620216801F06AFA0020BDE884
:10961000F0810CF083F905460CF074F980460CF0EB
:1096200077F9F268002A04BF280E207018D0012AAA
:1096300008BF280C0FD0022A08BF280A0BD0032A23
:1096400008BF25700CD0042A08BF84F8008007D01A
:10965000052A02D004E0207002E02070012038705A
:10966000501CF0600120BDE8F08110B503F0070246
:10967000FE4C012A02D0022A27D024E003F0EEFBA0
:109680000023002804BF236263621BD000F1500155
:1096900021624168B1F5887F90F820100CD390F8D2
:1096A000212001EB020C01FB02C190F8222090F86E
:1096B00023001044084404E090F822000A1801FB3B
:1096C00000206062E360002010BD636AE2689A4295
:1096D00028BF104607D2D4F820C01CF802C080F87A
:1096E00000C0501CE060984204BF012008700120B7
:1096F00010BD03F00702012A02D0022A05D002E0C1
:10970000DA490020C86000207047012202700A7008
:109710001046704710B513F0070F04D003F007028E
:10972000022A05D002E0104601F064FD002010BDC1
:10973000CF4A127802700120087010BD10B513F0E6
:10974000070F04D003F00702022A05D002E01046FA
:1097500001F0DEFF002010BDC64A12780270012021
:10976000087010BD002070471FB513F0070F07D118
:1097700002F0ECFF20B1012202A90B2001F0B0F9A8
:1097800004B0002010BD70B503F00700B74C1546BB
:10979000012804BF0020E06024D013F0070F21D17E
:1097A00002F0D4FFF0B1E068B34E03283CBF31684B
:1097B0000D54401CE060032814D1F8F7FAFB306820
:1097C000B0F8010045BAF8F72FFB040018BFF8F70E
:1097D00085FD306829460078F7F749FF002C18BF4F
:1097E000F8F77FFD002070BD70B503F007009F4CB7
:1097F0001646012804BF0020E06029D013F0070FAF
:1098000026D102F0A3FF18B3E0689B4D02283CBFAD
:1098100029680E54401CE060022819D1F8F7C9FBF2
:10982000F8F702FB040018BFF8F758FD2868007825
:1098300080B129684978F7F7AEFF28684178007849
:1098400040F01000F7F7A7FF002C18BFF8F749FD0C
:10985000002070BD286841780020F3E770B50D4600
:10986000044613F0070F04D003F00700022805D0C8
:1098700002E01046F8F742FD002070BDF8F741FD08
:1098800020700120287070BD7FB51C460E4605462D
:1098900013F0070F08D102F059FF28B1012202A9E5
:1098A000172001F01DF903E004F00700022802D0A0
:1098B00004B0002070BD06F008FE002814BF01228D
:1098C00000222A700120307004B070BD7FB51C46A4
:1098D0000E46054613F0070F08D102F037FF28B1F6
:1098E000012202A9182001F0FBF803E004F00700B0
:1098F000022802D004B0002070BD06F0D3FD28700D
:109900000120307004B070BD2DE9F04103F0070C68
:10991000564C0E460746BCF1010F07D0564D13F0CA
:10992000070F07D0BCF1020F19D015E00020E0604E
:10993000206111E0E06803283CBF29680A54401CFC
:10994000E060032808D12868B0F8010040BA01B2ED
:1099500028680078FDF7C6FE0020BDE8F081226986
:10996000022A12D242B928680078FDF7C4FE2A689C
:10997000010A517029688870286822691044012AF8
:109980004078387004BF012030702069401C20618D
:109990000120BDE8F08170B503F00700334C154697
:1099A000012804BF0020E06017D013F0070F14D186
:1099B00002F0CCFE88B1E0682F4B03283CBF196849
:1099C0000D54401CE060032807D11868B0F801006E
:1099D00041BA18680078F8F7CBFF002070BD10B5C9
:1099E00003F00702214C012A02D0022A07D004E02A
:1099F0000020E060F9F7B5FFE061002010BDE268EB
:109A0000042A07D2C2F10303D4F81CC0DB002CFAED
:109A100003F30370501CE060042804BF01200870A9
:109A2000012010BD10B503F00700012807D102F096
:109A30008DFE20B1002211461C2001F051F80020BB
:109A400010BD2DE9F04103F00705084E1746884682
:109A50000446012D04BF0020F06024D013F0070F4E
:109A60001FD102F073FEE0B1034B07E02085001028
:109A70006D85001073850010E41B0200F068032858
:109A80003CBF19680F54401CF06003280BD11868C4
:109A900090F9022090F9011090F90000FBF7E8FA24
:109AA00001E0022D02D00020BDE8F081F06830B165
:109AB000012809D002280CD003280FD015E014206B
:109AC000FBF79FF9207010E01520FBF79AF9207042
:109AD0000BE01620FBF795F9207006E01720FBF746
:109AE00090F92070012088F80000F068401CF060B8
:109AF0000120BDE8F08170B50D46044603F0070073
:109B00000021FD4E012814BF13F0070FF16001D0B2
:109B1000022801D0002070BDF06840B101280BD0B0
:109B200002280ED0032811D0042814D019E00120F7
:109B3000FBF767F9207014E00220FBF762F9207050
:109B40000FE00320FBF75DF920700AE00420FBF72B
:109B500058F9207005E00520FBF753F9207001202B
:109B60002870F068401CF060012070BD70B503F0F3
:109B7000070C0026E14CE04DBCF1010F06D013F0BC
:109B8000070F0CD0BCF1020F1FD01CE006F0DEFD69
:109B9000EE60216808702168000A487013E0E868E8
:109BA000022803D221680A54401CE86002280AD126
:109BB000EE602068007810F0010F04D00222192016
:109BC000216800F08DFF002070BDEA68022A28BFDE
:109BD000104604D223689B5C0370501CE860022886
:109BE00004D10120EE60087003202870012070BDB0
:109BF0007FB51C460E46054613F0070F08D102F04C
:109C0000A5FD28B1012202A9232000F069FF03E08D
:109C100004F00700022802D004B0002070BD0DF04F
:109C200013FD28700120307004B070BD7FB51C4654
:109C30000E46054613F0070F08D102F087FD28B144
:109C4000012202A91E2000F04BFF03E004F00700F0
:109C5000022802D004B0002070BD0DF000FD287075
:109C60000120307004B070BD7FB51C460E4605461D
:109C700013F0070F08D102F069FD28B1012202A9F3
:109C8000222000F02DFF03E004F00700022802D09C
:109C900004B0002070BD10F099FC287001203070D5
:109CA00004B070BD7FB51C460E46054613F0070F85
:109CB0000ED102F04BFD58B19DF80800002818BFE6
:109CC0000DF0D6FC012202A91D2000F009FF03E0DF
:109CD00004F00700022802D004B0002070BD0DF08F
:109CE000CAFC28700120307004B070BD2DE9FF411E
:109CF000814E1C460F46054613F0070F1CD102F09B
:109D000025FDC8B19DF80800002818BF012802D021
:109D1000022807D014E0F070012202A9082000F008
:109D2000DFFE0DE0F07004208DF80800012202A98A
:109D3000082000F0D5FE03E004F00700022803D05D
:109D400004B00020BDE8F081F07828700120387060
:109D500004B0BDE8F0817FB51C460D46064613F001
:109D6000070F08D102F0F2FC28B1012202A9082055
:109D700000F0B6FE03E004F00700022802D004B0B1
:109D8000002070BDFCF770F8801E052813D2DFE8B4
:109D900000F003070E05100000240DE001240BE085
:109DA000022405F044FD042808BF052404E0032430
:109DB00002E0042400E0FF2434700120287004B085
:109DC00070BD2DE9F0411C4617460E46054613F0BE
:109DD000070F0BD102F0BAFC40B1384606F0BEFACC
:109DE00000221146012000F07BFE03E004F0070092
:109DF000022802D00020BDE8F08106F0B2FA2870F7
:109E000001203070BDE8F08110B5104613F0070F47
:109E100008BF06F06DFB002010BD10B5104613F012
:109E2000070F08BF06F06BFB002010BD70B504469D
:109E300003F007000D4602281CBF002070BD06F08D
:109E400066FB20700120287070BD03F0070230B45B
:109E5000294B4FF0000C012A05D0022A04BF1A78C2
:109E6000022A0BD01EE0022018702548C3F80CC04F
:109E70006FF07F410068081AD86113E0DA68042A9D
:109E800028BF104606D2DD69D40025FA04F4047018
:109E9000501CD860042805D10120C3F80CC00870FC
:109EA0000320187030BC0120704713F0070F04BF67
:109EB000144802700020704710B503F007000E49E7
:109EC000012804BF0020C86013D013F0070F10D181
:109ED000C8680A4B04283CBFD3F800C00CF8002027
:109EE000401CC860042804D104221220196800F024
:109EF000F7FD002010BD000020850010E41B0200CB
:109F00008C840010278400102DE9F047164603F0DA
:109F100007020024F74F012A04BFFC603C6164D0B3
:109F2000DFF8D48313F0070F07D0022A33D0042AB6
:109F300004BF387806284FD058E0FD68002D08BFD0
:109F40003E6225D0012D06D0D7F81490AC1E4C45AA
:109F500016D284B908E0701C7861396A0844B0F5FB
:109F6000007F88BF7C6113E04FF400724FF43E31F4
:109F7000E24812F09BFBE249386A096820440E541B
:109F8000601C484504D1DD48C0F8FC8106203870CB
:109F9000681CF8602AE0FF2202707B69CBB1D7F819
:109FA00020C03A699444BCF5007F10D2D54D2D688D
:109FB000454518BF047005D10CF53C3C9CF800C821
:109FC00080F800C0501C984204BF01200870501C4B
:109FD00038610120BDE8F0874FF43E30F8F7C6FF46
:109FE000C6494FF43E30F9F763F83C700020BDE8F5
:109FF000F0872DE9F0478C4603F007010024BD4FA0
:10A000001646012904BFFC603C6162D013F0070FC3
:10A01000BD4BDFF8F88207D0022932D0042904BFF3
:10A02000387806284DD055E0FD68002D08BF3E6207
:10A0300024D0012D06D0D7F81490AC1E4C4515D273
:10A040007CB908E0701C7861396A0844B0F5007F7B
:10A0500088BF7C6112E04FF400721946A74812F0E5
:10A0600025FBA749386A096820440E54601C4845FE
:10A0700004D1A248C0F8FC8106203870681CF86042
:10A0800028E0FF2101707B69C3B13A6A39690A444B
:10A09000B2F5007F10D29E4D2D68454518BF047063
:10A0A00004D102F5383292F8002E0270481C984212
:10A0B00004BF01208CF80000481C38610120BDE875
:10A0C000F0871D461846F8F751FF8C492846F8F7E7
:10A0D000EFFF3C700020BDE8F08770B503F007008B
:10A0E000844C1546012804BF0020E06014D013F012
:10A0F000070F11D102F02AFB70B1E06880490228F5
:10A100003CBF0A681554401CE060022804D10222BA
:10A110000968052000F0E4FC002070BD2DE9F04145
:10A12000054603F00700764C724E0F4601280AD010
:10A1300013F0070F14D002281BD0042804BF307876
:10A14000062834D03FE00020F060216808702168C4
:10A150004870216888702168C8700520307032E02E
:10A16000F06804282FD221680A54401CF0600620B1
:10A1700028E0F06860B906F0E7F821680870226806
:10A18000010A51702268010C000E91702168C8709C
:10A19000F06804283ABF2168095CFF21297024BFB8
:10A1A00001213970401CF0600120BDE8F08102F00F
:10A1B000CDFA40B12068C178006861F31F6006F0F5
:10A1C000BEF8032030700020BDE8F0810020704709
:10A1D0007FB51C460E46054613F0070F08D102F066
:10A1E000B5FA28B1012202A9262000F079FC03E08B
:10A1F00004F00700022802D004B0002070BD06F071
:10A20000ACF928700120307004B070BD03F0070075
:10A210003849012808BF002009D013F0070F07D1E3
:10A22000C86818B93B4B1B681A448A61401CC86057
:10A23000002070472DE9F04103F007012D4C164630
:10A240000546012907D0334F13F0070F386806D0B1
:10A25000022919D015E00020E060206111E0A56915
:10A2600005F0F4FA01280CD1A0693968884224BFAE
:10A27000D031814205D9E068042838BF2E54401CF3
:10A28000E0600020BDE8F081A66905F0DFFA50B17A
:10A29000A26939688A4224BF01F1D000904284BF8C
:10A2A0002069305C00D8FF2028702069401C2061A4
:10A2B0000120BDE8F0817FB51C460E46054613F02F
:10A2C000070F08D102F042FA28B1012202A9112099
:10A2D00000F006FC03E004F00700022802D004B0FE
:10A2E000002070BD0FF0E5FF28700120307004B031
:10A2F00070BD000020850010554E564D08A8001076
:10A30000E41B0200FCF9020000EE0200324E564D42
:10A31000FCEF02006C8600100020704700207047A0
:10A3200070B50D46044613F0070F04D003F0070084
:10A33000022805D002E0104608F0F5FF002070BDAD
:10A3400008F0FDFF20700120287070BD10B503F0EB
:10A350000702FF4CFF4B4FF0000C012A02D0022AEB
:10A3600030D02DE0C3F80CC002F0F0F9002827D05F
:10A37000F94802F026FB18B3F8480068007E10F098
:10A38000040FF5480ED0C18A2268090A11702268AC
:10A39000817D5170818A2268090A91702168007D4F
:10A3A000C8700DE0818A2268090A11702268017D57
:10A3B0005170C18A2268090A91702168807DC87035
:10A3C000002010BDDA68042A28BF104604D2246891
:10A3D000A45C0470501CD860042803D10120C3F889
:10A3E0000CC00870012010BD70B503F00701D84DF6
:10A3F000D84C012902D0022914D011E0012001F02B
:10A40000C0FB0020E06001F0D1FB208129680870CA
:10A410002A68010A0028517004BF002001F0B1FB36
:10A42000002070BDE168022902D22A68525C0270E5
:10A43000481CE060012070BD2DE9F04103F00702E7
:10A440000026C44D0F460446012A02D0022A09D034
:10A4500005E005202870EE60288940006861002032
:10A46000BDE8F0812878052817D1EA68686982423A
:10A4700005D212F0010F1CBF6878207010D0E86878
:10A48000401CE8606969884207D10120EE6038709D
:10A4900003202870002001F074FB0120BDE8F0814A
:10A4A00001F09DFB010A21706870E8E71FB513F009
:10A4B000070F04D1012202A91A2000F011FB04B0F9
:10A4C000002010BD002070470020704703F00700F7
:10A4D000A049012806D013F0070F04BF087801280F
:10A4E00006D014E0012008700020C86088610DE0EB
:10A4F000C868042805D28B69401C42EA03228A619D
:10A50000C860042803D1032008708869086200200D
:10A51000704703F00700DFF83CC2012807D013F0B2
:10A52000070F04BF9CF80000022809D01EE002209B
:10A530008CF800000020CCF80C00CCF81C0015E0D2
:10A54000DCF80C00022808D2DCF81C10401C42EA9F
:10A550000121CCF81C10CCF80C00022806D1DCF844
:10A560001C00CCF8240003208CF800000020704769
:10A5700070B403F007020025764C012A02D0022AAB
:10A5800006D002E002202070E56070BC0020704719
:10A590002278022A1CD1D4F824C0E268624528BF80
:10A5A00010460ED212F0030F04D1236A53F8046B45
:10A5B000C4E90763237F0370E069000AE061501C6F
:10A5C000E060604504D10120E56008700320207040
:10A5D00070BC0120704770B503F0070000255D4C8A
:10A5E0000E46012806D013F0070F04BF207802287A
:10A5F00005D02BE002202070E560E56126E0616A6D
:10A60000E068884219D2E169090A41EA0262401C05
:10A61000E26110F0030FE0600FD1206AB0F5443F13
:10A6200028BF026006D2B0F5005F03D304224C4974
:10A63000F8F792FD206A001D2062616AE068884296
:10A6400004D10120E560307003202070002070BD2F
:10A6500070B503F0070C00253E4CBCF1010F08BF9C
:10A66000E5603AD013F0070F03D0BCF1020F36D0EB
:10A6700033E0052A08BF4FF43E302DD005DC16D25A
:10A68000DFE802F0171A1D2022003448202A006853
:10A6900008BFE43020D006DC102A1DD0112A08BFE4
:10A6A0002D4819D003E0302A11D0312A12D0A561EB
:10A6B00013E04FF400500FE04FF443300CE04FF440
:10A6C000203009E0274807E04FF4403004E001F073
:10A6D000D1FB01E00FF0CDF9A061002070BDE26870
:10A6E000042A07D2C2F10303D4F818C0DB002CFA05
:10A6F00003F30370501CE060042824BF012008709D
:10A70000012070BD70B403F0070C124DBCF1010FB5
:10A7100007D00F4C13F0070F07D0BCF1020F2ED05B
:10A720002AE00020E860286126E0E86805283CBFB0
:10A7300021680A5404281DD123682268A969D3F826
:10A74000013012781BBA23F0FF03D4F800C00BE0ED
:10A75000E41B020020850010F82F0110488600102D
:10A760003C85001000FE02009CF804C043EA0C0384
:10A7700041F82230401CE86070BC002070472B6913
:10A7800073B1042B07D22268032B1A44527802704B
:10A7900004BF01200870581C286170BC012070475C
:10A7A0002268D5F818C012785CF8222026684FEA93
:10A7B000126C86F801C026684FEA124C86F802C077
:10A7C00026684FEA122C86F803C0D4F800C08CF833
:10A7D0000420D8E710B503F00700012804D10022B7
:10A7E00011460E2000F07CF9002010BD2DE9F0414B
:10A7F00003F00704A94E174688460546012C04BFFE
:10A800000020F06017D013F0070F12D101F09EFF67
:10A8100078B1F068A24902283CBF0A681754401C6E
:10A82000F060022807D102220968072000F058F9D9
:10A8300001E0022C02D00020BDE8F081F26812B1E4
:10A84000012A04D009E0FBF70FFB287005E0FBF7B5
:10A8500011FB2870012088F80000F068401CF060AF
:10A860000120BDE8F08170B503F0070000258B4C96
:10A87000012808D013F0070F0BD0042804BF20785C
:10A88000062825D02DE0A561E5616570E56025709D
:10A8900027E0E068022807D2A16942EA0121A1610C
:10A8A00061781144617010E0042807D2E16942EA3E
:10A8B0000121E16161781144617006E0052804D24C
:10A8C00061788A4204BF06212170401CE06008E0E4
:10A8D000D4E9060101F02CFB002804BF0120A07080
:10A8E0002570002070BD10B56C4C13F0070F07D019
:10A8F00003F00700042804BF2078062822D02BE0AC
:10A90000E068022807D2A16942EA0121A1616178C9
:10A910001144617013E06349091808D2604909685D
:10A92000014401F8022C61781144617007E05E492E
:10A93000091804D261788A4204BF06212170401CA4
:10A94000E06009E05949A06901F014FB002804BF48
:10A950000120A07000202070002010BD03F0070C23
:10A96000BCF1010F00D0BEE74C490020886148705F
:10A97000C8600870704730B403F007050024DFF8A2
:10A980001CC1012D07D013F0070F0DD0022D3CD0B4
:10A99000042D54D06FE0CCF81840CCF81C40CCF813
:10A9A0000C408CF8004066E0DCF80C0002280BD26A
:10A9B000DCF8181042EA0121CCF818109CF80110BC
:10A9C00011448CF8011019E0042817D2DCF81C108F
:10A9D000032842EA0121CCF81C109CF801301A44EB
:10A9E0008CF801200AD106228CF80020DCF818200F
:10A9F000114304BF4FF4C471CCF81C102C49401C07
:10AA0000CCF83010CCF80C0035E0DCF80C20042A2F
:10AA100028BF10460AD2C2F10303DCF83050DB0035
:10AA200025FA03F30370501CCCF80C00042803D162
:10AA30000120CCF80C40087030BC012070479CF815
:10AA40000000062815D1DCF8180000224102DCF8CD
:10AA50001C0043021046B2EB930F06D251F8045B80
:10AA6000401C2A44B0EB930FF8D3CCF830208CF87C
:10AA70000040CCF80C4030BC002070474FF443300D
:10AA80000168880A424211EB822218BF401C4042F2
:10AA900001EB8000C01C20F00300704720850010EF
:10AAA000E41B0200FEFDFFFFFDFDFFFF08A80010F4
:10AAB000EFBEADDEF148002202704270827002717A
:10AAC0004271C270DFF8B8C3114600200CEBC1031D
:10AAD0001A54401C0828FBD3491C2029F5D3704781
:10AAE00011F048BE2DE9F04115460E460746F8F72D
:10AAF00049FE00F008040820F8F73FFE2A463146D8
:10AB0000384611F037FE05462046F8F731FE284654
:10AB1000BDE8F081D94880787047D84840787047C0
:10AB2000D649002048707047D44908208871704782
:10AB30002DE9F0410026F7F750FB044610F00F0511
:10AB400043D02846F7F74CFB012D18D0FBF792F9BC
:10AB500044EA0064002322460321072004F054FD48
:10AB600014F0060F31D00126FBF77EF9054605F0FB
:10AB700009FC0746022D17D0052D09D025E0FBF76B
:10AB800073F9BE498A79904218BF8871DED1E7E730
:10AB900014F0020F0BD1BB4C206840B10120F9F733
:10ABA0002FFF0020206002E00120F9F729FF01F0CB
:10ABB00031FA002818BF01F034FA022F05D0022D17
:10ABC0004FF0020004D001F005FA3046BDE8F081F4
:10ABD00005F080FCF9E72DE9F04F83B00026F9F786
:10ABE0005AFAFBF741F9022804D101F07BFD002855
:10ABF00018BF0126FBF738F9052814D1F9F716FF1D
:10AC000088B101F004FA5A280DD301F025FA002882
:10AC100018BF012001F023FA0120F9F7F1FE00200E
:10AC2000F9F7FEFE0126FFF783FF002818BF012673
:10AC3000DFF8489299F80200002800F08482D9F8E1
:10AC400008006D464FF0FF34002740B1D9F80820C6
:10AC500000230121084604F0D7FCC9F80870F8F772
:10AC600091FD00F0080A0820F8F787FD99F8030025
:10AC7000DFF80CB2F0B199F805000BEBC001401CF5
:10AC8000C0B289F80500202828BF89F8057099F816
:10AC90000300401E89F803004C7891F800800020E2
:10ACA000002C05DD0A1892782A54401C8442F9DCF5
:10ACB0000F704F705046F8F75BFD002CC0F23382E6
:10ACC00008F0FF000024272880F0EC81DFE800F086
:10ACD000C136F01D28391446EF4BC1888EC2EE9361
:10ACE0009DA9EDECEBEAE9F1E7E6E5E4E3E2E1E07A
:10ACF000DFC1DEDDC1DCA3009DF80000AC280CBF85
:10AD000001200220FBF77FF918E09DF800100120D8
:10AD1000FBF7C5F8012089F80100044600F0C2B92C
:10AD20009DF80310009861F31F6001F0C1FF01213D
:10AD30000320FBF7B4F8012089F80100012400F09A
:10AD4000B1B9BDF8000040BA05F001FB02210320B3
:10AD5000FBF7A5F8012089F80100EFE79DF8011045
:10AD60009DF8000087E04FF0010A89F801A099F8EA
:10AD7000000088BBF7F726FA70B39DF8005089F8F9
:10AD800000A0FBF771F8012808BF002515F0040F9B
:10AD900018BFFCF704FD15F0020F07D0FF210F20AC
:10ADA000FBF7E2FEF9F707FF45F0010515F0010F8B
:10ADB00010D0FBF759F8022802D105F0E3FA48B1A8
:10ADC000FBF752F8052802D101F00FF910B100206D
:10ADD000F9F7DDFE89F8007089F8017000F062B9BA
:10ADE0009DF80000401E01F01DFCA7E79DF8000043
:10ADF00005F093FBA2E79DF8000010F00F0018BFCC
:10AE000001200CF01CF800F04DB99DF800000CF08A
:10AE10000CF800F047B99DF8000005F092FB00F037
:10AE200041B99DF8000018B1012809D000F03AB9E5
:10AE300000200FF03BFA00200EF01DFE002006E07F
:10AE400001200FF033FA03200EF015FE01200EF062
:10AE500040FE27E19DF8000058B1FBF705F80228F5
:10AE600018BF012405F03EFB01460220FBF717F84E
:10AE700018E100210620FBF712F85FE7608500105B
:10AE80007CAA0010C885001008E100E1FAE0D3E0D8
:10AE9000CDE0DEE0BEE06CE0D3E023E01DE017E0B3
:10AEA00007E095E086E07FE066E057E02CE03DE0DB
:10AEB000B9E09DF80000002818BF012005F0FBFA5A
:10AEC0009DF80000002818BF012001F079F8E9E0A2
:10AED0009DF8000005F0DBFAE4E0BDF8000005F0A5
:10AEE000ACFB2BE79DF8000020B1012840D00228E0
:10AEF00005D0D7E04FF44330F8F738F8D2E001F04E
:10AF00007DFC00210420B6E7F8F73CFC00F00804C3
:10AF10000820F8F732FC99F80300002808BF89F8E8
:10AF200002702046F8F724FC0121A3E79DF80000F9
:10AF3000062805D2DFE800F004070A0C030F98E7A3
:10AF40000221084697E70221052094E7002103E04B
:10AF5000002104208FE7042103208CE79DF80300E3
:10AF6000009A002360F31F626221072004F04CFB6B
:10AF700098E0FAF711F9E1E69DF800009DF801105C
:10AF8000000140EA11100AF03DFC9DF801109DF807
:10AF9000020001F00F0140EA01200AF039FC9DF89F
:10AFA00003000AF041FC32E0BDF8000040BA0AF0AC
:10AFB00016FC77E09DF800000AF04EFC9DF80100B9
:10AFC0000AF05DFCBDF8020040BA0AF06BFC69E0D3
:10AFD0009DF800000AF07BFC9DF801009DF802102E
:10AFE000000140EA11100AF084FC9DF802109DF85F
:10AFF000030001F00F0140EA01200AF06EFC9DF809
:10B0000004000AF082FC9DF805000AF084FC0AF0B6
:10B010008EFC47E09DF800000CF02AFB9DF8000034
:10B0200000287FF48BAE0020F9F7EAFC86E69DF855
:10B03000000005F0B1FB81E69DF8000005F0B4FBCF
:10B040007CE69DF80000002818BF0120FBF70AF8F5
:10B0500074E60CF004FB9DF8004005F077FB012C32
:10B060000AD0022C08BF40F0805005D0042C14BF39
:10B07000082C40F0005001D105F0A1FA20460CF058
:10B08000E9FA5BE69DF800000FF0A3FA0AE09DF8EC
:10B0900000000CF0D6FA05F0ABF903E09DF80000D3
:10B0A00000F048F90CB101263DE0D9F808006D46E2
:10B0B0004FF0FF3440B1D9F80820002301210846A1
:10B0C00004F0A2FAC9F80870F8F75CFB00F0080A6F
:10B0D0000820F8F752FB99F80300F0B199F8050041
:10B0E0000BEBC001401CC0B289F80500202828BF26
:10B0F00089F8057099F80300401E89F803004C7820
:10B1000091F800800020002C05DD0A1892782A545E
:10B11000401C8442F9DC0F704F705046F8F728FB52
:10B12000002CBFF6CDADF8F72DFB00F00804082089
:10B13000F8F723FB99F80310002908BF89F802707B
:10B140002046F8F715FB002E14BF0120002003B0A5
:10B15000BDE8F08F02460020022928BF704752B197
:10B16000012A18BF704701EB4100C0EB4110FE49B6
:10B1700001EB8000704740F2DB104843FB49F7E7E2
:10B18000DFF8ECC300FB01F31CEB030C88BF704736
:10B19000F84B1A62C3E906017047DFF8D8C30028EC
:10B1A000DCF8183018BF0360F2480029C06918BFE6
:10B1B0000860002A1CBFDCF820101160584370475B
:10B1C000EC4801214171007840F2DB1180F0010070
:10B1D0004843E64901EB80007047E648C278002109
:10B1E00032B1027922B9027882F001020270C17094
:10B1F00041717047DF491E284A78487008BF002017
:10B2000003D01F2808BF012000D1087010467047E6
:10B21000D848007840F2DB1180F001004843D34960
:10B2200001EB800070472DE9F007D24F97F800C07E
:10B2300040F2DB140CFB04FCCC4CBE6904EB8C0C20
:10B2400003FB06F40CEB440C8E4234BF35460D462E
:10B25000FC69E31A934238BF1A46BB78012B16BF2C
:10B26000052B6C0800244FF00008002A9CBFBDE8A5
:10B27000F00770472346AC420FD297F80290B9F11D
:10B28000050F30F8139006BFA3EB040A2CF81A90B0
:10B290002CF813905B1CAB42EFD308F101080CEBC8
:10B2A000460C00EB41009045E4D3BDE8F007704741
:10B2B0002DE9F041AF4F14468C4601467A78069846
:10B2C0001D468A4218BFBDE8F0810121397101286D
:10B2D00002D0022824D029E0387840F2DB1148431C
:10B2E000A249BE6901EB8001A64234BF3246224624
:10B2F000F869A84238BF05460023002D16D9002062
:10B30000002A06D91CF8007021F81070401C8242F7
:10B31000F8D85B1C01EB4601A444AB42EFD305E037
:10B3200000232A4621466046FFF77DFFBDE8F04135
:10B3300000F0A2BC8F4A01281146D072497808BF9C
:10B34000242004D0002806BF2429FF207047507015
:10B3500070478848C07A704770B4DFF81CC2DCF8C8
:10B3600000C0DCF818C01CF0040F1ABF012424EA46
:10B370000C060CF0010605680C68002E1CBF1B1B98
:10B380005C1E1CF0020F1CBF521B551E1CF0040F4C
:10B3900019BF04600D6005600C6070BC7047002828
:10B3A00008BF70477349754B4A7875491B78002A66
:10B3B000097818BF022A05D0042A18BF092A01D02B
:10B3C000012230E76F4A1278012A84BF6E4A13784F
:10B3D000012200F06BBC2DE9F041664C0F460121C3
:10B3E00021716A4A1578654A167828B1A170002340
:10B3F00032462946FFF717FF3FB10520A070002312
:10B40000324629463846FFF70EFF00F035FCFF2094
:10B41000A070BDE8F0812DE9F04FDFF858918BB0B6
:10B42000012189F804105949564C574E0D7853495B
:10B43000DFF838B10F7899F8011012292FD00CDC01
:10B4400004291CD004DC002918BF02290DD116E004
:10B45000092914D0112922D007E013291FD021294E
:10B4600018BF22297ED024297DD0002800F0308109
:10B4700000233A462946FFF7D6FE00F029B9217885
:10B48000012902D9424937780D78002800F020813F
:10B4900000233A46294600F009FC00F019B9F6F7F6
:10B4A00088FDF6F7C1FC0090002818BFF6F716FFDC
:10B4B0002078012888BF3778F6F78CFE10F0040F4B
:10B4C00018BF7F1CDFF8CC8099F80100A0F11106AD
:10B4D00099F8000040F2DB114143D9F818000BEB5A
:10B4E0008104A84238BF0546D9F81C00B84238BFCD
:10B4F0000746F6F78CFF01900020F7F7A6FA4FF009
:10B50000000A002F52DD4FF00009002DC4BF0AEBE6
:10B510004A0000EB0A1B41DD019810F909002628BA
:10B5200024BF002024F8190018D200F0010108EB14
:10B53000413100EBD07001EB8B01401051F820102D
:10B540004FF0FF3046B3012E08BFC8B204D0022E20
:10B5500004BF0846F7F77FFA24F8190009F101093A
:10B56000A9451AE02FE036E054BA00107CAB001079
:10B570004AFCFFFF6C85001048860010EA8400102A
:10B58000F0840010EB840010ED840010E9840010BA
:10B59000EC840010008000300EE0BDDBF7480AF1BB
:10B5A000010ABA45806904EB4004ACDB009800282E
:10B5B00018BFF6F796FE8BE011F4803FC1F3072029
:10B5C00018BF4042C8E700287ED00023BA1C294695
:10B5D000FFF729FE7CE000287AD00646E84800689C
:10B5E000007E10F0040F07BF2C46BA463C46AA4620
:10B5F000A2084FEA9A000590A4EB940106900092ED
:10B600006008491ECDE901104FEA5A000790AAEBE5
:10B610009A00401E08900990CDE903215346224626
:10B6200005A96846FFF798FE5346224605AF06A9CE
:10B63000E84601A8FFF790FE5346224607F10801AD
:10B6400008F10800FFF788FE5346224607F10C0177
:10B6500008F10C00FFF780FE5346224607F1100167
:10B6600008F11000FFF778FE99F8000040F2DB11B6
:10B67000414300220BEB8100914620F8129058F8CC
:10B680002210A1F1010C491C61451CD357F822106E
:10B690004B1E491C99420FD303FB05C136F91140DB
:10B6A00030F912108C42C8BF20F8124057F822100F
:10B6B0005B1C491C9942EFD258F822100CF1010C86
:10B6C000491C6145E2D200E002E0521C052AD4D3B5
:10B6D0000BB0BDE8F04F00F0CFBAA848012181724D
:10B6E000807980F0010000EB4001C1EB4010A549DA
:10B6F00001EB80007047A148027A002132B1427A02
:10B7000022B9827982F001028271017281727047DE
:10B710009A491E28CA79C87108BF002003D01F2883
:10B7200008BF012000D18871104670479348807986
:10B7300080F0010000EB4001C1EB4010914901EBAA
:10B74000800070472DE9F04F8F4985B0012291F8B4
:10B7500000808E4991F8009088494A72C979894CD5
:10B7600011291CBF1229132936D0F8B183498979D0
:10B7700001EB4102C2EB411104EB8102002119EB04
:10B78000080C18BF7E4C11D02368B9F1000F5B8AFA
:10B7900003BF30F811500B4422F8135030F8113029
:10B7A00018BF22F81130491C8C45EDD8F7F7EAFF95
:10B7B00000F008050820F7F7E0FF704CA07A002899
:10B7C00018BF01217ED021722846F7F7D1FF002053
:10B7D000607205B0BDE8F08FF6F7EBFBF6F724FBDF
:10B7E0000190002818BFF6F779FD6448C179A1F1EE
:10B7F0001105416A0091807900EB4001C1EB4010D6
:10B8000004EB8006F5F79BFC614F62494FF0110A8B
:10B81000002804BF8B46012004D0BB4650460F468B
:10B820004FF0010AF7F711F9F6F7EFFD0024039046
:10B83000B9F1000F28D900984C2148430290039891
:10B840000057262824BF002026F8140019D200F043
:10B8500001010BEB413200EBD0700299401001EB7B
:10B860008000002D11584FF0FF3049D0012D08BF46
:10B87000C8B204D0022D04BF0846F7F7ECF826F84A
:10B880001400641C4C45DAD306EB49065046F7F722
:10B89000DCF8F6F7BCFD00248246B8F1000F29D988
:10B8A00000984C2100FB01F94FF0000B1AF904003D
:10B8B000262828BF26F814B019D200F0010107EBA2
:10B8C000413100E02AE000EBD070401009EB80002D
:10B8D00009584FF0FF30D5B1012D08BFC8B204D0D0
:10B8E000022D04BF0846F7F7B6F826F81400641CCA
:10B8F0004445DBD30198002818BFF6F7F2FC55E762
:10B9000011F4803FC1F3072018BF4042B7E711F49C
:10B91000803FC1F3072018BF4042E6E7A07980F0DE
:10B920000100A07100214EE770B50D4613490122B8
:10B930000A71194A49781678184A212914781EBFC5
:10B940002229232970BD002818BF002D11D0002303
:10B9500022463146FFF767FC631C01222146284638
:10B96000FFF761FC05EB4400A31C01223146FFF701
:10B970005AFCBDE8704000F07FB900006C850010F3
:10B980004886001054BA0010EE840010EF840010B6
:10B99000B09D0030189D0030E9840010EA8400104A
:10B9A00070B5E54D0446687890B9E06868B1E34940
:10B9B0000978012994BFE249E2490B78E249012262
:10B9C000097800F073F9687810B9A068FFF723FDD3
:10B9D0006878112804BF0020FFF71DFD6878122841
:10B9E00004BF0020FFF717FD6878132804BF00206C
:10B9F000FFF711FD206920B1E979002908BFFFF7A1
:10BA0000A1FEE879112804BF0020FFF79BFEE8792A
:10BA1000122804BF0020FFF795FEE879132818BF0D
:10BA200070BD0020BDE870408CE62DE9F74F8046E0
:10BA3000C6480D46002690F800A0C148BE493446CD
:10BA400090F80090BAFBF5F000FB09F701200871AF
:10BA5000487B0978DFF8F8B288420ED0B64A40F247
:10BA6000DB1148430BEB8001107840F2DB125043AE
:10BA70000BEB8000920010F028FE0298002888BF8F
:10BA8000DFF8B4B22DD99BF80EC00022BCFBF9F050
:10BA900009FB10C101FB0AF100FB0510002D12D9B2
:10BAA00038F814309BF8001040F2DB1E01FB0EFE4C
:10BAB000A749641C01EB8E0100EB020E521C21F819
:10BAC0001E309542ECD80CF10100C0B28BF80E008C
:10BAD000B84224BF00208BF80E00761C02988642E4
:10BAE000D1D39549887B401EC0B2887387429CBFE2
:10BAF000781E88730878487303B0BDE8F04F00F0F3
:10BB0000BBB8944A30B41268B2F810C0538A00220D
:10BB1000BCF1000F07D99C1830F8144021F81240EE
:10BB2000521C9445F7D80022002B9CBF30BC7047B4
:10BB30009C1A44BF30BC704700EB44040CEB020578
:10BB400034F8024C521C21F815409A42F0D330BC14
:10BB500070477948017800F1280281F0010132F83C
:10BB60001110002918BF7047017881F001010170A0
:10BB700000210182037822F81310774A00781154CB
:10BB800070476D49087370476B48007B704770B50C
:10BB9000694C0025257025732582658240F6D861A1
:10BBA0006B4810F088FDA562A58270BD62490878D7
:10BBB00000224A8280F001001431095C69B140F230
:10BBC000DB11634A414332F82110A1F55062B63AC5
:10BBD00002BF624931F81000704700207047564B91
:10BBE000187803F1140C80F001014FF6FF701CF877
:10BBF0000120012A18BF704740F2DB104843544A25
:10BC000002EB80005A8A30F81200521C5A82534BC1
:10BC100033F81120521E1204120C23F8112004BF15
:10BC200000220CF8012070474C49A1F1280213783A
:10BC300001EB43010B8803440B8092F800C0012103
:10BC400002F1140303F80C10118A084410827047A3
:10BC5000394A138A03EB5000414B01445B1824BF5F
:10BC600000207047117840F2DB125143384A02EB52
:10BC7000810101EB4000704770B5F7F783FD00F0DC
:10BC800008060820F7F779FD2B4C6079002500287D
:10BC900001BF207880F001002070E5701CBF0120FA
:10BCA000E0703046F7F764FD257170BD2DE9F0476F
:10BCB000994616460D460446F6F7AEFB5FEA000CC1
:10BCC0001CD01D49087840F2DB125043204AD1F8BD
:10BCD000188002EB800009FB08F200EB42004545AA
:10BCE00094BF2F464746C969A1EB0901B14238BF4D
:10BCF0000E460021002E09D8BDE8F0874B4632469B
:10BD000029462046BDE8F047FFF78DBA0023002FF3
:10BD100008D91CF9032034F8122020F813205B1CEA
:10BD20009F42F6D8491C00EB480004EB4504B142A1
:10BD3000ECD3BDE8F08700006C850010EB840010A8
:10BD4000EA840010ED840010F0840010E9840010F3
:10BD50007CAB001048860010808500109485001090
:10BD60004AFCFFFF3B49002814BF00200120087057
:10BD700070473848007800280CBF01200020704729
:10BD800001203449487070473248002141700178E1
:10BD900000291ABF4068002870474FF040204169D1
:10BDA00021F00101416170472A48017829B14FF023
:10BDB00040214A6942F001024A61002141608160EC
:10BDC000C160016170472348017829B14FF04021DB
:10BDD0004A6942F001024A61002141608160C1600C
:10BDE0000161704700B50178427883B0890141EA6A
:10BDF00082018DF80010418809098DF801108188B1
:10BE000009098DF80210817801F00F02017962F3BF
:10BE10001F118DF80310017A8DF80410417A8DF806
:10BE200005108179C27901F03F0102F00C0241EA6C
:10BE300002118DF80610C179807A890100F00100A5
:10BE400041EA40108DF80700684610F098FC03B0F6
:10BE500000BD000098850010002818BF2D482E490D
:10BE6000886370472C48806B2A4988420CBF0120A8
:10BE70000020704728487047284B4FF0000C1C6882
:10BE80001B1F1D68244B19605A602549D963DC6269
:10BE900014F0804F22D0290C5985290A83F82910E3
:10BEA00083F82850598D19B1598D012242EA014C6D
:10BEB00093F8291039B193F82920022141EA024C64
:10BEC00018490C681C6393F8281039B193F82810AE
:10BED000032242EA014C14490C685C634FF0402194
:10BEE0004C67C1F878C08269CA67B0E834109A60BC
:10BEF000DC601D61C3F814C090E815109861DA6128
:10BF00001C62C3F824C0986B024A904204BF0748E1
:10BF10000867FEE7504D5544005F01102CED00E02E
:10BF2000544C414638ED00E034ED00E0AD2007B060
:10BF300070B50E460446F9F797FF042811D1A4F511
:10BF4000A07048280DD2A019A0F24110482808D2AC
:10BF500065020024002E04D92846F7F707F80128C7
:10BF600001D0002070BD641C05F50075B442F3D308
:10BF7000012070BD70B50D460446F9F775FF042821
:10BF80000AD1A4F5A070482806D260022946F7F726
:10BF90008FF8012808BF70BD002070BD10B5074C98
:10BFA000FEF719FE012808BF10BD206800F0FAFC5A
:10BFB000002818BFF9F7BAFFF2E700004886001022
:10BFC000FB4A0028916814BF41F0010021F00100F4
:10BFD00090607047F64B99680A0E120721F07F4176
:10BFE00042EA0060084398607047F1488068C0F3F7
:10BFF00003607047EE488068000F7047EC483221BC
:10C00000C0684843EB49A1FB001080087047E8482E
:10C0100000697047E648006A7047E54901200862F8
:10C020007047E349002008627047E1480078704794
:10C03000002818BF0120DE4908707047DC48406ABC
:10C040007047DB480021416201707047002818BF2B
:10C050000120D74988707047D548807870470028FC
:10C0600018BF0120D249C8707047D148C0787047C6
:10C070002DE9F04184B000270EF0C1FA0646A02158
:10C08000CD4810F081FB002425464FF00308305DB9
:10C0900010F0800F19D0601C8DF801008DF807504A
:10C0A0008DF80080ADF804508DF80850ADF80250BE
:10C0B0008DF806508DF809508DF80E503555012732
:10C0C00000226946BC48F4F77BFA601CC4B20A2C13
:10C0D000DDD3BA4CE07A68B1012F0BD10021B6480C
:10C0E000F4F726F9E07C28B100231A460321042046
:10C0F000F4F715F904B0BDE8F0410EF0FCB870B5E6
:10C100000546002404F04CFA70B10BF0A8FA082898
:10C110000AD0AB4800EB0510C168A548C26A91423D
:10C120001CBF012101630124204670BDA44A0146C1
:10C1300002EB01110120CA689D49CB6A9A421CBFDB
:10C1400001220A6370472DE9F04FDFF878A287B02B
:10C15000DAF80000B0F90211B0F9000110F0FBFAB2
:10C16000F4F74AFB0120F8F74BFC0020F6F7CCF877
:10C170000EF01CFA042000F05FF9F8F727FC09F034
:10C1800085FCDFF82C9200240120C9F81040C9F882
:10C190001440C9E9064010F0FCFA0020C9F80C4030
:10C1A000F9F730FAF9F760FE052808BFDFF810B29A
:10C1B0006CD1D9F80800010FC0F30367B94206D06B
:10C1C0000020C9F81000C9F81400C9F81800DAF8FE
:10C1D0000000B9000024D0F8EC00A04620FA01F1DC
:10C1E00001F00F05C0F30320854204BF0020C9F809
:10C1F00030002AD1DAF80000D0F8EC100BEB041074
:10C2000002799200D14001F00F060F2E04D0816810
:10C2100020468847012807D0641C022CEAD3D9F8AD
:10C22000300001280BD102E03546A046F7E70BEBC2
:10C230000810C068C9F82C000020F8F7E1FBD9F815
:10C240002800A84218BFC9F828503946052003F035
:10C25000C2FA002F7ED0022F24D0042F7BD0D9F831
:10C2600008000A2F4FEA106120F07F404FEA017169
:10C2700018BF41F000710843C9F80800FEF7ABFC95
:10C28000012803D0F9F7F0FD052892D00EF033F81D
:10C29000F8F7B5FB0EF091F907B00020BDE8F04FBC
:10C2A000F9F79DB90D212846F9F762FF0028E5D07E
:10C2B00010F074FA10F077FAF8F74CFB04006FD125
:10C2C000F5F7B6F94048F5F7FAFD0120F5F7EAFD74
:10C2D000F7F77AFA3D48F7F730FBF7F717FBF7F770
:10C2E00040FBDAF800104000B1F8FA20B0FBF2F0A1
:10C2F000401CC0F34F00A9F8040091F8FC1089F825
:10C30000011059B1F7F72DFBDAF800104000B1F831
:10C31000F810B0FBF1F0401CC0F34F00F7F792FAB1
:10C320004FF040262A48B061F5F743FEF5F7BAFF13
:10C3300099F8010048B1401E10F0FF0089F8010093
:10C3400004BFB9F80400F7F77DFAD9F80800C0F384
:10C35000036501E068E06BE029460520F3F7C1FFC3
:10C36000FEF739FC012807D0D9F80800C0F30360B4
:10C37000A84208BF002C2FD0F6F725FA1548B06167
:10C38000F7F798FAF7F7CDFA0020F7F7D6FAF7F7AC
:10C3900026FAF5F70EFEF5F749FD0020F5F78FFDBB
:10C3A00010F001FA10F004FAFAF72CF866E7000032
:10C3B000AC850010ABAAAAAA908800107C88001057
:10C3C000E0850010488600100D400010D1380010A4
:10C3D00007005FA000005FA06846F6F7ACF9B0B1B7
:10C3E0006846FFF7DDFA0198F7F7A2FEF9F73CFD82
:10C3F0002946009A06F0B6FE684610F0DEF90446BB
:10C4000006F026FFF6F7DFF9F9F7B1FDA8E7DAF84D
:10C410000000D0F89C0010F0704F02D0F9F786FDB4
:10C420009EE7F9F7ABFD9BE7284610F0CBF925E72F
:10C43000284604F006FB21E72DE9F047DFF88CA041
:10C4400001468900DAF8000000242746D0F8EC0005
:10C4500020FA01F101F00F05C0F30320854231D12C
:10C46000DFF86C90002009F13408C9F83000DAF8E0
:10C470000000D0F8EC1008EB041002799200D140D3
:10C4800001F00F060F2E04D081682046884701284E
:10C4900007D0641C022CEAD3D9F8300001280BD154
:10C4A00002E035462746F7E708EB0710C068C9F8F1
:10C4B0002C000020F8F7A4FAD9F82800A84218BFE9
:10C4C000C9F828502846BDE8F087000048860010CB
:10C4D000AC8500107047002808BF704780220146D5
:10C4E000014810F0E3B870473CC3001070470528BE
:10C4F0003CBF9349087070470020914948609148BB
:10C50000006890F8B900052838BF08707047704778
:10C510008B480078704770B58A4D0024286890F8E1
:10C52000A40010F0020F0BD0F9F79EFC022807D1EF
:10C5300083482968007801EB8000B0F8BC0084B221
:10C54000204670BD70B57F4D4FF48054286890F838
:10C55000A40010F0020F0DD0F9F786FC022809D1D3
:10C5600077482968007801EB8000D0F8BC00000C07
:10C57000C0F31304204670BD71488078002818BFAE
:10C58000012070472DE9F041F9F76EFC022803D134
:10C5900003F0F8FE022803D04FF48050BDE8F0818C
:10C5A0004FF480552E4603F0B5FFDFF8988104461E
:10C5B000634FD8F8000090F8A41011F0010F0CD0D0
:10C5C000B0F8AE0079684042814206DC2CB1002010
:10C5D000641E7860204603F0A0FFD8F8001091F8A0
:10C5E000A40010F0040F18BF002C0AD0B1F8B4005A
:10C5F000621E9040B1F8B620824238BF1046C0F3A8
:10C600001306D1F8DC0010F0020F1CBFB978002926
:10C6100002D0000CC0F31305B54298BF354628463A
:10C62000BDE8F08100207047464845490068B0F8F1
:10C63000AE00424248688242BCBF401E486070471C
:10C64000002070473F4810B50068D0F8DC0010F4B7
:10C65000807F06D0C0F30330012101FA00F0F6F725
:10C66000F6FD374900204870887010BD70B5344D14
:10C670000024A878002814BF01260026687828B96D
:10C6800003F057FF002808BF002100D001218E428F
:10C6900026D00A1C18BF0122AA702A480068D0F8C8
:10C6A000DC3013F0040F0DD021B1C3F303100528C3
:10C6B00007D205E00021696090F8B900052800D292
:10C6C0002870012413F0020F18BF0124002A18BF9C
:10C6D000012200238221072002F096FFF3F731FEAA
:10C6E000204670BD174900200968D1F8DC1011F40C
:10C6F000807F08BF7047DFF848C09CF80120131CFA
:10C7000018BF012330B4104CC1F30332E46B012590
:10C7100005FA02F2224011F4007F01D00AB102E0D2
:10C720000AB1002100E001218B4204BF30BC7047F8
:10C73000081C18BF01208CF8010030BC96E70000EF
:10C7400034860010488600100010004081480078B0
:10C7500070478048406800F5407070477D484068E9
:10C7600000F58070704770B57A4C4FF420307A4AEB
:10C7700060600168914204BF4168B1F5087F3BD118
:10C780008168B1F5E04F37D8744AC568954223D027
:10C790004FF0000C03466246BCEB910F0AD253F8EF
:10C7A000046B521C86EA0C0CB2EB910FF7D3BCF170
:10C7B000000F21D1026A7AB14FF0000C03466246A5
:10C7C000BCEB910F06D253F8046B521CB444B2EB8D
:10C7D000910FF8D365450FD1012500F5807000F069
:10C7E000E1F848B1606800F5407000F0EAF8002810
:10C7F0001EBF2570012070BD002070BD554900206E
:10C8000008704FF42030F6F7B1BB5248017841B1BF
:10C810004068514A0168914202BF4168B1F5087F02
:10C820007047002070474B4B5B6803F580731844DA
:10C83000F6F792BC474B5B6803F540731844F6F774
:10C840008BBC4448406800F580607047414B5B6892
:10C8500003F580631844F6F77FBC3E4840680069E2
:10C8600070473C4949680A6982429CBF0020704772
:10C8700000EB400001EB001000F5A0607047354A66
:10C88000526802EB80035B6A1A44354B53F820C0B0
:10C89000403333F810000CEB0003401E5B1E23EA0C
:10C8A000000000FB012070472A4988607047294832
:10C8B000806870472DE9F00F264B0022DFF8A0803A
:10C8C000D3E90145012708F140069146831893F901
:10C8D00020C0BCF1000F18DB07FA02F32B4214D082
:10C8E000D3B204EB830A58F823B036F81330DAF8E1
:10C8F00024A09B445B1EABF1010BA2442BEA030373
:10C9000003FB0CA341F8223001E041F82290521CB5
:10C91000102ADBD3BDE8F00F70470029B8BF70477D
:10C9200030B494460B4A0F4C526802EB80035B6AAA
:10C9300013440B4A52F8202034F810001418401EFB
:10C94000641E24EA000001FB003030BC6146F6F7AB
:10C9500003BC00003C86001054465053EFBEADDED1
:10C96000E81B0200281C020010B5FFF7FCFEA8B16E
:10C97000FFF7EFFE0146E42217480FF097FEFFF79E
:10C98000EDFE164C01464FF4DE7220680FF08EFE6D
:10C990002068806BBDE8104003F040BD0220F9F72D
:10C9A00032FBE2E758B10E4A0168914207D1406874
:10C9B00020F00F00B0F5247F04BF01207047002055
:10C9C000704730B1006820F00F00702804BF0120CC
:10C9D0007047002070470000F82F011048860010B3
:10C9E00041505352A94810B5806810F0020F15D07D
:10C9F000F5F71AFA90B1F5F7D9F90402F9F734FA14
:10CA000044EA0044F9F736FA44EA00604EF2AF0116
:10CA100008434FF04021C867012010BD002010BD21
:10CA200010B572B60120F6F7A5F9F7F759F8F7F740
:10CA300083F84FF0FF30F6F7A0FE954880234FF4BF
:10CA40000052002152F821C040F821C0491CB1EB2E
:10CA5000930FF7D3F6F7A3FEF7F7E2FAF7F704FB25
:10CA60008C48F7F71DFB0120F7F7DBFAF6F716FA0B
:10CA70001E20F7F7CCFAF7F77BF8F6F7F3FBF7F79A
:10CA800077FAF7F7BBF8F6F79BFEF6F767FCF5F7D2
:10CA9000E0F9FFF769FFF6F71AFEF6F7E5FDFEF796
:10CAA00009F8FAF721FFFFF78EF962B6F9F756FB9E
:10CAB000794C206890F89C0000F00F00F6F76CF8B5
:10CAC0002068018BC1F30722418A008AFEF758FBD8
:10CAD0002068D0F8A000000C02F093FD6F480DF024
:10CAE000EBFB2068B0F900010DF05EFDF3F7DAFB17
:10CAF000FFF7FCFCF7F7F7FAF9F7C1FCFFF7EAFCE0
:10CB00000FF065FEFAF798FE00210320F9F7C7F948
:10CB10004FF040242069002300F0700219460220E3
:10CB200002F072FD206910F0200F17D0226F002351
:10CB30000521072002F068FD626F00230521072010
:10CB400002F062FDA26F00230521072002F05CFDC8
:10CB5000E26F00230521072002F056FDFFF772FD6A
:10CB60000020206710BD02244D4DFEF734F8012847
:10CB700006D0F9F779F9032802D102F058FE58B32C
:10CB8000002D05DC03F0AEFC01460220F9F787F921
:10CB9000DFF814914FF00108424FDFF810A14FF079
:10CBA0004026A9F1030BF9F75FF90546F9F762F999
:10CBB0000146284602F00FFEF9F75CF901462846C7
:10CBC000F3F78FFBFDF7B0FF072D5BD2DFE805F031
:10CBD0005A1D08272A192D006D1E002DC5DCD1E72E
:10CBE000387850B9FAF794FD38B900231A46202155
:10CBF000072002F009FD87F8008004F090FA022473
:10CC0000D1E7FFF7A0FA0524CDE7FAF7D0FBF9F753
:10CC10002BF9012804BF2046F9F738F9C3E703F0E0
:10CC200028FBC0E7FFF7BAF9BDE7C6F81890F6F79A
:10CC3000CBFDF6F76BFEF6F794FE4000AAFB001062
:10CC40004009401C4008F6F7FDFDFDF7C4FF012830
:10CC50000CD1F9F709F9062808D0F6F72BFEF6F7FC
:10CC600060FEF6F7BCFDC6F818B09CE7F9F7FFF8D0
:10CC70000546F9F77CF915B1F9F780F9E5E7F9F719
:10CC800055F9E2E70220F9F7BEF98CE70080004091
:10CC900000E9001095E9000048860010F82F011007
:10CCA000FF7002004C86001003005FA0CDCCCCCCFE
:10CCB000FE4948607047FD4880687047FB4908702E
:10CCC0007047FA48007870470200F9484FF00801B1
:10CCD0000068438A008A03FB00101CBFC01C20F0C0
:10CCE0000300704730B4481E022882BF002030BCC9
:10CCF00070474FF43C300122ED4B1B688A4204BF61
:10CD000030BC70474FF0080C5C8A1D8A521C04FB33
:10CD100005CC0CF1030C2CF0030C6044032AEDD974
:10CD200030BC70472DE9F04F0F4690F821A090F8E5
:10CD3000209000F15005ADF20C4D1646012411462D
:10CD40003846FFF7CFFFDB4A4FF0000830B10168EB
:10CD5000914204BF4068CDE9001001D0CDE9002820
:10CD6000D5480AFB09FC0068B0F93A20B0F9383020
:10CD7000002096469B46BCF1000F0ED935F91010E5
:10CD80007145D8BF8B4505DC9942C8BF0B4691421F
:10CD9000B8BF0A46401C8445F0D8981800EBD07004
:10CDA00042100023BCF1000F88BFE94616D935F9BF
:10CDB0001300801A00EBD07041107F29C8BF7F217B
:10CDC00005DC11F1800FB8BF6FF07F0100DA00249D
:10CDD00009EB03005B1C01729C45E8D88DF8044008
:10CDE0009DF80500FF283CBF401C8DF80500ADF8FC
:10CDF00006206C4631463846FFF774FF78B1AC49DF
:10CE0000082209684B8A098A03FB01222146F6F7AA
:10CE1000A3F901280CBF4FF001084FF0000840466D
:10CE20000DF20C4DBDE8F08F70B505460124F9F701
:10CE300018F8411E022984BF002070BD9B498988D3
:10CE400011F4007F05D0024603212846FFF76AFF50
:10CE50000446204670BD9549C8607047934810B499
:10CE6000C068002808BF4FF44030944A01689142DE
:10CE70001CD14168B1F5007F18D383680022844635
:10CE8000B3F5056F88BF4FF405630021B1EB930F35
:10CE900024BF10BC70475CF82140491C2244B1EB10
:10CEA000930FF8D3002A04BF10BC7047002010BCB9
:10CEB000704770B50022C260D0F808C00121134647
:10CEC0000446BCF5056F88BF4FF4056C0022B2EB39
:10CED0009C0F06D254F82250521C2B44B2EB9C0FEC
:10CEE000F8D35A42C260714A127912F0800F07D10A
:10CEF0004FF440304FF405622146F6F72DF9014614
:10CF000001290CBF0120002070BDFF2270B5002553
:10CF1000044605614FF4006150300FF0EAFBA58430
:10CF2000E584E562A56265632563E563A5636564E1
:10CF30002564E5640120A56470BD2DE9F0414FF43E
:10CF4000403104465D4E0868B04218D14868B0F5DB
:10CF5000007F14D38A6800230D46B2F5056F94BF95
:10CF600094464FF4056C0020B0EB9C0F26D255F888
:10CF70002070401C3B44B0EB9C0FF8D3F3B1FF2270
:10CF80004FF4056120460FF0B4FB4FF40870C4E97C
:10CF900000604FF40560A0600020E06084F820008D
:10CFA00084F8210084F8220084F823002061606165
:10CFB000A061E0612046FFF7A8FF07E0B2F5056F2A
:10CFC00088BF4FF4056220460FF070FB0120BDE8DA
:10CFD000F08170B402684FF408715160016801F18A
:10CFE000500291F821C091F820300CFB03F102EBC4
:10CFF00041010022BCF1000F08D900EB4204521C91
:10D00000B4F8DE4021F8024B9445F6D80022002BFC
:10D0100008D900EB4204521CB4F8064121F8024B37
:10D020009342F6D80022BCF1000F08D900EB42046D
:10D03000521CB4F8644021F8024B9445F6D8002203
:10D04000002B08D900EB4204521CB4F88C4021F8A4
:10D05000024B9342F6D8B0F8DA2021F8022BB0F850
:10D06000DC2021F8022BB0F8D82021F8022B002474
:10D070000022BCF1000F0ED904EB440505EB0415AA
:10D0800000EB850505EB4206521CB6F8526121F80B
:10D09000026B6245F6D30022002B1AD904EB44053B
:10D0A00005EB041500EB85050AE000005086001032
:10D0B0004886001046544D336C86001053454C464C
:10D0C00005EB4206521CB6F8826221F8026B9A42C6
:10D0D000EAD3641C042CCBD370BC70472DE9F74F06
:10D0E00088B000250A992C462E460968049101F162
:10D0F00050030999002984BFFD49D1F800801CD94B
:10D100000022002888BFB8F93A700DD933F9021B04
:10D110000029B4BFC1F1000C8C46BC45BCBF0D4416
:10D12000641C521C8242F1D30999761C8E42E7D3CB
:10D13000002CC8BF95FBF4FA08DC4908414301EB19
:10D140005002049901EB4201B1F950A00021029173
:10D15000019104995031009100210391099900290E
:10D1600069D9E349009E069609684FF0000B4FF01D
:10D170000109B1F81CE091F824105F46D846CDF8BB
:10D1800014B00791002829D9B6F900204FF0000CFF
:10D1900006999344634600280DD9B1F90040A51AB9
:10D1A00048BF151B7545B8BF0CF1010C01EB4901D7
:10D1B0005B1C8342F1D307998C4503D305997F1CEF
:10D1C0001144059108F1010806EB49068045DBD3BF
:10D1D000002FC4BF059991FBF7F101DC9BFBF0F137
:10D1E000039B0A9A09B202EB4302A2F86410C04AF8
:10D1F0001268538BAAEB0303994209DD128B524448
:10D200008A4205DD019A114401910299491C02915B
:10D210000099099A01EB400100910399491C03917F
:10D2200091429ED30299002905DDDDE9011291FBAF
:10D23000F2F1019102E05146CDF804A00A9AA2F859
:10D24000DA100021029103910499503100910021DC
:10D250000491002865D9A649009F069709684FF0F8
:10D26000000B099EB1F820E091F82510D846D94668
:10D27000CDF814B00791002E2BD9B7F900204FF04C
:10D28000000C069993446346002E0DD9B1F9004075
:10D29000A51A48BF151B7545B8BF0CF1010C01EB71
:10D2A00040015B1CB342F1D307998C4504D3059927
:10D2B00008F101081144059109F1010907EB400744
:10D2C000B145DAD3B8F1000FC4BF059991FBF8F16D
:10D2D00001DC9BFBF6F1049B0A9A09B202EB4302C4
:10D2E000A2F88C10824A1268538BAAEB030399426E
:10D2F00009DD128B52448A4205DD039A11440391E1
:10D300000299491C02910099891C00910499491CB9
:10D31000049181429FD302980028C4BF039991FBD6
:10D32000F0FA0A98A0F8DCA001980A99504400B2DB
:10D3300000EBD0704010A1F8D8000BB0BDE8F08F22
:10D340002DE9F74F8CB0441E0E990E9B684E0A686B
:10D35000002119620E9B4FF0010ED9610E9B99615D
:10D360000E9B59610B460D99A1F1010C002953D96F
:10D37000002100284CD9DD1703EBD56525F01F07E8
:10D38000DF1B0EFA07FB6F110E9D05EB870A0AF1F2
:10D390001C0903FB001502EB4505002BB5F9507085
:10D3A0007ED0012B7DD0002B7CD0012B7BD00BB10C
:10D3B000634506D1002912BFA1423568B5F9A650D0
:10D3C00002D03568B5F9A450002D04BF3568B5F911
:10D3D000A450AF4219DDDAF81C5045EA0B05C9F834
:10D3E0000050CD1701EBD5684FEA68170E9D28F065
:10D3F0001F0805EB870505F114076D69A1EB080807
:10D400000EFA08F845EA08053D60491C8142C0D380
:10D410000D995B1C8B42ABD3316891F8C530002B62
:10D420001CBF91F8C410002900F026820D9900233A
:10D43000002940F221821F25012101FB005102EB4E
:10D4400041010B91002101FB005102EB41010A91C6
:10D450000D99891E0991811E03910021002840F237
:10D4600006825D1E0026019505FB006502EB450561
:10D4700008955D1C009505FB006502EB45050795C9
:10D48000DD1703EBD56525F01F069E1B012707FA64
:10D4900006F606966E110E9D05EB8605059503E0D2
:10D4A00016E027E01BE02CE01C35049503FB00157B
:10D4B00002EB450A012BBAF950707BD81E2979DBA3
:10D4C0001F2977DC2BB3012B2DD03BB330D035E0B7
:10D4D0001E2904BF3568B5F9AC503FF475AF1F295C
:10D4E00004BF3568B5F9B0503FF46EAF62E7000095
:10D4F0006C8600101E2904BF3568B5F9AE503FF4A4
:10D5000063AF1F2904BF3568B5F9B2503FF45CAF73
:10D510004EE71E2908BFBAF94E500FD01F2908BF89
:10D520000B9D0BD108E01E2908BFBAF9525005D057
:10D530001F2908BF0A9D01D1B5F95050AF42CCBF99
:10D540003E462E46E6B17E1B4FF0640806FB08F609
:10D55000002E0BDBAF42D4BFA846B8464644A6F126
:10D56000010600DD3D4696FBF5F70BE0AF42CCBF70
:10D57000B846A846A6EB080606F10106F3DDF1E77A
:10D580004FF0FF07002B00F01081012B00F01981F4
:10D5900013B1634540F02181002918BFA14240F03A
:10D5A0001D81FE4D2D6895F9C76095F9C65000F0B4
:10D5B00034B9FFE7A1F11E05012D94BF4FF0020918
:10D5C0004FF000090D9D6D1E0295012B94BF4FF089
:10D5D0001D08A04600252E464B4509D0012B1FD023
:10D5E000019E012506FB001602EB4606B6F95060C7
:10D5F000DDF808B05B452DD0DDF824B05B451FD1C8
:10D60000002914BF4FF0000B4FF0010BA1420CBFDB
:10D610004FF0010E4FF0000E5BEA0E0B1AD10FE037
:10D62000002914BF4FF0000B4FF0010BA1420CBFBB
:10D630004FF0010E4FF0000E5BEA0E0BD8D1CFE792
:10D64000DDF800B06D1C0BFB001B02EB4B0BBBF9B4
:10D6500050B05E4429B1012919D0BAF94EB06D1C01
:10D660005E44414527D0DDF80CB059451FD1002B51
:10D6700014BF4FF0000B4FF0010B63450CBF4FF090
:10D68000010E4FF0000E5BEA0E0B14D10FE0002BE1
:10D6900014BF4FF0000B4FF0010B63450CBF4FF070
:10D6A000010E4FF0000E5BEA0E0BDAD1D5E7BAF9A6
:10D6B00052A06D1C56444B4516D149B1DDF800A06F
:10D6C0006D1C0AFB001A02EB4A0ABAF94EA0564436
:10D6D000414509D0DDF800A06D1C0AFB001A02EBE1
:10D6E0004A0ABAF952A05644DDF808A0534516D1AB
:10D6F00049B1DDF804A06D1C0AFB001A02EB4A0ACE
:10D70000BAF94EA05644414509D0DDF804A06D1C7D
:10D710000AFB001A02EB4A0ABAF952A0564481B930
:10D720004B451CBFDDF808A053450AD0DDF820A00A
:10D73000AD1CBAF952A05644DDF81CA0BAF952A0AB
:10D740005644414518D14B451CBFDDF80880434580
:10D7500012D0DDF80480AD1C08FB001802EB48086D
:10D76000B8F94E804644DDF8008008FB001802EB53
:10D770004808B8F94E804644002D18BF002F3FF4EA
:10D78000FFAE4FF0640806FB08F696FBF5F507EBD5
:10D79000C70606EB0716D5EB860559BF3D446D1E3F
:10D7A000ED1B6D1C95FBF7F7ECE61E2902D01F2937
:10D7B0000CD0F1E6794D2D6895F9C96095F9C850FE
:10D7C0002BE01E2918BF1F297FF4E3AE734D2D688F
:10D7D00095F9CB6095F9CA501FE009B1A14206D175
:10D7E0006E4D2D6895F9CD6095F9CC5015E0002B64
:10D7F00018BF634504D001291CBF039DA94206D16F
:10D80000664D2D6895F9CF6095F9CE5005E0634DD2
:10D810002D6895F9C56095F9C45056EA050805D1FB
:10D820005E4D2D6895F9C56095F9C450B74201DC8D
:10D83000AF4218DA059D4FF00108EE69069D2E43B0
:10D84000049D2E60CD1701EBD5656F110E9E25F05E
:10D850001F0506EB870606F1140776694D1B08FACB
:10D8600005F535433D60491C8142FFF41FAE0D991B
:10D870005B1C8B42FFF4F1AD0FB00120BDE8F08FCF
:10D880002DE9F04F146889B015460E460746A1F100
:10D890002008202928BF4FF0FF3A05D24FF00100A1
:10D8A00000FA06F0A0F1010A38BF4FF0000B05D3D3
:10D8B0004FF0010000FA08F0A0F1010B202F3DBF4E
:10D8C0000120B840401E4FF0FF3038BF002207D380
:10D8D000A7F120024FF0010101FA02F1A1F10102CA
:10D8E000C6F12009202E34BF20FA09F100FA08F110
:10D8F000B2401143B040CDE90001206920F4FE6040
:10D9000020612748406810F0010F71D010F4807F2B
:10D9100005D02A463146384601F0AFFA78E010F4D7
:10D92000007F2A463146384602D0FFF709FD6FE0F6
:10D9300001F08FF90020A8616861002F84BFDFF833
:10D940005CE001221BD905EB4001B1F98C100029E4
:10D95000B8BF494209B2DEF80030B3F938308B4223
:10D960000ADD410905EB810100F01F0C4B6902FA49
:10D970000CFC43EA0C034B61401CB842E3D300208B
:10D98000012F18BFA7F1010E42D005EB4001B1F9FC
:10D990008E30B1F98C20991A04E000006C860010DA
:10D9A0005086001048BFD11A09B2DFF880C4DCF8F5
:10D9B00000C0BCF932C08C4527DAB5F9DC10B2EBF7
:10D9C000010C48BFA1EB020C0FFA8CFC5A1A48BF9D
:10D9D000CA1A11B28C450CDB420905EB820100F03A
:10D9E0001F0C01224B6902FA0CF21A434A610CE047
:10D9F00021E0411C4B0905EB830201F01F0C0121C2
:10DA0000536901FA0CF119435161401C7045BCD3B4
:10DA10006969E869B14008432063A969286AB1408F
:10DA2000084360636969202E34BF21FA09F101FAC5
:10DA300008F108436063FE484068079010F0040F47
:10DA400000F0B88100202863E862002E88BFDFF86C
:10DA5000DCE31BD9DEF8002005EB4001B1F95211DF
:10DA6000B2F95C308B4203DCB2F95E208A420ADAFA
:10DA7000420905EB820100F01F0C0122CB6A02FA79
:10DA80000CF21A43CA62401CB042E3D30020A862E1
:10DA90006862002F88BFDFF894E31BD9DEF800200E
:10DAA00005EB4001B1F98212B2F95C308B4203DC24
:10DAB000B2F95E208A420ADA420905EB820100F0DF
:10DAC0001F0C01224B6A02FA0CF21A434A62401CF4
:10DAD000B842E3D300202864E863002E88BFDFF853
:10DAE0004CE31BD9DEF8002005EB4001B1F99E1193
:10DAF000B2F960308B4203DCB2F962208A420ADA62
:10DB0000420905EB820100F01F0C0122CB6B02FAE7
:10DB10000CF21A43CA63401CB042E3D30020A8634E
:10DB20006863002F88BFDFF804E31BD9DEF800200C
:10DB300005EB4001B1F9CE12B2F960308B4203DC43
:10DB4000B2F962208A420ADA420905EB820100F04A
:10DB50001F0C01224B6B02FA0CF21A434A63401C61
:10DB6000B842E3D300202865E864A8646864002E06
:10DB700088BFDFF8B8E21CD9DEF8003005EB4001C1
:10DB8000B1F9EA11B3F964208A4203DCB3F96620E3
:10DB90008A420BDA410905EB810C00F01F030121D9
:10DBA000DCF84C2099401143CCF84C10401CB0429A
:10DBB000E2D30020002F88BFDFF870E21BD9DEF827
:10DBC000002005EB4001B1F91A13B2F964308B4221
:10DBD00003DCB2F966208A420ADA420905EB8201C7
:10DBE00000F01F0C01224B6C02FA0CF21A434A643B
:10DBF000401CB842E3D3696AE86AB14040EA010ECA
:10DC0000C4F838E0A96A286BB1400843E063696A48
:10DC1000202E34BF21FA09F101FA08F141EA00008F
:10DC2000E0630590696BE86B01FA06F140EA0102D6
:10DC30002264A96B286C01FA06F140EA01006064D5
:10DC4000696B34BF21FA09F101FA08F141EA0001D8
:10DC500061646B6CE86C03FA06F340EA0300A064AD
:10DC60000490AB6C286D03FA06F340EA0300E0640D
:10DC70006B6C34BF23FA09F303FA08F343EA00009C
:10DC8000E0640290059832EA0E0521EA000C4EEAA3
:10DC900005022564069240EA0C00C4F844C006EB75
:10DCA0000701039008BFBCF1000F43D000231A46C0
:10DCB0001846002988BF01273CD94FEA501804EBC9
:10DCC000880800F01F09D8F8408007FA09F918EA17
:10DCD000090F03D0864294BF521C5B1C401C81423A
:10DCE000EBD8012B0FD105EA0A0040EA0E00A06331
:10DCF00005980CEA0B031843E06325EA0A00206448
:10DD00002CEA0B006064012A14D1226C009802EA0C
:10DD10000003A06B1843A063606C019BD4F83CC067
:10DD2000034043EA0C03E363009B9A432264019A95
:10DD300090436064069A049830EA0202A26406984E
:10DD400040EA020CDDE9020320EA0300E064039BE1
:10DD500043EA000508BF002821D000231A461846D0
:10DD6000002988BF012717D94FEA501804EB88080B
:10DD700000F01F09D8F8488007FA09F918EA090FD6
:10DD800003D0864294BF521C5B1C401C8142EBD8DE
:10DD9000002B18BF002A02D10020A064E06407987D
:10DDA00010F0010F06D0206B20EA0C002063606B9E
:10DDB000A8436063206B0099084203D1626B01990C
:10DDC0000A4203D0216941F01001216110EA0A0FD3
:10DDD00004BF606B10EA0B0F03D0206940F02000F5
:10DDE0002061A06B0099084203D1E26B01990A42BD
:10DDF00003D0216941F04001216110EA0A0F04BFFC
:10DE0000E06B10EA0B0F03D0206940F08000206126
:10DE1000206C0099084203D1626C01990A4203D038
:10DE2000216941F48071216104E000006C860010DA
:10DE30005086001010EA0A0F04BF606C10EA0B0F46
:10DE400003D0206940F400702061A06C002804BF5A
:10DE5000E06C002803D0206940F48060206109B0A4
:10DE60000120BDE8F08F2DE9F04FC7B016460D46F2
:10DE70000446F3F7DBFFF3F762F901004FF01100FE
:10DE80001DBF049001200590012108BFCDE90410B9
:10DE9000CDE93C54F4F7B9FA0022002D88BF23A93C
:10DEA00004D9835C8B54521C9542FAD8F4F7AFFA2C
:10DEB0000021002C88BF23AA07D9435C02EB010C88
:10DEC000491C8CF826308C42F7D8F4F783F943903C
:10DED000FE48007910F0200F67D0F3F730F9FC49C5
:10DEE000FC4A00280CBFCDE90021CDE9001206F163
:10DEF000DE00029028300025EA460DF108090DF1F8
:10DF0000F00B039004A85BF8257050F82500F4F797
:10DF10009CFD0024002F1FD905EB450000EB0510E8
:10DF200023A901EB400818F90400262828BF002087
:10DF30000BD2C10700EBD070890C401001EB8000C0
:10DF40005AF825104058F4F786FD59F8251021F8A5
:10DF50001400641CBC42E6D36D1C022DD2D3DE4CEF
:10DF600025781D2D21D100210A4606AF5BF822C07D
:10DF70000020BCF1000F88BF59F8223007D933F8D0
:10DF8000108027F81180401C491C8445F7D8521C8A
:10DF9000022AEBD31D2D08D13846FDF7D3FB20789C
:10DFA0001D2804BF06A8FDF7CDFBC84D287910F049
:10DFB0000C0F00F05583F3F7C2F8C849C84A00288F
:10DFC0000CBFCDE90E21CDE90E12C648F3F7D9FFFB
:10DFD0000120F3F73CFB1B900120F3F795FB199010
:10DFE0000120F3F79BFE15900498F3F7C2FB1E90F7
:10DFF0000598F3F7BEFB1C900498F3F72FFC1A90DA
:10E000000598F3F72BFC18900498F3F767FC16902B
:10E010000598F3F763FC14900498F2F7F9FC12905A
:10E020000598F2F7F5FC10903EA906A840AACDE9A4
:10E03000000102920AAB08AA0CA90498F3F792FD1A
:10E0400007AA009241A93FA8CDE901010BAB09AA9B
:10E050000DA90598F3F786FD0498F3F722FE429088
:10E060000498F3F71EFEA04C03902068B0F8481007
:10E070000120F3F7FCFA00210120F3F737FE2068B6
:10E0800090F84A100498F3F786FB206890F84A103D
:10E090000598F3F780FB00210498F3F7F8FB0021C3
:10E0A0000598F3F7F4FB00210498F3F730FC002106
:10E0B0000598F3F72CFC01210498F2F791FC01215B
:10E0C0000598F2F78DFC2068B0F84C100498F3F72F
:10E0D00096FD2068B0F84C100598F3F790FD0021EC
:10E0E0000120F3F730FE17907848007910F0040F04
:10E0F00000F09681206890F84B3090F85920B0F8E5
:10E1000050100091CDE9012390F84F3090F84E2047
:10E1100090F858100498F3F7E5FC206890F84B301D
:10E1200090F85920B0F850100091CDE9012390F8F3
:10E130004F3090F84E2090F858100598F3F7D2FC25
:10E1400000210120F3F7FFFD36ADF4F7ABF8FCF743
:10E1500042FD012806D02846F4F7EDFA00287DD0CC
:10E16000F4F731FBF3F762FE3A9900223CAD002050
:10E1700055F822C0BCF1000F0ED902EB420303EBAD
:10E18000021306EB031331F8027B03EB4008401C3B
:10E19000A8F852718445F6D8521C022AE7D3049895
:10E1A000F2F70CFC44900598F2F708FC119000215E
:10E1B0000498F3F741FB469001210498F3F73CFBE8
:10E1C000139000210598F3F737FB22900121059861
:10E1D000F3F732FB444C2090206890F84B3090F8D5
:10E1E0005920B0F852100091CDE9012390F84F303A
:10E1F00090F84E2090F858100498F3F773FC2068BC
:10E2000090F84B3090F85920B0F852100091CDE9B9
:10E21000012390F84F3090F84E2090F85810059850
:10E22000F3F760FC00240DF1100B00210120F3F73F
:10E230008AFD00210498F2F7A9FB00210598F2F766
:10E24000A5FB5BF824000121F2F7A0FB3CA8002508
:10E2500050F824900EA850F8240000E01FE0019030
:10E26000B9F1000F5FD904EB440000EB041023A9BF
:10E2700001EB400106EB001A0091009800221146C4
:10E2800010F905801046F3F76CFDB8F1200F09DB9B
:10E290000027A8F12001012000FA01F807E0F7F7B4
:10E2A00045FE54E7012000FA08F74FF000085BF83C
:10E2B00024003A460021F3F7ADFA5BF82400424609
:10E2C0000121F3F7A7FA6FEA08020FE05086001069
:10E2D000B09D0030189D003073850010CC0E0030CA
:10E2E000CC09003001000E006C860010F9430920B3
:10E2F000F3F737FD36AFF3F7D5FFFCF76CFC0128D9
:10E3000006D03846F4F717FA00287CD0F4F75BFA09
:10E31000F3F78CFD019800880AEB45016D1CA1F80C
:10E320009E014D45A9D3002211461046F3F719FD71
:10E33000641C022CFFF479AF44990498F2F726FB91
:10E3400011990598F2F722FB0021469A0498F3F7F9
:10E3500061FA0121139A0498F3F75CFA0021229ADA
:10E360000598F3F757FA0121209A0598F3F752FA26
:10E37000FE4C206890F84B3090F85920B0F85410BB
:10E380000091CDE9012390F84F3090F84E2090F89D
:10E3900058100498F3F7A6FB206890F84B3090F8DB
:10E3A0005920B0F854100091CDE9012390F84F3076
:10E3B00090F84E2090F858100598F3F793FB012140
:10E3C0000846F3F7C0FC36ACF3F76CFFFCF703FC30
:10E3D000012806D02046F4F7AEF900287DD0F4F7E6
:10E3E000F2F9F3F723FD3A9900223CAC002054F8EF
:10E3F00022C0BCF1000F10D902EB420303EB021361
:10E4000006EB031300E065E031F8025B03EB400725
:10E41000401CA7F8EA518445F4D8521C022AE5D3DF
:10E42000D348007910F0080F7ED0D04D286890F8BE
:10E430004B3090F85920B0F856100091CDE90123E7
:10E4400090F84F3090F84E2090F858100498F3F759
:10E4500049FB286890F84B3090F85920B0F85610D6
:10E460000091CDE9012390F84F3090F84E2090F8BC
:10E4700058100598F3F736FB00210A463CAF002000
:10E4800057F82130002B0CD901EB410C0CEB011C8F
:10E4900006EB0C1C0CEB4004401CA4F83622834213
:10E4A000F8D8491C0229EAD32868002490F86800AB
:10E4B000B4EB400F38DA286890F86800A042D4BF67
:10E4C000012100210120F3F73EFC36AFF3F7EAFE0D
:10E4D00006E002E0F7F72AFD0FE7F7F727FD75E7FB
:10E4E000FCF779FB012805D03846F4F724F9E0B3AE
:10E4F000F4F769F9F3F79AFC3A994FF000090DF136
:10E50000F00E00225EF829701046002F05D931F96F
:10E510001030401C1A448742F9D8B2FBF7F2781E3B
:10E520003FD009EB490300E04AE003EB091306EB97
:10E53000031A31F9103001EB400C3CF9028CB3EBBB
:10E54000080348BF5B4231F91080B8EB020831F98B
:10E5500010804CBFA2EB0808A8EB02083CF902BCF3
:10E560003CF902CCBBEB020B00E00FE04CBFA2EB8E
:10E570000C0CACEB020CE0450AEB400C09DDBCF9DD
:10E5800036824345C8BFACF8363208E0F7F7CEFC18
:10E59000A6E7BCF934829845B8BFACF83432401EC7
:10E5A000C7D109F1010901EB4701B9F1020FA8D365
:10E5B0002868641C90F86800B4EB400FFFF67BAF4E
:10E5C00001201B99F3F753F801201999F3F7A7F8E5
:10E5D00001201599F3F78AFB1E990498F3F7DBF8ED
:10E5E0001C990598F3F7D7F81A990498F3F74FF99F
:10E5F00018990598F3F74BF916990498F3F787F9EA
:10E6000014990598F3F783F912990498F2F7E8F949
:10E6100010990598F2F7E4F93E990698409ACDE9E9
:10E62000000102920A9B089A0C990498F3F75AFA8F
:10E63000419A07983F990292CDE900010B9B099AF4
:10E640000D990598F3F74EFA42990498F3F7D7FA23
:10E6500003990598F3F7D3FA01201799F3F773FBA1
:10E660004398F3F78EFC47B0BDE8F08F4049012096
:10E670008860FDF799BB3E490020886070472DE90E
:10E68000F04F3B4EADF5737D0125B560FDF78CFB7A
:10E6900070684FF4407131EA000004BF0020F1902F
:10E6A00000F0AC821D20FCF7A5FD07461D20FDF7FC
:10E6B0002FF82F4EED904FF46D716846F4680DF011
:10E6C000FAFF0094B08810F4804F1CBF2046FEF77C
:10E6D0001CFC6A46009890F8203090F821C0503019
:10E6E0000CFB03F100EB41000021BCF1000F08D945
:10E6F00002EB410930F8028B491CA9F8DE808C45F9
:10E70000F6D80021002B08D902EB410930F8028B22
:10E71000491CA9F806818B42F6D80021BCF1000FF4
:10E7200008D902EB410930F8028B491CA9F8648032
:10E730008C45F6D80021002B08D902EB410930F8AE
:10E74000028B491CA9F88C808B42F6D830F8021B4A
:10E75000A2F8DA1030F8021BA2F8DC1030F8021B25
:10E76000A2F8D8104FF00008002103E06C860010DA
:10E7700050860010BCF1000F0ED908EB480909EBD8
:10E78000081902EB890909EB410B30F802AB491C6F
:10E79000ABF852A16145F6D30021002B0ED908EB4E
:10E7A000480909EB081902EB890909EB410B30F81C
:10E7B00002AB491CABF882A29942F6D308F10108DA
:10E7C000B8F1040FD0D361461846FEF787FC01204C
:10E7D000F190706810F4004F03D1694600F06DFDB0
:10E7E000F1903846FCF706FDED98FCF791FF94F8A0
:10E7F0002000EF9094F82100F090F19800281FBFBE
:10E80000EF980028F098002800F0F881FE48406852
:10E81000F29010F0020F00F00F81009DDDE9EF276C
:10E8200028696E4620F00F00286147F6FF706FEAF6
:10E830000009ED90002005F150080490039002902B
:10E8400082460190002F54D90AFB02F04FF0010CD0
:10E8500038F9101000208B465B46EE90012A1BD938
:10E860000AFB02C038F910009842C8BF034688422C
:10E87000B8BF0146B0EB0B0E48BFABEB000E0FFA72
:10E880008EFBDDF8B8E3F345C8BFCDF8B8B38346D7
:10E890000CF1010C9445E3D34B45C8BF9946ED9864
:10E8A0008142B8BFED91581A48BFC81A01B2D74883
:10E8B0000068B0F91C308B4204DBB0F91E10EE98F2
:10E8C000884212DD4FEAEA700AEBD060411106EB94
:10E8D000810120F01F0001F10C03AAEB000CC968B4
:10E8E000012000FA0CF0084318600AF1010ABA4549
:10E8F000AAD34FF0000A002A51D938F91A00002192
:10E9000083465B464FF0010CEE91012F1BD90CFBA7
:10E9100002A138F911109942C8BF0B468142B8BF15
:10E920000846B1EB0B0E48BFABEB010E0FFA8EFBA6
:10E93000DDF8B8E3F345C8BFCDF8B8B38B460CF1AA
:10E94000010CBC45E3D34B45C8BF9946ED998842BD
:10E95000B8BFED90191A48BFC11A09B2AB48006898
:10E96000B0F920308B4204DBB0F92210EE988842D7
:10E9700011DD4FEAEA700AEBD060411106EB81012C
:10E9800020F01F000B1DAAEB000C4968012000FAC3
:10E990000CF0084318600AF1010A9245ADD3F06803
:10E9A000002804BF3069002803D0286940F008001F
:10E9B00028617068002804BFB068002803D0286967
:10E9C00040F0040028617168F068B9400843A8620B
:10E9D000B1683069B9400143E9627068202F39BFDE
:10E9E000C7F12002D040A7F1200290400843E8621E
:10E9F000ED98A884A5F82690B6F9D810B9EB0100D7
:10EA000048BFA1EB090081490968B1F9182090427B
:10EA100003DD286940F002002861B6F9D820ED989E
:10EA2000101A44BFED98801AB1F91A10884203DD1C
:10EA3000286940F001002861F298734D10F0050F2D
:10EA400004D0DDE9EF016A46FEF71AFFD5F804A00D
:10EA50001AF0080F7CD0009ADDE9EF9311694FF0AE
:10EA6000000B21F4C05111616846CDF860B05946E1
:10EA7000CDF85CB0002B84BFDFF890E101261AD9F5
:10EA8000DEF8007000EB410CBCF936C2B7F96A70D1
:10EA900067450DDA4FEA511C00EB8C0C01F01F08A2
:10EAA000DCF85C7006FA08F847EA0807CCF85C70F6
:10EAB000491C9942E4D3C0F858B00021C0F854B0C2
:10EAC000B9F1000F84BF514E01271AD9D6F8008042
:10EAD00000EB410CBCF966C3B8F96A80E0450DDA79
:10EAE0004FEA511800EB880C01F01F0BDCF8548042
:10EAF00007FA0BFB48EA0B08CCF85480491C49453F
:10EB0000E4D3916BD0F85CC041EA0C01D0F854C05A
:10EB10000CFA03FC41EA0C019163D16BD0F860C0A0
:10EB200041EA0C01D0F858C00CFA03FC41EA0C0C85
:10EB3000C2F83CC0416D202B39BFC3F12003D9403E
:10EB4000203B994041EA0C01D163416D002900E06E
:10EB500011E004BF816D002903D0116941F4006107
:10EB60001161C16D002904BF006E002803D0106937
:10EB700040F4805010611AF0400F0FD16069401CC2
:10EB800060612069002814BFE069A06900F10100FC
:10EB900014BFE061A0616846FEF71BFA0020E06048
:10EBA000A36821460246A446B3F5056F88BF4FF41B
:10EBB00005630020B0EB930F06D25CF82070401C78
:10EBC0003A44B0EB930FF8D35042C860287910F064
:10EBD000800F05D14FF440304FF40562F4F7BCFAD2
:10EBE000F7F73FF9411E022908D8A98811F4007FE0
:10EBF00004D0024603212046FEF794F841208DF808
:10EC0000B403F198E8B103E0508600106C86001060
:10EC1000207C8DF8B503607C8DF8B603A07C8DF860
:10EC2000B703E07C8DF8B80300230522EDA9072087
:10EC300000F073FDFE49002088600DF5737DBDE88E
:10EC4000F08FFF208DF8B5038DF8B6038DF8B7036C
:10EC5000E8E72DE9F74F84B04FF00008C2F82080B4
:10EC6000C2F81C80059BF34E01274146002B1ED99C
:10EC700002EB4103B3F96430002BB8BF5B421BB217
:10EC8000D6F800C0BCF938C09C450CDD4B0902EB3E
:10EC9000830301F01F04D3F81CC007FA04F44CEA04
:10ECA000040CC3F81CC0059B491C9942E0D3002109
:10ECB000012B1CBF059BA3F1010940D002EB4103CE
:10ECC000B3F96640B3F964C0B4EB0C0348BFACEBD6
:10ECD00004031BB23568B5F930509D422CDAB2F905
:10ECE000DA30BCEB030548BFA3EB0C052DB2B4EB47
:10ECF000030C48BFA3EB040C0FFA8CF39D420DDB11
:10ED00004B0902EB830301F01F04D3F81CC007FA80
:10ED100004F44CEA040CC3F81CC00DE04B1C4FEA91
:10ED2000531C02EB8C0C03F01F03DCF81C4007FAA9
:10ED300003F32343CCF81C30491C4945BED331684A
:10ED400091F83630002B7DD091F8371014688B4243
:10ED500088BF19460023DDF814C0BCF1000F84BF42
:10ED6000491C00916ED94FF0010EDDF800C04FF044
:10ED700000090121CA46BCF1010F52D9DFF8B4C223
:10ED800003FB0005DCF800C0CDF80CC0BCF93AC0AC
:10ED900002950EFB0005019503FB001504EB4505EC
:10EDA000B5F95080B8F1000FB4BFC8F10005454671
:10EDB000AC4536DB0EFB001504EB4505B5F950708C
:10EDC000002FB4BF7D423D46AC452ADB029D6D1A43
:10EDD00004EB4505B5F94E60002EB4BF75423546CB
:10EDE000AC451EDB019D6D1A04EB4505B5F94E508F
:10EDF000002DB4BFC5F1000BAB46E34511DCA7EB1A
:10EE00000808039FB7F934704745B8BF09F10109F5
:10EE1000AD1BBD42C8BF0AF1010A491C009DA942B1
:10EE2000BAD3BAEB090148BFA9EB0A01DFF804C263
:10EE3000DCF800C09CF836C061450FDB590902EBD5
:10EE4000810100E015E003F01F064FF0010CCD69D1
:10EE50000CFA06FC45EA0C0CC1F81CC005995B1CB9
:10EE60008B4206D2002B18BFA3F1010E7FF47DAFB9
:10EE700079E707B00120BDE8F08F2DE9F04F0023BE
:10EE800088B017681362D36193615361DFF8A8B14A
:10EE9000DFF8A0E147F6FF7A0093019302939C46C6
:10EEA000A1F10109A0F10108039300296FD9002302
:10EEB000002868D94FEAEC740CEBD46424F01F05E9
:10EEC000ACEB0505012606FA05F5641102EB840496
:10EED000CDE906451C3405940CFB003407EB4404D3
:10EEE000BCF1010FB4F9504014D81E2B0FDB1F2BBF
:10EEF0000DDCDEF80050BCF1000F19BFB5F99E60C3
:10EF0000B5F99C50B5F99660B5F9945010E0BCF194
:10EF1000000F02D0CC4540F0DA80002B18BF4345EB
:10EF200040F0D580DEF80050B5F99260B5F9905008
:10EF3000002E04BFDEF80060B6F98A60002D04BF21
:10EF4000DEF80050B5F98850B44201DCAC4217DA63
:10EF5000069CE569079C2543059C2560DC1703EBAF
:10EF6000D4656C1102EB840404F11406049625F0B8
:10EF70001F055E1B0125B5406469049E2C43346067
:10EF80005B1C8342A8D30CF1010C8C458FD3DEF8B7
:10EF90000030B3F88E30002B1CBFABEB0A0C9C4545
:10EFA00034DD039BDDF80CC05B0902EB83030CF03E
:10EFB0001F05DC694FF0010C0CFA05F52C43DC61F0
:10EFC000019B019C5B0902EB830304F01F04DD69D4
:10EFD0000CFA04F42C43DC61029B029C5B0902EBFB
:10EFE000830304F01F045D690CFA04F42C435C6194
:10EFF000009B009C5B0902EB830304F01F045D6926
:10F000000CFA04FC45EA0C0CC3F814C0094B1B684D
:10F0100093F88C30002B00F04C814FF0000C00284E
:10F020007ED98B1E034E4FF0010E039306E00000C5
:10F03000508600106C8600100080FFFF07EB4C0329
:10F04000B3F950500023B9F1000F6AD94FEAEC74BC
:10F050000CEBD46424F01F0AACEB0A0A0EFA0AFA8D
:10F06000641102EB8404CDE9014A143400945C1C61
:10F0700004FB00C407EB4404B4F95040002CC8BFA3
:10F08000002D6BDDB4EB050A48BFA5EB040AAC42CA
:10F09000C8BF25464FF4484B0AFB0BFA9AFBF5F51F
:10F0A00005F2FF154FEA552A012B22D8BCF11E0F9D
:10F0B0001EDBBCF11F0F1BDC002B08BFBCF11F0FB8
:10F0C000356814BF95F89A5095F899501FE0DEF80E
:10F0D00000505C45B5F98A60B5F98850C4BFA346B5
:10F0E000CDE9023C5445BCBFA246CDE9003C1FE738
:10F0F00013B1039DAB4207D1BCF1000F12BFC44551
:10F10000356895F88D5002D0356895F88C50002DF3
:10F1100004BF356895F88C50AA451FDDDD1701E066
:10F1200025E01FE003EBD56B4FEA6B1502EB85057D
:10F1300005F11C0A2BF01F0BED69A3EB0B0B0EFA6C
:10F140000BFB45EA0B05CAF80050019DD5F814A049
:10F15000029D4AEA050A009DC5F800A05B1C2546F1
:10F160004B4584D30CF1010C8445FFF45FAF4FF0A5
:10F17000000C002984BF861EDFF85CA47DD90CFB3F
:10F1800000F307EB4303B3F950500023B8F1000F2D
:10F1900074D94FEAEC740CEBD46424F01F0BACEB85
:10F1A0000B0B4FF0010E0EFA0BFB641102EB840403
:10F1B000CDE9024B1C3401940CFB003407EB4404F2
:10F1C000B4F95240002CC8BF002D69DDB4EB050B2B
:10F1D00048BFA5EB040BAC42C8BF25464FF4484ED0
:10F1E0000BFB0EFB9BFBF5F505F2FF154FEA552BCC
:10F1F000BCF1010F03D0BCF1000F05D00BE0A3F16F
:10F200001D05012D02D906E01E2B06D1DAF80050AB
:10F2100095F89A5016E0CC4508D1002B12BFB342A6
:10F22000DAF8005095F88D500CD000E033B1B342BD
:10F230001CBFDAF8005095F88C5003D1DAF8005072
:10F2400095F89850002D04BFDAF8005095F88C50CE
:10F25000AB4525DD029DD5F81CB0039D4BEA050B9F
:10F26000019DC5F800B0DD1703EBD56B4FEA6B15B8
:10F2700002EB850505F1140E01E01AE014E0CDF86B
:10F2800000E02BF01F0BA3EB0B0E4FF0010B0BFA62
:10F290000EFB6D69DDF800E045EA0B05CEF8005085
:10F2A0005B1C2546434587D30CF1010C8C45FFF4CC
:10F2B00066AF08B00120BDE8F08F2DE9F04F04469D
:10F2C000C64887B00F460068002590F8E40000F0BB
:10F2D0000F0600F0CDFA01280AD00F213046F6F7CC
:10F2E00047FF012813D0002000F0BFFA00F070B9EA
:10F2F00000210846F2F768FEF1F707FF50B1B84861
:10F30000D0F8401341F48031C0F8401302E00120EE
:10F3100000F0ABFAB34890F80080B34890F8009042
:10F32000B9F1000F18BFB8F1000F00F04F81386835
:10F33000002180F8208080F8219080F8221080F849
:10F340002310F3F7D8FBF2F745FF8346002014F0B3
:10F35000030F18BF4FF4817014F0200F1CBF40F250
:10F36000012108439C4E00287ED000EA0B0014F4D3
:10F37000407F18BF40F42020F2F703FE0020F8F78A
:10F38000BAF960F30F0500210846F8F7ABF9012040
:10F39000F8F7B1F960F31F4500210120F8F7A2F951
:10F3A0000020F2F754F905900020F2F7ADF904902F
:10F3B0000020F2F7DEF903900020F2F74FFA0290F6
:10F3C0000020F2F78BFA0190F2F714FC14F4807F1E
:10F3D0004FF0FF3A009027D03068B0F88410002931
:10F3E0001CBF0020F2F743F9306890F8861000291E
:10F3F0001CBF0020F2F7CFF9306890F8870010F0BA
:10F400000F0F05D000F00F00411E0020F2F73FFA69
:10F41000306890F8870010F0F00F34D00AEB10112C
:10F420000020F2F774FA2EE014F4007F2BD030683D
:10F43000B0F8A01000291CBF0020F2F718F93068BE
:10F4400090F8A21000291CBF0020F2F7A4F9306840
:10F4500090F8A30010F00F0F05D000F00F00411E30
:10F460000020F2F714FA00E035E0306890F8A300CD
:10F4700010F0F00F04D00AEB10110020F2F747FA59
:10F480000020F2F7ADFBFF210F20F7F76DFBF2F73D
:10F49000CDFC00200599F2F7EAF800200499F2F774
:10F4A0003EF900200399F2F776F900200299F2F76D
:10F4B000EEF900200199F2F72AFA0098F2F790FB92
:10F4C00029B20020F8F70EF929140120F8F70AF9FB
:10F4D0005846F2F756FD14F02C0F04D03A46494630
:10F4E0004046FEF7C0FC14F0030F6ED00097D7F82B
:10F4F00000A00AF15005F2F78AFF8346F2F796FC66
:10F500003A4CA08810F4407F03D00020F2F731F984
:10F5100001903648406810F4807F04D0306890F83D
:10F52000861051B106E010F4007F06D0306890F8E4
:10F53000A21011B10020F2F72EF90020F3F785FA9E
:10F540000026B9F1000F23D906EB4600002400EB9A
:10F55000061716E01BF90400262811D2C107890CF2
:10F5600000EBD07001EB8701401001EB800000F14F
:10F57000405000F500400068F3F76DFA25F8020BE3
:10F58000641C444538BF262CE4D3761C4E45DBD39F
:10F590001648808810F4407F03D000200199F2F7CC
:10F5A000FAF8134C20781D280AD10AF15000FBF715
:10F5B00032FF20781D2804BF0AF15000FBF72BFF13
:10F5C00049464046009AFDF789FD0125F2F7C3FD43
:10F5D00007B02846BDE8F08F6C8600104886001002
:10F5E00000500040E9840010EA84001050860010AA
:10F5F0006D85001070474FF0FF30704789484068B4
:10F60000704788494860704710B582B007280BD111
:10F610004FEA111C012404FA0CFC824C64681CEAB9
:10F62000040F04BF02B010BD9B0100F00F0043EABD
:10F63000800040F001008DF800008DF801108DF879
:10F640000220100A8DF80300100C8DF80400100E33
:10F650008DF8050000208DF806008DF8070068463B
:10F660000DF01FF802B010BD2DE9F04F0E464FF01F
:10F67000000183B05FEA020800914FF001024FF0F1
:10F6800002070D460C46019104BF03B0BDE8F08FA0
:10F69000EB467B0100F0070943EA890040F0030ACA
:10F6A00016F814000BF80200501C36F81420C0B2F3
:10F6B000120A0BF80020401CC2B2481CC1B2B94269
:10F6C0000ED1681C85B28DF800A0FF2D94BF28468E
:10F6D000FF208DF8050068460CF0E3FF00210122B1
:10F6E000601C84B24445DBD3002904BF03B0BDE8ED
:10F6F000F08F480140EA890040F003008DF80000D7
:10F70000681C80B2FF2888BFFF208DF8050068467E
:10F710000CF0C7FF03B0BDE8F08F10B582B007282A
:10F720000DD191F800C001244FEA1C1C04FA0CFC16
:10F730003C4C64681CEA040F04BF02B010BD9B017E
:10F7400000F00F0043EA800040F001008DF8000057
:10F75000072A88BF072200206B46002A09D911F822
:10F7600000C01C18401C84F801C09042F7D3072841
:10F7700005D200211A18401C51700728FAD31846E8
:10F780000CF08FFF02B010BD10B59B0100F00F0010
:10F7900082B043EA800040F002008DF80000072AA2
:10F7A00088BF072200206B46002A09D911F800C043
:10F7B0001C18401C84F801C09042F7D3072805D2DA
:10F7C00000211A18401C51700728FAD318460CF073
:10F7D00068FF02B010BD70B5124E40EA0125022844
:10F7E0003488224618BF052803D1002918BF0229F2
:10F7F00000D12C46A24209D051B17088002344EABE
:10F80000004290210720FFF7FFFE3480758070BD15
:10F81000F4F7A7F844EA0042002390210720FFF7FD
:10F82000F3FEF2E760860010FE4908707047FD485D
:10F830000078704710B50446FDF703F80146D02262
:10F8400020460CF033FFF748446010BD58B1F64A2B
:10F850000168914207D1406820F00F00B0F5807F29
:10F8600004BF0120704700207047EE494870704780
:10F87000EC484078704710B5EC48EA4C86B0006818
:10F880006178808F0429C0F3032008D0E849F6F797
:10F890006FFC01281CBF002060700FD044E00021E5
:10F8A0000846F2F791FBF1F730FC88B1E148D0F857
:10F8B000401341F48031C0F8401309E00420607027
:10F8C00005210020F1F7D3FE00210846F2F794F855
:10F8D000FF210F20F7F748F90CF060FF0CF063FFF1
:10F8E0000020F5F70DF9F1F710FC10F0010F04BF3F
:10F8F0000120F1F79DFEF2F781FCFBF76CF901287E
:10F900000CD06846F2F717FF28B16846FCF748F8B4
:10F91000F2F759FFF1E7F6F709FBEEE7F2F786FA9F
:10F920000CF041FF0CF044FFF2F715FC06B010BDDF
:10F930002DE9F05FBD48BB4EADF5865D0068D0F89F
:10F940003CC07078CCF30322022828D0B0680F2185
:10F9500010F4007F1EBFCCF303330F2B1A4610F0B8
:10F96000800F1EBFCCF303130F2B1A4610F0040FA9
:10F9700008BF0B2110F0020F08BF21F0020110F0A8
:10F98000010F08BF21F001011046F6F7F1FB012835
:10F9900014BF00200220707040F065840DE000214B
:10F9A0000846F2F711FBF1F7B0FB30B1A148D0F8EF
:10F9B000401341F48031C0F84013F2F70BFC0D9076
:10F9C000307A10F0100F18BFF3F75DF8307A10F0AE
:10F9D000080F03D1FF210F20F7F7C6F896480078EB
:10F9E0000190964800780A909548077895480078E5
:10F9F00008900A9800281CBF019800281AD00CF023
:10FA0000CDFE0CF0D0FEB06810F4803F04BF0020A3
:10FA1000F5F776F8B06810F4003F04BF0020F5F762
:10FA2000A8F8307A10F0100F0BD00120F5F7AFF8DE
:10FA300001200AE00898002818BF002FDFD100F04D
:10FA400012BC0020F5F7A3F80020F5F7A0F8B06885
:10FA500010F4803F18BFF4F7ECFFB06810F4003FDB
:10FA600018BFF5F775F80120F1F7E2FDF2F7C6FBD4
:10FA70001E20FBF7BFFB00210846FBF76BFB81460E
:10FA800001210020FBF766FBB468804614F4002FC8
:10FA900004D04FF4BE6114A80CF00DFE14F4800FD6
:10FAA00008D00DF5C8604FF4BE610C900CF06CFEF0
:10FAB00000200B9014F4000F05D041F2380074219F
:10FAC00068440CF0F8FD0A9A0199002001FB02FB42
:10FAD000BBF1000F84BF47F6FF71CA4306D929F86E
:10FAE000102028F81010401C8345F8D81E20FBF782
:10FAF0000FFE00210120FBF72DFB044601210846E3
:10FB0000FBF728FB05464748806810F4801F04D0A7
:10FB1000E8210DF575600CF0CEFD089900207E18E7
:10FB20001CBF47F6FF72D14306D024F8101025F809
:10FB30001020401C8642F8D83A484FF0000A40880E
:10FB4000002840F29C810198401E12900899701C78
:10FB50003944491E0F9108994008491E0E91711EA3
:10FB6000CDE91001FBF737F8012800F0888102A8E1
:10FB7000F2F7E1FD002800F07B810398F4F7D8FA52
:10FB8000049800284DD00CF027FE07462548007A3F
:10FB900010F0100F08D0384604990CF022FE09909E
:10FBA000B84208BF049F0DE00020002300901A46D1
:10FBB000194604980CF01AFE09901A48007A10F0C1
:10FBC000200F09D1F4F708FB0A9A00920146384643
:10FBD000019B099A0CF00FFE1248008910F4804F27
:10FBE0001EBF09980028F4F73DFB002F1CBF002022
:10FBF000BBF1000F60D90B49D1F808E037F91010BC
:10FC000039F910208A42B8BF29F8101038F91020AD
:10FC10008A42C8BF28F810101EF4002F29D014AA59
:10FC200012E049E068860010545354524886001090
:10FC300004000A0000500040E9840010EA8400102B
:10FC4000EE840010EF84001032F9102047F6FF7C9C
:10FC500053189C45DCBF14A921F810C009DD0DF133
:10FC6000500C13F5004FD4BF4FF4004111442CF851
:10FC700010101EF4800F1CD00199B0FBF1F201FBB3
:10FC8000120212998A4214D007EB400137F9103062
:10FC9000B1F90220991A48BFD11A0C9A32F91020F2
:10FCA0008A423CBF0C9A22F810100B9A914288BFEE
:10FCB0000B91401C8345A1D80D9810F0010F1CBF7B
:10FCC000069800287CD00CF01EFD0746F848806896
:10FCD00010F0400F05D00022114606980CF090FD60
:10FCE00010E010F4003F02D0F4F773FA01E0F4F7EB
:10FCF00038FA0222009201463846109B069A0CF010
:10FD00007AFD0698EA49098911F4005F1CBF0028B2
:10FD1000F4F731FA002F53D0E548826812F4806F6F
:10FD20002FD008990020012910D007EB400137F9A6
:10FD30001030B1F902C0BCEB030148BFA3EB0C01CA
:10FD400027F810100E99401C8842EED34FF0000E99
:10FD500027F810E00F99401C884210D207EB4001B1
:10FD600037F91030B1F902C0BCEB030148BFA3EB77
:10FD70000C0127F810100F99401C8142EED827F88B
:10FD800010E00020002E88BF0DF5756E36D937F9CA
:10FD9000101034F910308B42B8BF24F8101035F928
:10FDA00010308B42C8BF25F8101012F4801F04D009
:10FDB0005EF820C061444EF8201012F4000F00E0FD
:10FDC00051E01FBF0E9981421199814213D007EB78
:10FDD000400137F910C0B1F90230BCEB030148BF54
:10FDE000A3EB0C0141F2380CEC443CF910308B428F
:10FDF00038BF2CF81010401C8642C8D812F4806F0F
:10FE000031D0AC4A0AF10100A2FB00318908494215
:10FE100001EB8101C14226D1A2FB0A108008A2FB9E
:10FE200000210909494201EB810100EB810040F208
:10FE3000493141430DF5C86000EBC10C0020002E94
:10FE400084BF47F6FF73DA430DD934F8101035F844
:10FE50001070C91B2CF8101024F8102025F8103051
:10FE6000401C8642F1D8F2F7AEFC0AF1010A01E02B
:10FE7000F6F75CF88E4840888245FFF473AEF1F7E0
:10FE8000D5FF0CF090FC0CF093FC89484088019061
:10FE90008245C0F0E2810D9810F0020F7ED08649B5
:10FEA00000204A0C0990BBF1000F52D9804B9B688F
:10FEB000009339F910C038F91030009FACEB030EF5
:10FEC00017F4002F6BD00DF1500C47F6FF773CF97B
:10FED00010309F42D8BF2CF810700BDD13F5004F87
:10FEE000D1BF4FF40043019F03EB570393FBF7F39C
:10FEF0002CF810303CF910308B42C8BF19469342A1
:10FF0000B8BF1A4628F8103029F810E0009B13F407
:10FF1000800F05D00C9B33F810C0684B23F810C03D
:10FF2000DDF824C0E645C8BFCDF824E0401C834579
:10FF3000BFD8B1F5004FA8BF47F6FF7112F5004FCB
:10FF4000B8BF5D4A0998B0F5806FA4BF40F2FF309A
:10FF5000099042208DF80000080A8DF801008DF804
:10FF60000210100A8DF803008DF8042009988DF80E
:10FF70000500C02101EAA0008DF806000722002339
:10FF800069461046FFF7C9FB4948806810F4800FA6
:10FF900012D047208DF800000B9801E00CE05AE0E9
:10FFA000000A8DF801000B988DF80200002303224F
:10FFB00069460720FFF7B1FB0D9810F0010F00F024
:10FFC0004C813B4FD7F8088018F4806F79D03948BE
:10FFD0004FF00009A0FB0A108308142B88BF1423DC
:10FFE0004FF0000A5146002E4CD9981E0DF5C86BF3
:10FFF00000904FF0000C304F47F6FF786246002B20
:020000021000EC
:1000000015D902EB4200C0EB421001EB400000EBBF
:10001000400ECEEB40100BEB80008444B842C8BFCA
:1000200007464045B8BF8046521C9A42E9D3002B90
:1000300004BF002024F8110014D09CFBF3F024F836
:100040001100022B0ED9ACEB0700A0EB08020098C0
:1000500092FBF0F007E08C45C8BF61469342B8BF01
:100060001A4653E7002025F8110034F911005045D5
:10007000C8BF824635F911004845C8BF8146491CB2
:100080008E42B6D843208DF800004FEA1A208DF832
:1000900001008DF802A04FEA19208DF803008DF8B9
:1000A00004900023052269460720FFF736FBD4E0C1
:1000B00068860010CDCCCCCC0080FFFF1828011042
:1000C000FFE7A4490023DDF820C04A0C1846BCF124
:1000D000000F88BF0DF5756E40D934F910A035F9C1
:1000E000109018F4801FAAEB090C26D05EF820A00F
:1000F000B7F802900AEB590A9AFBF9F94EF82090EA
:100100008945C8BF49469145B8BF4A4625F8109071
:1001100018F4000F08BF24F810C017D041F2380CB3
:10012000EC443CF810C024F810C041F2380CEC4408
:100130003CF910C09C450CDD0AE08A45C8BF514619
:100140009145B8BF4A4618F4000FEED19C4500DD3A
:100150006346DDF820C0401C6045BED343208DF8C7
:100160000000080A8DF801008DF80210100A8DF8C1
:1001700003008DF80420C0208DF8053000EAA300AC
:100180008DF806000722002369461046FFF7C5FADE
:100190007049089800234A0CB04244D2DFF8B8C135
:1001A00041F23809E944DCF8088034F910B035F937
:1001B00010A0DFF8A4C1ABEB0A0718F4801F23D00E
:1001C0000DF5756ABCF802C05AF820B00BEB5C0B59
:1001D0009BFBFCFC4AF820C08C45C8BF6146944597
:1001E000B8BF624625F810C018F4000F1ABF39F8DE
:1001F00010C024F810C024F810700ED039F910C0C7
:100200009C45C8BF63460BE08B45C8BF5946924525
:10021000B8BF524618F4000FF0D19F42C8BF3B460A
:10022000401C8642C1D844208DF80000080A8DF891
:1002300001008DF80210100A8DF803008DF80420DB
:10024000C0208DF8053000EAA3008DF806000722D3
:10025000002369461046FFF760FAFF20FAF7CAFF4D
:10026000FF20FBF755FAF1F776FF0DF5865DBDE847
:10027000F09F70B5ADF5126D4FF0FF30FCF714FB39
:100280000DF50565FCF7DDFA0146D02228460CF095
:100290000DFA314C6560002565702846F2F7AFF81D
:1002A000F2F73CF80646FF224FF4056168460CF071
:1002B00020FA6846FCF741FE6846FCF7CCFDFAF7E9
:1002C0008AFC012803D1F5F7CFFD032827D1207838
:1002D00010F0010F07D0FEF7D2F9207820F00100CE
:1002E0002070FAF71DFC207810F0020F07D0FFF7FE
:1002F0001FFB207820F002002070FAF711FC207814
:1003000010F0040F07D0FFF7B6FA207820F00400B1
:100310002070FAF705FCF5F7A7FD03280CD00020A4
:10032000FCF799FD30466560F1F7EEFF0120F2F72A
:1003300066F80DF5126D70BDF5F7F8FDBFE70649DB
:100340008860002048707047034880687047024901
:10035000488070470080FFFF68860010F7490870EA
:100360007047F64800787047F44948717047F34881
:1003700040797047F148406AB0F5B47F2CBF012046
:1003800000207047ED4840787047EC49002280B16A
:10039000012818BF7047487802280CD0042818BFDD
:1003A000486A06D0B0F5B47F84BF4FF4B470486299
:1003B00070474A627047486A401C4862F2E7E0486A
:1003C00000787047DD48407910F0010F18BF704782
:1003D00010B50020DA490870F5F72BFEBDE8104093
:1003E0000020F4F7C0BBD6488088C0F300207047D7
:1003F000D34910B589880020C1F3002151B107F01D
:1004000023F964280FBF4FF0C040012101FA00F02A
:1004100040F08040BDE8104007F019B9C84A10B557
:1004200081B25160C54AC0F30743C0F303609361D2
:10043000507090700020C1F30021D06151B107F0DD
:1004400003F964280FBF4FF0C040012101FA00F00A
:1004500040F08040BDE8104007F0F9B8B74890F987
:100460000C007047B548407B7047B448807B7047AC
:10047000B34A0028516814BF41F0020021F0020085
:1004800050607047AE480079C0F340007047AC4AF6
:1004900010F0010F506814BF40F0020020F002007D
:1004A00050607047A64900200979C1F34001002936
:1004B00018BF012070470028A14A516814BF41F0BD
:1004C000010021F00100506070479D48007900F064
:1004D0000100704799494A788A7048707047974878
:1004E0008078704797480068806BC0F3036070475E
:1004F0000121814091488269114081617047012149
:1005000081408E48826922EA0101816170478B48EF
:10051000806970478948C0697047884910B5CC69BF
:10052000C8610246002381210720FFF76DF82046AD
:1005300010BD83488088C0F3802070477F480079D1
:10054000704702283CBF7D49086220B1012818BFCE
:10055000704709F0D9BA09F04FBA7848006A704775
:10056000FCF70AB810B5FCF707F87449896A8842A5
:1005700014BF0120002010BD71480079C0F3800035
:1005800070476F480079C0F3C00070476C4880889E
:10059000C0F3402070476A480079C0F3C01070472C
:1005A00067488088C0F34030704765488088C0F352
:1005B000C020704762488088C0F30030704770B533
:1005C0005F4E0446C0F340707568C5F34031884201
:1005D00005D014F0005F04BF0120F4F711FA14F005
:1005E000805F14BF45F4806025F4806014F0005FE4
:1005F00014BF40F4005020F400507060FCF736F84F
:1006000003F0A3F9002803BF4F4890F86C00C0081E
:10061000002003F0A3F9BDE87040EFF792BE484810
:100620004168002011F4806F18BF4FF0805011F422
:10063000005F18BF40F0005070472DE9F04140497D
:10064000044610F0040F4D68284614BF40F4807033
:1006500020F4807014F0080F14BF40F4007020F4F0
:10066000007014F0100F14BF40F4006020F400601C
:1006700014F0400F14BF40F4805020F4805014F068
:10068000200F14BF40F0800020F08000486000215F
:10069000C0F3002050B106F0D7FF64280FBF4FF021
:1006A000C041012101FA00F040F08041084606F007
:1006B000CEFFC4F38007C5F3002087422CD006F09C
:1006C0005CFF06463846EFF761FE0120F4F798F923
:1006D00016F4817F0CBF01200020F1F715FE16F003
:1006E000020F04D0022009F0C6F9002009E016F438
:1006F000807018BF012009F0BEF9134890F86C0013
:10070000C00803F02BF90D4A5078002818BF0428C0
:1007100002D1042190705170C4F3C000C5F3402190
:10072000884208BFBDE8F0810120F4F769F904F0C0
:100730000800BDE8F04109F033B9000074860010EC
:100740009832011048860010F82F0110F8484168CF
:10075000002011F0040F18BF012011F0080F18BF7E
:1007600040F0020011F4807F18BF40F0040011F443
:10077000007F18BF40F0080011F4006F18BF40F070
:10078000100011F4805F18BF40F0400011F0800F9E
:1007900018BF40F02000704703283CBFE54948617E
:1007A0007047E448007D7047E249C8737047E148EC
:1007B000C07B7047DF48406B7047DE49CA6A104310
:1007C000C862704770B5DB4EF06A40F000740020DC
:1007D000F062D748456815F0040F18BF44F00104D3
:1007E00015F0080F18BF44F0020415F4807F18BFFD
:1007F00044F0040415F4007F18BF44F00804FBF72C
:10080000BBFE002818BF44F0805415F4006F18BFD9
:1008100044F0100415F0800F18BF44F0200415F4C4
:10082000805F18BF44F0400415F4005F18BF44F027
:100830000054F16944EA0140002918BF40F080608B
:1008400070BDBC4908637047BA4890F8300000F0AA
:1008500001007047002818BF0120B6498872704710
:1008600070B50546B24800248088C0F3403070B1AE
:1008700006F0F5FE08280AD0AF4800EB0510C16865
:10088000AC48C26C91421CBF012101650124204685
:1008900070BD70B50546002406F06FFE10F4817F30
:1008A0000AD0A54800EB0510C168A248C26C91426D
:1008B0001CBF012101650124204670BD70B50546AD
:1008C000002406F0A8FA012817D1FBF755FE0128ED
:1008D00008D006F089FA012804D0F4F7AFFDB0F58E
:1008E000D77F0ADA9448012400EB0510C1689148CB
:1008F000C26C91421CBF01210165204670BD70B5DC
:1009000005460024F5F7A8FB50B18B4800EB051015
:10091000C1688848C26C91421CBF01210165012455
:10092000204670BD844A014602EB01110020CA68CE
:100930008049CB6C9A4208BF704701200865704718
:100940002DE9F041002486B02746A046F5F78CFA41
:100950007A49052808680CBF90F8EC0090F83C0034
:1009600000F00F052846FBF77CFF002818BFC06980
:1009700010F0010F18BF022603D10426F0F7C5FBC3
:10098000804646F400312846F5F7F2FB002804BF04
:1009900006B0BDE8F08118F0010F04BF2020EFF78A
:1009A000E7FF0120F0F744FEF1F77CFCFAF713F9BA
:1009B000012838D06846F1F7BEFE00282FD00198F4
:1009C000F3F7B6FB0298B8B101465D480BF01DFF86
:1009D0005B4A904209D05B4A5B4B014612781B7818
:1009E00052005A4356480BF070FE58480078492888
:1009F00004BF5348FAF70FFD049848B154485549CD
:100A00000078097808444200534804990BF05DFED1
:100A1000484901208872F1F7D6FE012703E0F5F777
:100A200085FA002CC2D0F1F701FAF5F7EBFC06B01D
:100A30003846BDE8F0813F48807A002818BF012081
:100A400070472DE9F04F4FF0000A89B006460F2499
:100A5000D146F5F709FA0546F5F70CFADFF8D4B0F8
:100A60000190052D07D1FBF7D5FA002804BF00201F
:100A70008BF80A0002D09BF80A0058B9F5F76BFB17
:100A800007464FF48050F5F763FBFFF759FF3846F0
:100A9000F5F75EFB052D0CBFDFF8C080DFF8C080E6
:100AA00021463046F5F764FB002804BF09B0BDE8D5
:100AB000F08F0BF073FE0BF076FEF3F74BFF0400A4
:100AC0007BD10126F0F721FB07460020F0F7B0FDAF
:100AD0001848022D066408BFF6F76CFE3046F1F7A1
:100AE000A6FBF2F741FFA6F1010BFAF774F8012813
:100AF0000AD0F5F7B9F9A84206D1F5F7BBF9019983
:100B0000884208BF002C2DD0F1F790F90848808862
:100B1000C0F3402000281CBF012008F041FF054E13
:100B200017F0010F757858D0012C4BD055E000001C
:100B30009832011074860010D0860010488600108C
:100B400080E90010E9840010EA8400106D8500102F
:100B5000EF840010EE84001070EF0010C536001016
:100B6000673C001002A8F1F7E6FD38B317F0010F5B
:100B700003D00120F3F744F9824602A8FAF710FFE8
:100B80000398F3F7D5FADDE90112284602F0EAFAF4
:100B900002A8C047044602F05BFBF1F714FE002CEC
:100BA000A3D116B9039858459FD1F1F73DF9002814
:100BB00004BF3046F1F73BFB97E73BE0FFE7F5F773
:100BC000AAF992E70120F3F71BF9504505D2AAEBE9
:100BD00000010120F3F724F98146F2F7ECFE17F04B
:100BE000010F27D0012C25D1B9F1000F22D0F0F749
:100BF0005BFC0446F0F79AFA00EB800004EB40003F
:100C00004844002144F20902904284BFA0F580408C
:100C10000938002D08BF43F6390103D0022D08BF63
:100C200041F6F901884205D2091A0120F3F727F9A4
:100C30000120F0710BF0BCFDF5F7E4FB09B0BDE855
:100C4000F08F2DE9F04F89B04FF000098046CDF8C4
:100C50000490CDF81090CDF82090CDF81C90F5F7C9
:100C600003F9CB46DA46CDF818B00590FE48047873
:100C7000FE480678FE4804FB06F70078462804BFC5
:100C80004046FAF7C8FB08EB4700054641460BF023
:100C9000BCFD0390804504D101467A0028460BF044
:100CA00014FDF34D28784B2804BF0398FAF7B3FBE3
:100CB000EF480078FF2805D07A0008EB8700ED495F
:100CC0000BF003FD07EB470008EB400502902346BD
:100CD0000096E8492846039A0BF08DFDE448007819
:100CE000492804BFE348FAF796FBE14800784C280E
:100CF00004BF2846FAF78FFB0598052836D1FBF785
:100D00009DF9012807D17A002946DB480BF0DDFC6C
:100D10000120FBF78DF9FBF788F938B30020014675
:100D20000090D148DFF850C30278D048007802FB29
:100D300000F30020002B19D935F810203CF810E002
:100D4000A2EB0E0212B2002AB8BF524212B28A427D
:100D5000C8BF1146401C9842EED36429DCBF0098FE
:100D6000002803D0FBF75DF9FBF76BF905EB4702B1
:100D70004FF0000C0092002E26D90021601E13D0E7
:100D800005EB400E35F810303EF802ECA3EB0E03F5
:100D90001BB2002BB8BF5B421BB222F810308B4253
:100DA000C8BF1946401EEBD10598022800F0E78025
:100DB000118005EB440502EB44025945C8BF8B4640
:100DC0000CF1010CB445D8D3AC48B0F91000039035
:100DD0008345A4BF4FF00109CDF80490DDF800C0B1
:100DE00000200CEB47030090002E26D90021601E46
:100DF000022812D90CEB40023CF8105032F802ECF9
:100E000032F8042C75442A4412B223F810208A4286
:100E1000C8BF1146401E0228ECD800201980588017
:100E200098800CEB440C03EB44035145C8BF8A4641
:100E30000098401C0090B042D8D3904AB2F91210EA
:100E40008A45A4BF4FF00109CDF81090B9F1000F09
:100E500014BF506D906D00F1010014BF5065906596
:100E600083480078FF287DD0029828F82090DDE99B
:100E7000010308EB830568800498A8800798E88040
:100E800008982881506DC31700EB13536FF30B03C1
:100E9000C01A6881906DC21700EB12526FF30B02FB
:100EA000801AA881A5F80EB0A5F810A0069868824F
:100EB0000398A882E982FBF7ADF8A883012006EB2E
:100EC00046014FF0020A00EB4103B9F1000F224640
:100ED0004146CDF800A00CBF4E204D20FAF7E8F9AE
:100EE000C7EBC70547F6FF7B28F815B0F6F7D2FC2D
:100EF00008EB450568806248006CC0F30820A880B4
:100F00006048D0F844030021C0F30B00E8800A22B7
:100F10000846F6F782F9288108EBC700B0F90810F7
:100F200009116981B0F90800C11700EB117121F0B6
:100F30000F01401A00EB80004000C11700EB117058
:100F40000011A881F6F72FFCE881A5F810B0C6EBD8
:100F5000C6056B1C224641464F20CDF800A0FAF78B
:100F6000A7F900E007E06B1C224641464720CDF878
:100F700000A0FAF79DF909B04846BDE8F08F02EBF2
:100F8000440030F9023C142BB9BF30F9040C14288A
:100F90004FF00109CDF804900AE73B4870472DE96E
:100FA000F84F834635483B490025B0F91080384852
:100FB0000978364C00782E46AA464718F1F70AF908
:100FC00000903548A4F264690078492804BF484677
:100FD000FAF7B8FB0020002F09D93BF8101039F8B8
:100FE0001020891A24F81010401C8742F5D8DFF829
:100FF000A89099F800004C2804BF2046FAF7A2FBFD
:10100000009810F4007FA7F1010012D000281CBF47
:101010001A49B1F9123026D034F910100029B4BFA2
:101020004A420A469A42BCBF0D44761C401EF3D188
:1010300019E000281CBF1149B1F9123013D004EB9C
:10104000400234F8101032F8022C891A09B224F840
:1010500010100029B4BF4A420A469A42BCBF0D4450
:10106000761C401EEBD119E0E9840010EA840010E0
:101070006D85001080E90010E4EF00107486001008
:10108000006000400050004070EF0010D4F50010E8
:10109000EF840010EE84001073850010002EC8BF8E
:1010A00095FBF6F52EB2268099F800004F2804BF74
:1010B0002046FAF747FB0025781E0ED034F81010B2
:1010C000891B09B224F810100029B8BF494209B29F
:1010D0008D42B8BF0D46401EF0D1258006F04DFA76
:1010E00010F4817F18BF4FF00508454506DD99F8DB
:1010F00000004FF0010A4D2807D103E099F80000E5
:101100004E2802D12046FAF71DFB99F80000472827
:1011100004BF2046FAF716FB5046BDE8F88F2DE9CC
:10112000F04F87B0FBF7E8F9BE4C2068B0F91E100D
:10113000B0F91C000BF00FFB0120F3F761FC06F087
:101140001CFA10F4817F14BF00200120F1F7DCF8B5
:10115000DFF8D49299F8180010F0100F06D0042090
:1011600000F01AF90F2818BFF3F730FC07F08FF9D9
:1011700004F08CFCFF2089F806004FF0FF3005F0EA
:1011800064FE06F0ACF94FF0000A89F80EA089F869
:101190000DA089F80CA05046F4F738FAF4F764FE75
:1011A000022840F0EB8099F801709E4AC9F838A0F7
:1011B000C9F83CA01068BB000024C06BA046C0F377
:1011C0000321D84000F00F058D4204BFDFF85CB268
:1011D000C9F850A025D193480068C16B0BEB0410EF
:1011E00002799200D14001F00F060F2E04D08168E1
:1011F00020468847012807D0641C052CEBD3D9F87A
:10120000500001280BD102E03546A046F7E70BEB72
:101210000810C068C9F84C000020F3F7F1FBC9F8CA
:10122000485039460220FEF7D6FA052F5FD2DFE894
:1012300007F09103030395000F2199F801602846F8
:10124000F4F796FF002852D00BF0A8FA0BF0ABFA97
:10125000F3F780FB05003FD199F8000000281CBF80
:101260000001F0F735F97248F0F729FE0024F0F795
:10127000B1FF0690EFF749FF10F0010F0FD0F0F724
:10128000D1F902280BD399F8070040B1069840F431
:101290000030F0F776FE0124F1F704F801E0F0F7F2
:1012A000ADFF89F807A0F3F7D3FBF4F7D4F8F4F710
:1012B000A7F8DFF88081DFF880B14FF0E027F9F779
:1012C0008AFC012808D0F4F7CFFD022802BF99F864
:1012D0000100B042002D0BD00020F0F7F0FDF2F736
:1012E0005FFE0BF060FA0BF063FAF5F78BF838E06D
:1012F0006846F1F720FA18B32CB1641E0698F0F78F
:1013000040FEF0F77BFF6846FAF74AFB0198F2F7D8
:101310000FFFF4F7A9FD3146009A01F023FF68465C
:101320000BF078FA054601F093FF98F8000020B121
:10133000B869CBF80000C7F810A0F1F744FABEE78F
:10134000386910F0010F02D0F4F7E5FDB7E7F4F7C4
:10135000EDFDB4E728460BF035FA02E02846FFF72A
:1013600070FBF9F738FC012803D1F4F77DFD022862
:1013700004D1F4F779FD02283FF415AF08F0BBFF64
:10138000F3F73DFB07B0BDE8F04FFBF7B5B84A00F7
:1013900001462A480BF099B92DE9F047DFF884A0FF
:1013A00002469200DAF8000000242746C06BC0F322
:1013B0000321D04000F00F068E421CBF3046BDE82E
:1013C000F0870020DFF8609009F15C08C9F8500050
:1013D000DAF80000C16B08EB041002799200D140EA
:1013E00001F00F050F2D04D08168204688470128A1
:1013F00007D0641C052CEBD3D9F8500001280BD181
:1014000002E02E462746F7E708EB0710C068C9F848
:101410004C000020F3F7F4FA3046C9F84860BDE804
:10142000F08700004886001074860010D0860010F7
:10143000B5430010278400108C84001070EF00105A
:101440003A4A30B4146894F86CC01CF0040F1ABF08
:10145000012222EA0C050CF00105B0F90030B1F9C7
:1014600000201DB1E58AAA1A521E12B21CF0020F0A
:1014700003D0A48AE31A5B1E1BB21CF0040F19BF31
:1014800002800B8003800A8030BC70474FF6FF71EA
:10149000A0F87010A0F87210A0F87410A0F87610E0
:1014A00070472DE9F05F16468A46834606F027F816
:1014B000074606F01AF8002500F1D309002E8CBF6C
:1014C0004FF6FF78BDE8F09F05EBC50000EB40004C
:1014D00007EBC00494F8C40010F0010F0DD0A4F87D
:1014E0007080A4F87280A4F87480A4F876802346F3
:1014F0004A465146584602F047FFD4F8CC0002282D
:1015000018BF03280DD0B4F87000A4F87400B4F824
:101510007200A4F87600681CC5B2B542D4D3BDE809
:10152000F09F204600F00FFFF5E70000088800104C
:10153000FC4948707047FB4840787047F94800788C
:10154000002818BF01207047F748006890F8700025
:1015500000F001007047F44909680A6F60F3000267
:101560000A677047F04B10B4D3F800C0BCF81230D3
:1015700003FB00F4BCF81A005943B4FBF0FCB1FBC8
:10158000F0F10CFB0CF4DFF8A4C34943CCE90841AB
:1015900003FB02F1B1FBF0F04043CCF8280010BC93
:1015A000704710B44FF6FF7C0CEA0024DF480CEAC9
:1015B0000121C48501860CEA022141860CEA03213F
:1015C000818610BC70472022D84906280ED2DFE859
:1015D00000F00D030D05080A102000E0402088856A
:1015E00070478020FBE74FF48070F8E78A857047EA
:1015F00010B5032208211120FFF7B4FFCA4C0A23BB
:101600001422206890F87400C0F3031100F00F005A
:10161000FFF7C7FF2068B0F87400BDE81040C0F3C2
:101620000330D0E72DE9F04190460D46044605F021
:101630005CFFBF4847190A384619BB4DD4B1012C8D
:101640003DD0022C50D0032C78D0042C75D0052C22
:1016500018BFBDE8F081032208211120FFF782FFA7
:1016600028680A231422406F0221C0F30340FFF7C9
:1016700098FF1CE0032208211120FFF773FF16F8E2
:10168000010C002801BF17F8010C0028D8F8CC0085
:10169000032828684FF00A034FF0140290F87400F2
:1016A000C0F3031100F00F00E1D1FFF77AFF2868C3
:1016B000B0F87400BDE8F041C0F3033083E70322C3
:1016C0001D211E20FFF74EFF28680A231422B0F8C0
:1016D0007400C0F3032100F00F00491CFFF761FF05
:1016E000BDE8F04104206EE716F8010C012804BFA4
:1016F00017F8010C01284FF0080219BF22212320FE
:1017000018211920FFF72EFF16F8010C022828686F
:10171000406F18BFC0F30351C0F303404FF00A03FA
:101720004FF0140208BF0321FFF73BFF2868406F0A
:10173000BDE8F041000F46E700E00DE008221D2162
:101740001E20FFF70FFF28680A231422B0F8740048
:10175000C0F3032001468AE708221D211E20FFF75F
:1017600001FF0A2314220321022080E710B56E4CEA
:1017700003222068418A408BC1EBC1014900B1FBC3
:10178000F0F068494043886008211120FFF7EAFE25
:1017900020680A23142290F87400C0F3031100F0AB
:1017A0000F00FFF7FEFE2068B0F87400BDE810409F
:1017B000C0F3033007E75D4B03EB400003898B4226
:1017C00088BF991A38BF991808BF704701817047C0
:1017D0002DE9F04F83B09B460E46044605F085FE8A
:1017E000029005F0A2FE84464F4894F85C504D4BA1
:1017F00000684E4A418A408B01EB4101C900B1FBB0
:10180000F0F0D4F8CC10404302291CBF94F87E10AD
:1018100001290FD0474901EBC50151E90278616DFB
:10182000B6F800900229B6F802A0D4F8981013D0A8
:1018300039B336E0002102EB05093788B6F802809B
:1018400009F8011C02EB450AB2F83490AAF8089096
:10185000012D08BF1970E2E719B394F85D1001EB90
:10186000C10101EB41010CEBC101D1F89810C1B9E4
:1018700002EB4501B2F830C0B1F808E0E64510D9F6
:101880000DE083450DD3D4F8CC10022909D002EB2A
:101890004501B2F830C0B1F808E0E64501D9A1F839
:1018A00008C0B4F8C41011F4006F04BFD4F8981045
:1018B000002903D1834538BF918E00D3518E5186C4
:1018C000D4F898C0BCF1000F05D183450DD3D4F8EE
:1018D000CC00022809D0614601911878002804BF85
:1018E000012DBCF1030F0BD101E00221F4E701202F
:1018F00018700E484189108E814284BF0B4948817F
:101900000A4A0C990198136A5B4503D8022801D052
:10191000012911D0054A526A5A452FD902283ED1D1
:101920002CE00000208700100888001098F60010B6
:10193000DAF6001048F60010FEF732FE012807D054
:10194000D4F89C00032804BF94F87F00002809D035
:10195000FE490120294401F8010C04200021C4F8AB
:101960009C003FE0F9490220294401F8010C0320C2
:10197000C4F89C0094F87F00401C25E079B1F3493D
:101980005A4598BF9B4535D2022835D0002084F8AF
:101990007F00481910F8011C032926D033E0FEF718
:1019A000FFFD012807D0D4F89C00042804BF94F858
:1019B0007F0000280BD0E5490220294401F8010CE2
:1019C00003210020C4F89C1084F87F001BE0DF494D
:1019D0000120294401F8010C0421C4F89C1094F85A
:1019E0007F00411C84F87F100DE0022100F8011CEB
:1019F000032006E0022806D12944032001F8010C47
:101A00000220C4F89C0005F070FDDFF840C30346D7
:101A10000CEB0502BCF82C00009012F8012CBCF86D
:101A20003010BCF82EB0BCF83200022A04D0012AD3
:101A30001CD0032A2FD033E00CEB450001EB410B07
:101A400002895A4507D993F80CE0BEF1000F08BF90
:101A5000A0F808B005D08A4203D91A7B002A18BF23
:101A600001812846009AFFF7A6FE19E00CEB45021B
:101A70001089884209D9411AA0EB6100000A4FF68B
:101A8000FF7101EA002010810AE059462846009AB9
:101A9000FFF791FE04E001462846009AFFF78BFE0F
:101AA0000CEB45000289002A04BF0020014620D02B
:101AB0001046B2F5807F36BF4FF4807101464FF477
:101AC0008072A348019B022B25D094F85CC00023B0
:101AD0000CF80030A1F58070784300EB0920B0FBD2
:101AE000F1F0A2F5807101FB08F101EB0A21B1FBD5
:101AF000F2F194F85C30974A02EBC30343F8080C08
:101B000094F85C3002EBC30242F8041CB080F18010
:101B100003B0BDE8F08F94F85CC01CF80030FA2BDD
:101B20003CBF5B1C0CF8003094F85C30185C3C281F
:101B3000D0D30298090A120A90F84A00022886486F
:101B4000006816D3B0F818B0058A0BFB09F3B0F89B
:101B50001AC0408A0CFB0AF9B3FBF5F30BFB07FA3A
:101B60000CFB08FCB9FBF0F9BAFBF5F5BCFBF0FC8B
:101B700015E0B0F814B0058A0BFB09F3B0F816C0F5
:101B8000408A0CFB0AF9B3FBF5F30BFB07FA0CFBDD
:101B900008FCB9FBF0F9BAFBF5F5BCFBF0FCA1F1D0
:101BA000010000FB0530B0FBF1F3A2F1010000FBE6
:101BB0000C90B0FBF2F268480168B1F8109009FB94
:101BC00003F009D3B1F81890B1F812A0B0FBF9F006
:101BD0000AFB02F9498B08E0B1F81490B1F812A0A1
:101BE000B0FBF9F0C98A0AFB02F9B9FBF1F1AB428B
:101BF00018BF62457FF47DAFAB4208BF38466245EF
:101C000008BF414675E72DE9F04F90F85CC08FB0F2
